:1000000000000220057700002D7700002F77000008
:1000100031770000337700003577000000000000E2
:100020000000000000000000000000003777000022
:1000300039770000000000003B7700003D770000AA
:100040003F770000B9540000C97A00003D760000F7
:10005000317600003F7700003F7700003F770000D7
:10006000053600003F7700003F7700003F77000033
:100070003F7700003F7700003F7700003F770000A8
:100080003F7700004D7B00003F7700003F77000086
:100090003F7700003F7700003F7700003F77000088
:1000A0003F7700003F7700003F7700003F77000078
:1000B0003F7700003F7700000000000000000000D4
:1000C0003F7700003F7700003F7700003F77000058
:1000D0003F7700003F7700003F7700003F77000048
:1000E0003F7700000000000000000000000000005A
:1000F000000000003F770000000000003F77000094
:1001000000000000000000000000000000000000EF
:1001100000000000000000000000000000000000DF
:1001200000000000000000000000000000000000CF
:1001300000000000000000000000000000000000BF
:1001400000000000000000000000000000000000AF
:10015000000000000000000000000000000000009F
:10016000000000000000000000000000000000008F
:10017000000000000000000000000000000000007F
:10018000000000000000000000000000000000006F
:10019000000000000000000000000000000000005F
:1001A000000000000000000000000000000000004F
:1001B000000000000000000000000000000000003F
:1001C000000000000000000000000000000000002F
:1001D000000000000000000000000000000000001F
:1001E000000000000000000000000000000000000F
:1001F00000000000000000000000000000000000FF
:1002000010B5054C237833B9044B13B10448AFF350
:1002100000800123237010BD400200200000000078
:10022000DCCF000008B5034B1BB103490348AFF313
:10023000008008BD0000000044020020DCCF000068
:10024000154B002B08BF134B9D46A3F5803A0021A8
:100250008B460F461348144A121A09F0F9FE0F4B49
:10026000002B00D098470E4B002B00D09847002061
:10027000002104000D000D48002802D00C48AFF307
:10028000008009F09DFE2000290007F075FC09F0B0
:1002900071FE00BF00000800000002200000000006
:1002A0000000000040020020048E01200000000039
:1002B0000000000010F0010310D104280CD90368DD
:1002C000C3F30F1343B1013B9B001A1DC1180979F9
:1002D00011B101339342F9D1184670470023FBE76F
:1002E000037883B11A0601D40130704703F0C003CC
:1002F000C02B08BF0130024610460132037803F0DC
:10030000C003802BF8D0704708B5002103780BB9E3
:10031000084608BDFFF7E4FF0131F7E738B50022D2
:1003200004460D46411C092003F0A0FC40B16300C7
:10033000024643F0010342F8043F0023A34200DBDE
:1003400038BD55F8231042F8041F0133F6E70128A1
:1003500038B504DC1C20BDE8384001F0DBB80D687E
:10036000EA0701D41120F6E74868C30706D4042839
:1003700004D9036803F00F03042B01D00E20EAE731
:1003800003F0D8FA6D10002D044603DDFFF7BCFF23
:10039000A84206DA1220DEE72046FFF7A1FF013D62
:1003A0000446012DF8D120787F2808DDDF280ADCFB
:1003B0006378800100F4F86003F03F0318434000C5
:1003C00040F0010038BDEF280ADC637800039B0190
:1003D00080B203F47C630343A07800F03F00EDE7B4
:1003E000F72810DC637880041B0303F47C3300F4EB
:1003F000E0101843E37803F03F030343A078800143
:1004000000F47C60DAE74FF0FF30D8E7486838B591
:10041000C3070D4606D4042804D9036803F00F026D
:10042000092A04D00B20BDE8384001F073B84468B5
:10043000C3F30F1364105A1EA2420BD8032194FB7E
:10044000F1F16429A8BF64210329ACBF5918D91C54
:1004500003F048FC0368C3F30F13013B9C4208D22E
:10046000A31C013464002A6840F8232044F00104EE
:100470004460002038BD01282DE9F84304DC1C202D
:10048000BDE8F84301F046B802284E680CD08C68ED
:10049000E70709D56410012CB8BF0124F50705D57D
:1004A0004FF0FF30BDE8F8830124F7E7042EF7D9B9
:1004B00033680D6803F00F02042A2DD1E80706D433
:1004C000042D04D92B6803F00F03042B01D00E2058
:1004D000D6E73046FFF7EEFEA042E1DB304603F000
:1004E00029FA0646284603F025FA013C0146301950
:1004F0000AF07DF901460028D2D0012433780BB1EF
:100500008E4203D3640044F00100CBE73046FFF78E
:10051000E7FE01340646F1E7092A34D177687F10F7
:10052000BC42BDDCE90725D4042D23D92B6803F098
:100530000F03042B1ED1284603F0FCF9804604F17A
:10054000010956F829008542DCD0C2070ED40428E0
:100550000CD9036803F00F03042B07D103F0EAF969
:10056000014640460AF00AF90028CBD0B9454C466E
:10057000E5DD95E7631C56F82320AA42C2D0BB42B2
:100580001C46F7DD8CE7032A8AD1C3F30F17C3F3A8
:100590004173C3EB8707BC4282DCEB072AD4042DEE
:1005A00028D9286800F00F03032B19D1C0F30F13CB
:1005B000C0F3417005F10408C0EB83003F1A013C11
:1005C00040440336BC423FF76BAF32194346834287
:1005D000194611D317D10134600040F0010061E7E2
:1005E000042B07D1284603F0A5F980462846FFF7DB
:1005F00061FEE3E70F2043E712F8015F09788D42BF
:1006000003F10103E3D00134DCE708B503F076F928
:10061000400040F0010008BDC30711D404280FD9E1
:10062000026802F00F03032B0AD101F00303C3F1A8
:1006300004035B0703F0C04322F0C042134303608E
:10064000704701282DE9F0470546884604DC1C2048
:10065000BDE8F04700F05EBF4C6814F0010701D11F
:100660000D20F5E7022802D08B68DA07F8D5D8F814
:100670000060F30700F1A980042E40F2A6803268E2
:100680006410012C02F00F03B8BF0124092B28D1FC
:100690007668022D4FEA660605D0D8F808305B1060
:1006A0009E42A8BF1E46351B0135012225EAE5758D
:1006B000A918092003F0DAFA074648B16D0003468D
:1006C00045F00105D8F8002043F8045FA64202DA9D
:1006D0003846BDE8F087013452F8241043F8041F6F
:1006E000F4E7042B43D1304603F024F9FFF70CFE66
:1006F000022D824605D0D8F808305B109842A8BF7A
:100700009A46A24504DA0020BDE8F04703F028BB72
:10071000304603F00FF90546A74222DB304603F0CE
:1007200009F9A94606462846FFF7DAFD0134A24535
:100730000546F8DAA0EB0905284603F011FB074649
:100740000028C5D003F0F6F80446D8F8000003F0FE
:10075000F1F8A9EB060101442A46204609F054FCB1
:10076000B6E72846FFF7BCFD01370546D4E7032B63
:100770002BD1C2F30F13022DC2F34172C2EB8302DD
:1007800005D0D8F808305B109A42A8BF1A46A2429A
:1007900006DA002211460320BDE8F04703F066BAEE
:1007A000151B0423291D002291FBF3F1032003F004
:1007B0005DFA074600288BD001352946FFF72CFF4C
:1007C000E11C2A4631440430C8E7212040E70028D4
:1007D000F8B504DC1C20BDE8F84000F09BBE0C68B6
:1007E00014F001060FD0641024EAE474E11C002226
:1007F0008910032003F03AFA054610B12146FFF7AD
:100800000BFF2846F8BD042C01D80025F9E7256820
:1008100005F00F05042D19D12046FFF74BFD324698
:10082000C11C074691FBF5F1032003F01FFA0546B2
:100830000028E6D03946FFF7EFFE204603F07AF8AD
:100840003A460146281D09F0DFFBDAE7092DDCD125
:1008500067687F100423F91C324691FBF3F10320F3
:1008600003F004FA05460028CFD03946FFF7D4FE3E
:100870000434BE42C5DA54F8043FDA0742BFAA196D
:10088000A3F3480313710136F3E77F2902DC0170FB
:1008900001307047B1F5006F0CDA03468A1162F03F
:1008A0003F0203F8022B01F03F0161F07F0141702C
:1008B00018467047B1F5803F0FDA0B1363F01F0342
:1008C0000370C1F3851301F03F0163F07F0361F012
:1008D0007F014370817003307047B1F5883F0DDAB6
:1008E000F0230370902343708B1101F03F0163F0FC
:1008F0007F0361F07F018370C17004307047000096
:100900000028F7B50F4603DC1C2000F003FE0CE0C6
:100910000A6812F001000AD06C4651102046FFF719
:10092000B4FF011B204603F022FA044616E0042A15
:100930003BD9136803F00F03092B36D155681C49C6
:100940006D100124AC420CDD03F00AFA044628B114
:100950003F6802F0EFFF0126AE421DDD204603B0E6
:10096000F0BD013452F8243013F0010601D10D20FE
:10097000CBE75B107F2B09DDB3F5006F08DBB3F528
:10098000803F07DB8B42D4BF042600263044D9E7E2
:100990000226FBE70326F9E7013657F82610CB07B6
:1009A000E5D54910FFF771FFD6E72120ADE700BF7D
:1009B000FF0F010010B5044611F0010011D1042908
:1009C0000ED90B6803F00F03042B09D1084602F07F
:1009D000B1FF0146204609F0D1FEB0FA80F040098F
:1009E00010BD0020FCE700000128F8B50E4604DC2D
:1009F0001C20BDE8F84000F08DBD4D6815F00107E2
:100A000006D1042D04D92B6803F00F02092A01D066
:100A10000B20EEE76C6809681F486410C3F30F13DE
:100A2000A34298BF03F1FF34FFF7C4FF40B1012395
:100A3000BC4201DA0020F8BD013745F82730F7E75E
:100A400031681648FFF7B6FF50B1002CF2D0631C96
:100A50000122013C944045F8232014436C60E9E7EF
:100A60003368DA0701D40D20C3E75B10002B0DDDDE
:100A70009C420BDB05EB830305EB84029A4207D112
:100A80000123013C9C4053601C43E7E71220B0E780
:100A9000996843F8041FF1E7F7B60000FBB60000C1
:100AA000002310B50B70C3070C4606D50E49421043
:100AB0002046BDE8104009F025BE28B90B49204664
:100AC000BDE8104009F03EBE042801D10849F6E710
:100AD00009D9036803F00F03042B04D102F02AFFA5
:100AE00004490246E4E710BDC4C1000000B700009D
:100AF00006B700000BB700002DE9F04301288FB0C6
:100B000081460E4607DC1C2000F004FD0546284601
:100B10000FB0BDE8F0830B6813F0010440F0A18032
:100B2000042B40F2D5801B6803F00F03092B40D142
:100B3000274656F8273013F0010806D1042B04D9B4
:100B4000186800F00F00092801D02220DCE75B685C
:100B50000137B94504EB6304EBD10122A11803F07E
:100B600085F8054608B90025D1E7640044F0010482
:100B70004460424600F1080456F822104B680868A9
:100B80005B10C0F30F10984298BF00F1FF3304319F
:100B90000020834207DC013223EAE373BA4204EB0C
:100BA0008304E9DBB3E751F804CF44F820C00130F7
:100BB000EFE7032B40F08C80274656F8270010F013
:100BC0000108C2D10428C0D9036803F00F02032A28
:100BD00038D1C3F30F12C3F34173C3EB82031C4438
:100BE0000137B945E9D10423E11C002291FBF3F15F
:100BF000032003F03BF805460028B4D02146FFF758
:100C00000BFD00F1040956F82840E10720D4042C1C
:100C10001ED9206800F00F03032B19D1C0F30F1366
:100C2000C0F34170C0EB830003344B46A3EB0902D1
:100C3000824211DB08F101080028A8BF8144B845B1
:100C4000E1DB64E7042A80D1FFF734FB0444C7E703
:100C50002046FFF72FFBE7E714F8012F03F8012BDD
:100C6000E4E700252C4656F82500C20732D40428B4
:100C700030D9036803F00F02042A32D1FFF71AFBC0
:100C800004440135A945EED1204603F069F8054634
:100C900000283FF468AF041DB04606EB890958F8F8
:100CA000046BF30728D4042E26D9336803F00F020F
:100CB000042A34D13046FFF7FDFA0746304602F0E9
:100CC00039FE3A460146204609F09EF93C4421E0AF
:100CD0002546C8E701A9FFF7E3FE01A809F058FD82
:100CE000CEE7032A7FF431AFC3F30F12C3F341738E
:100CF000C3EB82031C44C4E701A93046FFF7D0FED2
:100D000001A809F045FD01A906460246204609F062
:100D10007BF93444C145C2D100232370F7E6032A8E
:100D2000F8D1C3F30F17C3F34173C3EB87073A46F8
:100D3000311DC8E72DE9F04F002893B00F4607DCBE
:100D40001C2000F0E7FB0546284613B0BDE8F08FF5
:100D50000D6815F0010806D1042D04D92B6803F0A5
:100D60000F03092B01D00B20EBE76E687610002EE5
:100D700003DC404602F0F4FFE5E7012826D048688E
:100D8000C20723D4042821D9036803F00F03042BDE
:100D90001CD102F0CFFD0446204609F0F9FC0435D1
:100DA000731E8146009303FB00FB05EB860A55F892
:100DB000040FC30771D404286FD9036803F00F022E
:100DC000042A05D1FFF776FA83440AE0384CE3E7BA
:100DD000032A69D1C3F30F12C3F34173C3EB820338
:100DE0009B44AA45E3D1584602F0BAFF05460028C5
:100DF000AAD0D7F800A0B9F1000F03D0786802F0AC
:100E000099FD0446284602F095FD0AF104030746C1
:100E10000193019B53F804AF0193504602F08AFD01
:100E20001AF001030146029302D1BAF1040F04D86B
:100E300005A95046FFF734FE05A90846039109F0BD
:100E4000A7FCDDE9023183468BB9BAF1040F0ED954
:100E5000DAF8000000F00F0CBCF1030F01BFC0F383
:100E60000F13C0F341700AF10401C0EB830B384645
:100E70005A4609F0C9F85F44B9F1000F08D0009B49
:100E8000434505DD38464A46214609F0BDF84F4442
:100E900008F101084645BCD156E705A9FFF700FE59
:100EA00005A809F075FC8FE702F044FDF9E700BFE3
:100EB000B2BB0000002810B511DD0B6813F001046F
:100EC00002D05C1024EAE4740122A118092002F087
:100ED000CDFE18B1640044F00104446010BD00244C
:100EE000F2E70A6838B512F0010436D1042A34D981
:100EF0001368496803F00F00092818D15068C3F33C
:100F00000F134010834298BF03F1FF30151DA0421C
:100F100005DC01330220984205DB002038BD45F88E
:100F2000041F0134F3E742F820100130F3E70328EF
:100F300013D1C80704D41320BDE8384000F0EABA42
:100F40004910FF29F7D80432C3F30F1302EB8303D0
:100F50009A42E2D202F8011BFAE70B2000F0DAFA1B
:100F6000DBE700002DE9F0414E6816F001078846E6
:100F700028D1042E26D9346804F00F03092B11D18F
:100F80007568C4F30F146D10AC4200D8651ED8F814
:100F90000010CB071AD54C10002C01DDA54220DA39
:100FA000122034E0042B04D13046FFF783F90546C4
:100FB000EDE7032B08D1C4F30F15C4F34174C4EB60
:100FC0008505E4E70025E2E73D46E0E72848FFF72E
:100FD000F1FCA8B109F02EFB90FBF5F404FB15041D
:100FE0000134002F41D1042E3FD9336803F00F03A1
:100FF000092B12D1013456F824402046BDE8F08177
:10100000D8F800101B48FFF7D5FC20B91120BDE827
:10101000F04100F07FBA2C46E3E7042B1DD13046A7
:1010200002F088FC012C05460FDCFFF759F9461B3E
:10103000304602F095FE04460028DED002F07AFC2D
:101040003246294608F0E0FFD7E72B78013C002B19
:10105000A6D02846FFF744F9E4E7032B05D1344432
:10106000E478640044F00104C7E70B20CFE700BF39
:10107000F0B60000FBB600002DE9F0414C6814F01A
:10108000010688462ED1042C2CD923688F6803F0E2
:101090000F02092A13D16568C3F30F136D10AB4219
:1010A00000D85D1ED8F800102848FFF783FC68B30D
:1010B000236803F00F03092B1ED1012317E0032A35
:1010C00010D1FA0704D41320BDE8F04100F022BA91
:1010D0007E10FF2EF7D8C3F30F15C3F34173C3EB94
:1010E0008505DFE70B20EFE7013344F823709D42CD
:1010F000FADA0020BDE8F081032BFAD10334012392
:101100009D42F6DB04F8016F0133F9E7D8F80010CF
:10111000CB0706D54910002901DD8D4208DA1220DF
:10112000D2E70B48FFF746FC08B91120CCE7294667
:10113000236803F00F03092B03D1013144F8217018
:10114000D7E7032B04BF6418E670D2E7F7B60000B8
:10115000FBB60000086808B5C3071BD4042819D9DA
:10116000036803F00F02092A01D1406808BD032A71
:1011700009D1C3F30F12C3F34170C0EB82004000EA
:1011800040F00100F2E7042A04D102F0D3FBFFF79C
:10119000BBF8F4E70120E9E7024A03480B2104F019
:1011A00055BA00BF98B6000090B600000020704706
:1011B0000420704701207047002002F0D1BD0020BC
:1011C00070470020704700207047002070470020C3
:1011D00070470020704700207047002070470000D3
:1011E000024A03480C2104F031BA00BF80B7000066
:1011F000E0B700007047037883B11A0601D40130CC
:10120000704703F0C003C02B08BF013002461046F0
:101210000132037803F0C003802BF8D07047000040
:10122000F8B511F0010506461446084626D10429F2
:101230003FD90B6803F00F03042B3AD1D30714D422
:10124000042A36D9136803F00F03042B31D102F0BE
:1012500071FB0546204602F06DFB0146284609F069
:101260008DFA00282DDB1ED126E002F063FB294613
:101270000A2209F051FB0546601011E012F0010747
:1012800015D1042A15D9136803F00F03042B10D1CC
:1012900010464D1002F04EFB0A22394609F03CFB85
:1012A00085420EDB08DD002E09DC00200CE04D102D
:1012B000E2E7064B0F221A700136022EF5D8042001
:1012C00002E0701700F00400F8BD00BF80020020AB
:1012D0002DE9F0412B4F06460024E500EB191B7960
:1012E000032B07D00134FF2CF7D14FF0FF342046F9
:1012F000BDE8F081304609F04BFA31460246E0B2D3
:1013000004F0E0F90028F2D1EB5959681A1D88421F
:10131000E8D052F8045FF02D00F10100F7D1800011
:1013200008301A18D107DDD4042ADBD91B5803F082
:101330000F010429D6D1C3F30F13013302EB83004D
:10134000C507CFD40428CDD952F8233003F00F03BA
:10135000042BC7D102F0EEFA4FF00308054609212D
:10136000284609F0FEF90028BCD0B8F1010800F1C8
:101370000105F4D13146284609F039FA8542B6D044
:10138000B0E700BFD883012010B510F0010402D0EF
:101390004410204610BD042812D9026802F00F0242
:1013A000042A07D102F0C6FA0A222146BDE81040FD
:1013B00009F0B2BA032A03D10A2221460430F5E724
:1013C000014B0D221A70E4E78002002010F00102A8
:1013D00010B516D1042802D90268C2F30F1211F019
:1013E000010310D1042902D90B68C3F30F139342F0
:1013F00016D1043000EB83020331904205D3012063
:101400000BE00022EBE70023F1E710F8014B11F8A5
:10141000013F1CB9B3FA83F0400910BD9C42ECD0E7
:101420000020FAE72DE9F74F804689469A46304F6B
:10143000304E6AB102233B70012333603368DFF81A
:10144000D0B00024FC54444504DB03B0BDE8F08F69
:101450003260F3E759F824003168C30707EB010550
:10146000C1F5487105D5244A4310284609F016F9FC
:1014700004E0C8B9214A284609F010F91C4809F0CF
:1014800087F93060BAF1000F0CD008F1FF33A342A6
:1014900008DDB0F5487F05D2431C20223A540022D3
:1014A000FA5433600134CEE7042801D1144AE2E74C
:1014B0001BD9026802F00F03042B06D1019102F040
:1014C00039FA104A01990346CFE7092B03D1436843
:1014D0005A465B10C9E7032B08D1C2F30F13C2F3BE
:1014E0004172C2EB8303084ABFE70123074ABCE706
:1014F00081020020A4050020C4C1000000B7000044
:1015000006B70000EFC700005FBA00006ABA00002B
:1015100050BA0000014B1870002070478002002074
:1015200010B501F009FF084C231D01461F22184683
:1015300009F048F909F02CF904308008000140F066
:1015400004002060204610BD5C0200202DE9F04F11
:1015500085B000F1180104690291D0E90232824697
:1015600001EB8404C34F4169029800EB810939788B
:1015700003EB820529BB53F82230BF4A1E1203F049
:101580007F03043552F82330904643F00103184797
:101590009AF8010004F0C0FC00238AF8003021E032
:1015A0003B7873B92B681E1203F07F03043558F89B
:1015B0002330EAE7029A231D9A1AD82A26DD1A2335
:1015C0003B70DAF808209AF8023039789AF801006E
:1015D000AA1A921043EA022204F0A4FC00238AF81B
:1015E00000303B70DAF80830ED1A029BE41AA9EBE0
:1015F0000309AD10A4104FEAA903CAF80C50CAF8A9
:101600001040CAF8143005B0BDE8F08F22461C46E1
:101610003B781660002BD4D12B681E1203F07F0399
:10162000043558F82330B0E7029A231D9A1AD82AB5
:1016300002DD1A233B70C4E721461C462B680B6071
:101640003B782A1D0BB11546BBE76B681E1203F0F1
:101650007F03083558F8233097E7029A231D9A1A1A
:10166000D82A02DD1A233B70ABE722461C463B78A2
:1016700005EB86061660002BA3D12B681E1203F023
:101680007F03043558F823307FE7029A231D9A1A06
:10169000D82A02DD1A233B7093E722461C46774B7B
:1016A00053F8263013603B78002B8AD12B681E122A
:1016B00003F07F03043558F8233066E76F4B54F886
:1016C000042D43F826203B78002B7FF47AAF2B685B
:1016D0001E1203F07F03043558F8233055E7674B9B
:1016E000009353F82600FFF74FFE834654F8040D8D
:1016F000FFF74AFE5844009B400040F0010043F8C9
:1017000026003B78002B7FF45CAF2B681E1203F0A1
:101710007F03043558F8233037E7029B221DD31A84
:10172000D82B02DD1A233B704BE7029B21464B4529
:1017300034BF59F80C3C01230B603B781446002B56
:101740007FF43FAF2B681E1203F07F03043558F877
:1017500023301AE7029B221DD31AD82B02DD1A234D
:101760003B702EE7029B4B4518D259F80C3C06F112
:1017700080465B10C3EB8373033E334459F8233038
:1017800023603B781446002B7FF41BAF2B681E129E
:1017900003F07F03043558F82330F6E618233B7036
:1017A0000023EDE7029B4B4518D259F80C3C54F846
:1017B000042D5B1006F18046C3EB8373033E334474
:1017C00049F823203B78002B7FF4FBAE2B681E12D8
:1017D00003F07F03043558F82330D6E618233B7016
:1017E000F0E7029B4B4529D259F80C3C06F18046A4
:1017F0005B10033EC3EB8373334459F82300FFF7B8
:10180000C3FD834654F8040DFFF7BEFD59F80C3CA8
:101810005B10C3EB837358441E44400040F001004A
:1018200049F826003B78002B7FF4CBAE2B681E12C4
:1018300003F07F03043558F82330A6E618233B70E5
:10184000F0E7029A231D9A1AD82A02DD1A233B7068
:10185000B7E622461C4659F8263013603B78002B29
:101860007FF4AFAE2B681E1203F07F03043558F8E7
:1018700023308AE68002002050B80000D08B01207F
:1018800054F8043D49F826303B78002B7FF499AE9C
:101890002B681E1203F07F03043558F8233074E6DA
:1018A00059F826004FEA600B54F8040DFFF76CFD61
:1018B000584440003B7840F0010049F82600002BD6
:1018C0007FF47FAE2B681E1203F07F03043558F8B7
:1018D00023305AE6029BA4EB8604A3420BD83B7844
:1018E000002B7FF46EAE2B681E1203F07F030435CD
:1018F00058F8233049E6C24802F00CF83B78002B38
:101900007FF45FAE2B681E1203F07F03043558F896
:1019100023303AE6002E05EB8605FFF663AE3B78F2
:10192000002B7FF44EAE2B681E1203F07F030435AC
:1019300058F8233029E654F8043D042B04D1002E36
:1019400005EB8605FFF64EAE3B78002B7FF439AEF3
:101950002B681E1203F07F03043558F8233014E679
:1019600054F8043D042B04D0002E05EB8605FFF649
:1019700039AE3B78002B7FF424AE2B681E1203F0A7
:101980007F03043558F82330FFE554F8040CC307EF
:10199000A4F1040B0BD54010013800280ADB4000ED
:1019A00040F0010005EB8605CBF800001AE6FFF7D2
:1019B000EBFCF1E73B780BB15C4602E62B681E12AC
:1019C00003F07F035C4658F823300435DDE57300EF
:1019D00003F4FF7343F001032360DAF80830EB1AD5
:1019E0009D109AF8023043EA05235B0043F001039F
:1019F0006360029BA9EB030322465B1043F00103E3
:101A0000361293608AF802607E4B3A78F6B20C4642
:101A100053F83630CAF808301AB103F10805894680
:101A2000CFE503F10C059B681E1203F07F03894686
:101A300058F82330A9E5029B54F8046C4B452FD18C
:101A4000F70720D4042E17D9336803F00F03042BB3
:101A500013D1304601F06EFF08F09AFEB0F5487FD2
:101A600028BF4FF448700630643003F05DFE70B953
:101A7000043DDDF80890B5E507D0002E14BF4FF403
:101A800000700720F0E70A20EEE70720ECE7314678
:101A90009AF8010004F05DFA00238AF80030E8E7C4
:101AA00059F80C3C57495A106FF0030353430C3B51
:101AB00009EB030449F8036059F8083C5A108AF806
:101AC0000220D2B2C3F3552351F83220CAF80820BD
:101AD00059F8041C4FEA6109029901EB8909397828
:101AE000043402EB830500297FF46BAD52F82330F8
:101AF0001E1203F07F03043558F8233045E554F8EF
:101B0000040CFFF741FC1E288346A4EB860425DC69
:101B100000280BDC3B78002B7FF453AD2B681E12A2
:101B200003F07F03043558F823302EE501F0EEFB77
:101B3000ABF1030B344E834401F0E8FBA0EB0B0048
:101B4000B042F9D83B78002B7FF43BAD2B681E12D6
:101B500003F07F03043558F8233016E501238AF893
:101B6000003001F0D3FB0A385844CAF8040039E5C4
:101B700054F8040CFFF708FCA4EB8604061E0BDCEB
:101B80003B78002B7FF41DAD2B681E1203F07F0302
:101B9000043558F82330F8E41C4B9E4202DD1D2327
:101BA0003B700EE501238AF8003001F0AFFB4FF4E3
:101BB0007A7303FB06000A38D7E700233046A4EB0C
:101BC0008604134E1A462146FFF72CFC3168114853
:101BD00002F0CDF8104B316818600E4804F080F820
:101BE00031680C4804F0BAF93B78002B7FF4E9AC7B
:101BF0002B681E1203F07F03043558F82330C4E429
:101C00007CBA0000D88301203F420F0080EE3600EE
:101C1000A405002081020020080000203B78A4EBEE
:101C20008604002B7FF4CDAC2B681E1203F07F03DB
:101C3000043558F82330A8E4504603F0D9FD3B782A
:101C4000002B7FF4BEAC2B681E1203F07F0304351B
:101C500058F8233099E454F8043C002B44D154F84C
:101C60000C0C10F0010B1ED04FEA600B4FEA4B0337
:101C700043F0010344F8083CBBF1000F40F38880B7
:101C80004FEA4B0343F0010354F80C0C44F8043CB6
:101C900054F8083CC107CBEB63032AD501335B0042
:101CA00043F0010330E004281BD9036803F00F025E
:101CB000092A01D14068D7E7042A09D101F03AFE88
:101CC0000378002BD2D0FFF796FA0BF1010BF7E760
:101CD000032A06D1C3F30F1BC3F34173C3EB8B0B72
:101CE000C4E719233B706CE44FEA630B0BF1FF3B35
:101CF000C2E7042849D9026802F00F02092A11D16B
:101D000003F1020B50F82B3049F826303B78002BBA
:101D10007FF457AC2B681E1203F07F03043558F88C
:101D2000233032E4042A2BD1039309EB860300937A
:101D300001F000FE039B83465E1C012E12DC584618
:101D4000FFF759FAA0EB0B06304602F009F80346FC
:101D500070B1039001F0EEFD3246594608F054F997
:101D6000039B05E09BF80030013E23B912223A7034
:101D7000009A1360CAE75846FFF73DFA8346DCE74E
:101D8000032A02D11844037989E719233B7018E428
:101D90000435BBE7029A04EB86039B1AD82B11DCAF
:101DA0000122002E06F1FF3310DC3B78002B7FF47C
:101DB00008AC2B681E1203F07F03043558F823305B
:101DC000FFF7E3BB1A233B70FFF7FBBB22601E4605
:101DD0000434E6E7029A231D9B1AD82B03DD1A234D
:101DE0003B70FFF7EEBB029B4B452AD254F8040C24
:101DF000FFF7CAFA002821DD59F80C3C5B1083423A
:101E00001CDBC3EB8373184400F180400438A4EB5F
:101E1000860359F820201A606FF0030303FB064481
:101E20003B780434002B7FF4CCAB2B681E1203F0FC
:101E30007F03043558F82330FFF7A7BB20233B70FE
:101E4000EAE71823FBE7C14B1A68A4EB86031A6084
:101E50006FF0030303FB06443B780434002B7FF44C
:101E6000B0AB2B681E1203F07F03043558F8233003
:101E7000FFF78BBB54F8043C042B3B78A4F104021D
:101E800004BF05EB8605224613B11446FFF799BB44
:101E90002B681E1203F07F03144658F823300435D4
:101EA000FFF773BB54F8043D042B1CBF00232360D1
:101EB0003B781CBF05EB86050434002B7FF481AB17
:101EC0002B681E1203F07F03043558F82330FFF708
:101ED0005CBB002EA4EB860115DC1C233B700022AA
:101EE0006FF0030303FB06443B780A600434002BC5
:101EF0007FF467AB2B681E1203F07F03043558F89C
:101F00002330FFF742BB0B684FF0000C5B1051F819
:101F10002C0010F0010202D10D233B70E0E74010CD
:101F200083420CF1010CA8BF03466645EFDC5B0061
:101F300043F00102D4E7002EA4EB860115DC1C233C
:101F40003B7000226FF0030303FB06443B780A60FA
:101F50000434002B7FF435AB2B681E1203F07F0393
:101F6000043558F82330FFF710BB0B684FF0000C16
:101F70005B1051F82C0010F0010202D10D233B70D0
:101F8000E0E7401083420CF1010CB8BF0346664500
:101F9000EFDC5B0043F00102D4E754F8081C11F0B9
:101FA000010F4FEA86031FD054F8042C12F0010FE2
:101FB0001AD05210B2EB610FA4EB0303D4BF00227E
:101FC00004221A606FF0030303FB06443B780434D9
:101FD000002B7FF4F6AA2B681E1203F07F03043552
:101FE00058F82330FFF7D1BA54F8042C6FF00100F1
:101FF000A4EB030BFFF714F9CBF80000E2E754F869
:10200000081C11F0010F4FEA86031FD054F8042C6E
:1020100012F0010F1AD05210B2EB610FA4EB0303C0
:10202000B4BF002204221A606FF0030303FB0644CE
:102030003B780434002B7FF4C4AA2B681E1203F0F3
:102040007F03043558F82330FFF79FBA54F8042C67
:102050004FF0FF30A4EB030BFFF7E2F8CBF80000E2
:10206000E2E754E9020181424FEA860314D1E31A00
:1020700004221A606FF0030303FB06443B78043428
:10208000002B7FF49EAA2B681E1203F07F030435F9
:1020900058F82330FFF779BA0428A4EB030B01D8D2
:1020A000002315E0C307FBD4036803F00F03042BE0
:1020B000F6D1CB07F4D40429F2D90B6803F00F034F
:1020C000042BEDD1FFF782F900280CBF0023042375
:1020D000CBF80030CEE754E9020181424FEA860393
:1020E00014D1E31A00221A606FF0030303FB0644C5
:1020F0003B780434002B7FF464AA2B681E1203F093
:102100007F03043558F82330FFF73FBA0428A4EBC7
:10211000030B01D8042315E0C307FBD4036803F0C5
:102120000F03042BF6D1CB07F4D40429F2D90B68A2
:1021300003F00F03042BEDD1FFF748F900280CBF83
:1021400004230023CBF80030CEE700BF08000020B6
:1021500054F8081C11F0010F4FEA86031FD054F801
:10216000042C12F0010F1AD05210B2EB610FA4EB45
:102170000303CCBF002204221A606FF0030303FBA9
:1021800006443B780434002B7FF41BAA2B681E12F4
:1021900003F07F03043558F82330FFF7F6B954F8FD
:1021A000042C0120A4EB030BFFF73AF8CBF8000056
:1021B000E3E754F8081C11F0010F4FEA86031FD023
:1021C00054F8042C12F0010F1AD05210B2EB610F28
:1021D000A4EB0303ACBF002204221A606FF00303D8
:1021E00003FB06443B780434002B7FF4EAA92B68F8
:1021F0001E1203F07F03043558F82330FFF7C5B9EA
:1022000054F8042C0220A4EB030BFFF709F8CBF8D9
:102210000000E3E754F8043C042BA4EB860314BF4E
:10222000042200221A606FF0030303FB06443B788C
:102230000434002B7FF4C5A92B681E1203F07F0322
:10224000043558F82330FFF7A0B954F8080CFFF70D
:102250009BF8834654F8040CFFF796F85844A4EB17
:102260008603400040F0010018606FF0030303FB99
:1022700006443B780434002B7FF4A3A92B681E127C
:1022800003F07F03043558F82330FFF77EB954F884
:10229000080CFFF779F8834654F8040CFFF774F83C
:1022A000ABEB0000A4EB8603400040F00100186097
:1022B0006FF0030303FB06443B780434002B7FF4E8
:1022C00080A92B681E1203F07F03043558F82330D1
:1022D000FFF75BB954F8080CFFF756F8834654F83B
:1022E000040CFFF751F800FB0BF0A4EB8603400051
:1022F00040F0010018606FF0030303FB06443B78D5
:102300000434002B7FF45DA92B681E1203F07F03B9
:10231000043558F82330FFF738B954F8040CFFF7A8
:1023200033F88346B8B91F233B70A4EB8603C3F888
:1023300000B06FF0030303FB06443B780434002B2A
:102340007FF43FA92B681E1203F07F03043558F871
:102350002330FFF71AB954F8080CFFF715F890FB73
:10236000FBFB4FEA4B0B4BF0010BDEE754F8040C80
:10237000FFF70AF88346B8B91F233B70A4EB860326
:10238000C3F800B06FF0030303FB06443B7804344A
:10239000002B7FF416A92B681E1203F07F0304356F
:1023A00058F82330FFF7F1B854F8080CFEF7ECFFAB
:1023B00090FBFBF303FB1B0B4FEA4B0B4BF0010BAA
:1023C000DCE754F8040CFEF7DFFF0028B8BF4042FA
:1023D000A4EB8603400040F0010018606FF0030397
:1023E00003FB06443B780434002B7FF4EAA82B68F7
:1023F0001E1203F07F03043558F82330FFF7C5B8E9
:10240000A4EB860B012EDBF8000028D1FEF7BCFF01
:10241000324603460393009208F00CF9039B009A9E
:10242000012BB8BF012390FBF3F101FB130313440D
:102430005B0043F00103CBF800306FF0030303FBB4
:1024400006443B780434002B7FF4BBA82B681E1293
:1024500003F07F03043558F82330FFF796B8FEF7F2
:1024600093FF0090DBF80400FEF78EFF009A013026
:10247000831ACFE7A4EB860B5946304601F00CFED9
:102480006FF0030303FB06443B78CBF800000434F1
:10249000002B7FF496A82B681E1203F07F030435EF
:1024A00058F82330FFF771B854F8080CFEF76CFFAA
:1024B000834654F8040CFEF767FF0BEA0000A4EB18
:1024C0008603400040F0010018606FF0030303FB37
:1024D00006443B780434002B7FF473A82B681E124B
:1024E00003F07F03043558F82330FFF74EB854F853
:1024F000080CFEF749FF834654F8040CFEF744FF2E
:102500004BEA0000A4EB8603400040F00100186095
:102510006FF0030303FB06443B780434002B7FF485
:1025200050A82B681E1203F07F03043558F823309F
:10253000FFF72BB854F8080CFEF726FF834654F833
:10254000040CFEF721FF8BEA0000A4EB8603400099
:1025500040F0010018606FF0030303FB06443B7872
:102560000434002B7FF42DA82B681E1203F07F0388
:10257000043558F82330FFF708B854F8040CFEF778
:1025800003FFC043A4EB8603400040F00100186045
:102590006FF0030303FB06443B780434002B7FF405
:1025A00010A82B681E1203F07F03043558F823305F
:1025B000FEF7EBBF54F8080CFEF7E6FE834654F82E
:1025C000040CFEF7E1FE0BFA00F0A4EB86034000DA
:1025D00040F0010018606FF0030303FB06443B78F2
:1025E0000434002B7EF4EDAF2B681E1203F07F0342
:1025F000043558F82330FEF7C8BF54F8080CFEF72E
:10260000C3FE834654F8040CFEF7BEFE4BFA00F0FE
:10261000A4EB8603400040F0010018606FF0030354
:1026200003FB06443B780434002B7EF4CAAF2B68CE
:102630001E1203F07F03043558F82330FEF7A5BFC0
:1026400054F80C0CFEF7A0FE834654F8080CFEF775
:102650009BFE8BFB002354F8040CCDE90023FEF70E
:1026600093FEDDE90023C0F1200CB0F1200103FA54
:102670000CFC22FA00F040EA0C005CBF43FA01F1C6
:1026800008436FF00303A4EB860E400003FB0644EF
:102690003B7840F00100CEF800000434002B7EF4BB
:1026A00090AF2B681E1203F07F03043558F82330D7
:1026B000FEF76BBFA4EB860B59463046FEF7FAFBDC
:1026C0006FF0030303FB06443B78CBF800000434AF
:1026D000002B7EF476AF2B681E1203F07F030435C7
:1026E00058F82330FEF751BFA4EB8604214630464C
:1026F000FEF7F7FB3B78002B7EF463AF2B681E12CE
:1027000003F07F03043558F82330FEF73EBFA4EBF7
:10271000860B59463046FEF725FC6FF0030303FB9A
:1027200006443B78CBF800000434002B7EF449AF1C
:102730002B681E1203F07F03043558F82330FEF790
:1027400024BFA4EB860421463046FEF795FC3B7877
:10275000002B7EF436AF2B681E1203F07F03043586
:1027600058F82330FEF711BFA4EB860B59463046CC
:10277000FEF7F0FC6FF0030303FB06443B78CBF855
:1027800000000434002B7EF41CAF2B681E1203F0F3
:102790007F03043558F82330FEF7F7BE54F8040CD5
:1027A00001F0C8F854F8083CDA072AD4042B0CD9F5
:1027B0001B6803F00F03013B082B10D8DFE803F080
:1027C000052127230F0F0F0F2500CC4907F0D6FF57
:1027D000A4EB8603002814BF002204221A606FF0C5
:1027E000030303FB06443B780434002B7EF4E9AE7C
:1027F0002B681E1203F07F03043558F82330FEF7D0
:10280000C4BEBF49E2E7BF49E0E7BF49DEE7BF49D1
:10281000DCE7029B261DF31AD82B03DD1A233B703D
:10282000FEF7CFBE00F07AFD2346400040F00100E5
:1028300018603B783446002B7EF4C3AE2B681E1222
:1028400003F07F03043558F82330FEF79EBE029B49
:10285000261DF31AD82B03DD1A233B70FEF7B1BEF9
:1028600000F054FDAA4A234602EA400040F001006D
:1028700018603B783446002B7EF4A3AE2B681E1202
:1028800003F07F03043558F82330FEF77EBE029B29
:10289000261DF31AD82B03DD1A233B70FEF791BED9
:1028A00000F03CFD9B4B1B6898423DBFC3F5830382
:1028B00003F63713C018C01A4000234640F0010049
:1028C00018603B783446002B7EF47BAE2B681E12DA
:1028D00003F07F03043558F82330FEF756BE00F0AE
:1028E0001DFD8C4B18603B78A4EB8604002B7EF416
:1028F00068AE2B681E1203F07F03043558F82330AE
:10290000FEF743BE00F016FDB30068B9E41A3B7849
:10291000002B7EF456AE2B681E1203F07F030435A5
:1029200058F82330FEF731BE304627467A4EE41A77
:1029300001231A462146FEF775FD3068643002F027
:10294000F3FE18B9043D3C46FEF74CBE9AF8012050
:102950003168724803F015FB01238AF8003000F05B
:10296000D5FC6F4A33681268063302FB0300FFF799
:10297000FCB800F0DFFCB30068B9E41A3B78002B28
:102980007EF41FAE2B681E1203F07F03043558F847
:102990002330FEF7FABD304627465F4EE41A002288
:1029A00001232146FEF73EFD3068643002F0BCFE94
:1029B0000028C7D0594803F07FF8CDE7FEF7B0FDF7
:1029C0006FF00303A4EB860B03FB06443B78CBF8C4
:1029D00000000434002B7EF4F4AD2B681E1203F0CB
:1029E0007F03043558F82330FEF7CFBD3B78A4EBC6
:1029F0008604002B7EF4E5AD2B681E1203F07F03E6
:102A0000043558F82330FEF7C0BDA4EB860B5846BA
:102A100000F0BDFC6FF0030303FB06443B78CBF8EA
:102A200000000434002B7EF4CCAD2B681E1203F0A2
:102A30007F03043558F82330FEF7A7BDA4EB860BBF
:102A4000584600F0A6FC6FF0030303FB06443B78F6
:102A5000CBF800000434002B7EF4B3AD2B681E12BB
:102A600003F07F03043558F82330FEF78EBDA4EB46
:102A7000860B5946304600F08FFC6FF0030303FBD2
:102A800006443B78CBF800000434002B7EF499AD6B
:102A90002B681E1203F07F03043558F82330FEF72D
:102AA00074BDA4EB8604204600F0A8FC3B78002B04
:102AB0007EF487AD2B681E1203F07F03043558F8AF
:102AC0002330FEF762BDA4EB860B5946304600F07A
:102AD000CFFC6FF0030303FB06443B78CBF8000008
:102AE0000434002B7EF46DAD2B681E1203F07F03BF
:102AF000043558F82330FEF748BD00BF8CBA0000FB
:102B000094BA00009BBA0000A2BA0000A7BA000065
:102B1000FEFFFF7FAC050020A405002081020020FD
:102B200004000020A4EB8604204600F05DFD3B7805
:102B3000002B7EF446AD2B681E1203F07F03043594
:102B400058F82330FEF721BD0121304600F01AFD70
:102B50003B78002B7EF435AD2B681E1203F07F030B
:102B6000043558F82330FEF710BD0021304600F040
:102B700009FD3B78002B7EF424AD2B681E1203F078
:102B80007F03043558F82330FEF7FFBCA4EB860B17
:102B9000584600F0AFFC6FF0030303FB06443B789C
:102BA000CBF800000434002B7EF40BAD2B681E1212
:102BB00003F07F03043558F82330FEF7E6BCA4EB9E
:102BC000860B584600F0AAFC6FF0030303FB064493
:102BD0003B78CBF800000434002B7EF4F2AC2B6879
:102BE0001E1203F07F03043558F82330FEF7CDBCE6
:102BF000A4EB8604204600F065FC3B78002B7EF4B5
:102C0000E0AC2B681E1203F07F03043558F8233024
:102C1000FEF7BBBCA4EB8604204603F00FFE3B7816
:102C2000002B7EF4CEAC2B681E1203F07F0304351C
:102C300058F82330FEF7A9BCA4EB860B584603F0E6
:102C4000A1FE6FF0030303FB06443B78CBF80000C2
:102C50000434002B7EF4B5AC2B681E1203F07F0306
:102C6000043558F82330FEF790BCA4EB86042046C8
:102C700003F052FD3B78002B7EF4A3AC2B681E12B0
:102C800003F07F03043558F82330FEF77EBCA4EB35
:102C9000860B584603F05CFD6FF0030303FB06440C
:102CA0003B78CBF800000434002B7EF48AAC2B6810
:102CB0001E1203F07F03043558F82330FEF765BC7D
:102CC000A4EB86042146304601F08AFC3B78002BB9
:102CD0007EF477AC2B681E1203F07F03043558F89E
:102CE0002330FEF752BCA4EB86042146304601F0A7
:102CF0009DFA3B78002B7EF464AC2B681E1203F027
:102D00007F03043558F82330FEF73FBCA4EB86045C
:102D10002146304601F09AFB3B78002B7EF451AC03
:102D20002B681E1203F07F03043558F82330FEF79A
:102D30002CBCA4EB86042146304601F0ADFB3B7869
:102D4000002B7EF43EAC2B681E1203F07F0304358B
:102D500058F82330FEF719BCA4EB860B59463046D1
:102D600003F0EAFE6FF0030303FB06443B78CBF865
:102D700000000434002B7EF424AC2B681E1203F0F8
:102D80007F03043558F82330FEF7FFBBA4EB860B16
:102D90005946304603F0D8FE6FF0030303FB0644A8
:102DA0003B78CBF800000434002B7EF40AAC2B688F
:102DB0001E1203F07F03043558F82330FEF7E5BBFD
:102DC000A4EB860B5946304603F0C6FE6FF00303B2
:102DD00003FB06443B78CBF800000434002B7EF460
:102DE000F0AB2B681E1203F07F03043558F8233034
:102DF000FEF7CBBBA4EB860B5946304603F044FBF1
:102E00006FF0030303FB06443B78CBF80000043467
:102E1000002B7EF4D6AB2B681E1203F07F03043523
:102E200058F82330FEF7B1BBA4EB860421463046A8
:102E300001F026FA3B78002B7EF4C3AB2B681E1200
:102E400003F07F03043558F82330FEF79EBBA4EB54
:102E500086042146304601F047FB3B78002B7EF488
:102E6000B0AB2B681E1203F07F03043558F82330F3
:102E7000FEF78BBBA4EB860B5946304601F0AEFA49
:102E80006FF0030303FB06443B78CBF800000434E7
:102E9000002B7EF496AB2B681E1203F07F030435E3
:102EA00058F82330FEF771BBA4EB86042146304668
:102EB00001F058FA3B78002B7EF483AB2B681E128E
:102EC00003F07F03043558F82330FEF75EBB002E75
:102ED0005ADD012E54F804BC39D11BF0010F43D147
:102EE000BBF1040F40D9DBF8003003F00F03042BD3
:102EF0003AD1584600F01EFDFEF7EAF90028A4EB8F
:102F0000860441DB022E3DD11BF0010F35D1BBF110
:102F1000040F32D9DBF8003003F00F03092B2CD15A
:102F2000DBF80460211FC6F347060123B3421EDD10
:102F300004EB860446EA0026029B04F10C01CB1A3E
:102F4000D82B7EF744AD1A233B70FEF73ABB022E16
:102F50000AD154F8080CC30706D4042804D903681E
:102F600003F00F03042BC5D04FF0FF30C6E7013349
:102F70005BF8232041F8042FD8E7C4F800B00126FD
:102F80000434D7E70026D5E7002323603B78221DD1
:102F900013B11446FEF715BB2B681E1203F07F0316
:102FA000144658F823300435FEF7EFBA029BE31AB3
:102FB0009B10A4EB8604CAF810302146304602F07C
:102FC000BBFD3B78002B7EF4FCAA2B681E1203F09D
:102FD0007F03043558F82330FEF7D7BA029BE31A73
:102FE0009B10A4EB860BCAF810305946304602F00D
:102FF000A3FD6FF0030303FB06443B78CBF800000E
:103000000434002B7EF4DDAA2B681E1203F07F032C
:10301000043558F82330FEF7B8BA00BF2DE9F84F51
:10302000224D0023002B03F1FF3706DA01F07AFB73
:1030300002F08CFE03F004F819270026DFF87880F0
:103040003046D8F80020B24215DD2B68184C013309
:103050009342A8BF00232B60D5F80090F02303FB18
:1030600009F304EB030AE35CA346EBB1022B04D1A2
:103070005046FEF76BFA3B46D4E7012B0ED108B958
:1030800000F044F9F02303FB09F39B440949DBF802
:103090000420821A8A429CBF0222E254F02303FBDE
:1030A00009F3E35C022BE3D00136CAE700000020FD
:1030B000787A01203F420F00A80500200A4B4FF408
:1030C00080721A60094B01211964D3F8402505323A
:1030D000C3F84825C3F84C254FF44022C3F8042315
:1030E000034B1970704700BF00E100E00080004012
:1030F000D305002004207047F8B5D1E9004514F04D
:1031000001002DD015F001002AD064101C2C3CD8F1
:103110001F4F6D1041F288363B5DAE42A8BF2E4670
:10312000012B05D00121204604F0AAFE01233B55C6
:10313000184B1B780BB9FFF7C1FF002D4FF00003B0
:10314000154A0EDC154940F2DC50FF25D65CB4422E
:1031500004BF21F81300D5540133042BF6D1042009
:10316000F8BDD15C8C4203D10C4A22F81360F6E71B
:103170000133042BF5D10023D15CFF2901D1D454B4
:10318000F2E70133042BF7D1E9E70020E8E700BFBD
:10319000B4050020D30500201C0000200E000020F4
:1031A00070B5D1E9004514F001001BD015F0010005
:1031B00018D064101D2C28BF1B24154E335D012B25
:1031C00005D00121204604F05BFE01233355114B4D
:1031D0006D10A5F110029A420F4B04D94FF0FF3247
:1031E0001A60042070BD1C600C4B0D4890FBF5F07C
:1031F00018800C4B1B780BB9FFF760FF0A4B0122BC
:103200009A64D3F848251044C3F84805E9E700BF9D
:10321000B405002090860100180000200C0000205A
:1032200020A10700D30500200080004070B50D6884
:103230000128CCBF4C68012415F0010042D014F0E5
:1032400001003FD06D10002D05DC1F4B0122C3F89B
:103250000825002036E064101C2CFAD81B4E335D84
:10326000012B05D00121204604F00AFE012333552D
:103270000A22174B93FBF5F3053393FBF2F3154A40
:10328000154952F824201548120242F00312C1F8E1
:1032900010250D4AC2F81005C2F814150121C2F814
:1032A0000415A2F5A83210690020C2F810054FF6E7
:1032B000FF708342A8BF0346C2F840350420C2F81D
:1032C0000012116070BD00BF00F00140B405002085
:1032D00000B4C40444CB00000060004040A10040A2
:1032E000002802DC1C20FEF715B9012070470420DD
:1032F0007047002802DC1C20FEF70CB90B68DB07C6
:1033000001D40D20F8E7002070470000024B012295
:103310001A64D3F84005704700800040044B012236
:103320001A64D3F840054FF47A73B0FBF3F070479A
:1033300000800040012070470048704710BB00002B
:103340001D20704770B5054D2B5C8B4204460E4620
:1033500002D004F095FD2E5570BD00BFB4050020CD
:1033600070B50024084D2646635D012B08D100216D
:10337000204604F0AFFD0021204604F081FD665593
:1033800001341D2CF0D170BDB405002070470F2012
:1033900070473B2070470000F8B50B68DA07074616
:1033A0000D4604D40D20FEF7B5F8012007E05B10B0
:1033B000062B05D103F0DEF9400040F00100F8BD16
:1033C000F3D80C4A0C4E52F82340335D2BB1002148
:1033D000204604F055FD00233355012F06DD6B68B0
:1033E000042B03D10221204604F04AFD204604F0BC
:1033F00051FCE1E7F4BA0000B405002070B50468A0
:10340000E20702D54568EB0704D40D20BDE8704003
:10341000FEF780B864101C2C23D8124E335D012BAC
:1034200018D00121204604F02BFD01231B2C33551D
:1034300010D10D4BDA6E0D4B202AB8BF4FF0A043D0
:1034400002F01F0203EB8203D3F8002742F440721C
:10345000C3F80027A5F34A012046BDE8704004F0F8
:10346000BDBC70BDB405002044CB0000000300507B
:1034700070B50C68E30704D40D20FEF74BF801206B
:1034800070BD64101C2C14D8012814DD4B68042B6B
:1034900014BF002502250A4E335DAB4204D02946F5
:1034A000204604F0EDFC3555204604F02FFD0128A0
:1034B00003D00020E4E70025EDE70420E0E700BFAB
:1034C000B405002013B50A4A044692E803002268B6
:1034D0006B46042A83E8030019464FF0020003D12B
:1034E00000F0B4FF02B010BD00F0D6FFFAE700BF55
:1034F000B4BA000010B5084C63792BB10021052047
:1035000004F0BEFC00236371052004F0FFFC0028DA
:103510000CBF0420002010BDB405002010B5084CDD
:10352000E37A2BB100210B2004F0AAFC0023E37204
:103530000B2004F0EBFC00280CBF0420002010BD81
:10354000B405002010B50B4A0B4C0C480C49002365
:10355000C2F80035A2F5C832C2F810350122626007
:1035600042604A60C4F80035C0F80035C1F8003543
:1035700010BD00BF00F0014000C00140001002403B
:10358000002002401C2870B504460D4625D8134E75
:10359000335C012B04D0012104F072FC012333556C
:1035A0001C2C12D1FFF7CEFF0D4B1A6F0D4B202AAA
:1035B000B8BF4FF0A04302F01F0203EB8203D3F821
:1035C000002742F44072C3F80027291C204618BF88
:1035D0000121BDE8704004F07DBC70BDB405002041
:1035E00044CB0000000300500368D90702D40D202B
:1035F000FDF790BF41680A1F514251415810FFF733
:10360000C1BF0000F8B5324CD4F84831ABB100234B
:10361000D4F84855C4F848312E4B186800280CDB04
:103620002D4A1178B1FA81F14909117004F052FC68
:103630002A4B1B882B44C4F84835254BD3F84C2122
:10364000002A37D00021264ED3F84C45C3F84C1140
:103650003378244D33B12B68032B03D8224AD05C36
:1036600004F038FC2B68204F01335A4202F0030269
:1036700003F0030358BF53422B600022042B19466A
:1036800019D00133F81810F8010CFF2801D10122DC
:10369000F4E702B12960012104F01CFC012333701E
:1036A0002A68124B33F8122004F10C031344084A21
:1036B000C2F84C35F8BD4FF0FF3304F58C44044A92
:1036C0002B605C3400233370C2F84C45F2E700BF36
:1036D0000080004018000020D20500200C000020CF
:1036E000D1050020B00500201C0000200E000020A5
:1036F000094B0A4940F2DC521A805A809A80DA80DB
:10370000074A00231370074AFF200870487088702A
:10371000C8701360704700BF0E0000201C0000201E
:10372000D1050020B0050020024B4FF0FF321A6097
:10373000704700BF18000020024A0348072101F02B
:1037400085BF00BFBCBA0000F6C2000038B54FF418
:10375000E131284804F074F8274B012200211A6156
:10376000C3F804150321C3F808150421C3F8101584
:103770001A604FF080430221C3F818159A604FF089
:103780001023D3F80C32DB070FD51C4BC3F80425EC
:10379000D3F80024002AFBD04FF010226FF0010173
:1037A000C2F80C120022C3F804250A2004F06CFAB7
:1037B000134A0023FF21995401331D2BFBD1114BD8
:1037C000114D01221A600020104A0423014614689A
:1037D000002CFCD02C681160013B44EA0020F6D19B
:1037E0000B4B01221A6004F085F9BDE8384001F066
:1037F00035B800BFF87901200080004000E00140AA
:10380000B405002000D0004008D5004000D10040A1
:1038100004D00040F8B506460948094F0C4604F0AC
:103820004FF88442A8BF04463546AB1B9C4205DDD9
:10383000384604F04BF805F8010BF6E72046F8BDD2
:10384000F87901200146014803F0FFBFF879012013
:1038500010B5054C204604F005F820464FF4E13140
:10386000BDE8104003F0ECBFF8790120C3070CD489
:10387000064B1B68834208D8054B1B68984204D846
:1038800050F8043C002B18BF18467047DC05002098
:10389000D80500200B4908B50122002341F8232058
:1038A0000133642BFAD1084B1A60084B084A1846BA
:1038B000002106F0CDFB074B40F8043F064B186093
:1038C00008BD00BFD08B012008000020E0050020CB
:1038D00070670100A09D0500D4050020034B044A39
:1038E0001A60044B044A1A60FFF7D4BFDC050020BD
:1038F000E0050020D8050020506D0120044B1B6816
:103900001868C0F30F10023820EAE070704700BF5B
:10391000D405002000B59BB00246054901A806F079
:10392000F1FE01A802F0E5F802F08AFBFCE700BF17
:10393000A2BB0000C30713D4042802D812D00B483E
:103940007047036803F00F03042B01D10430704764
:10395000092B09D0064A0748032B18BF10467047A9
:1039600005487047054870470548704700B7000094
:103970008DBB000096BB00007CBB000006B70000BA
:1039800086BB0000064B074900201A6843F8040C68
:10399000C2F30F12023203EB82038B42F5D370475E
:1039A000E4050020506D01202F4B304A1868304B41
:1039B0002DE9F0411C682F4D136803F00F01072912
:1039C00028D81368C3F30F13023302EB8302AA4211
:1039D000F2D32949002251F82200FFF747FF41F8AE
:1039E00022000132642AF6D1244A1068FFF73EFF14
:1039F0001060234A106810B1FFF738FF1060214BA8
:103A0000214C1E680021F0274FF03C08B14214DB26
:103A1000BDE8F081C3F30F1302EB83039A42D0D0C9
:103A20001968CE0707D4884205D28C4203D351F8D7
:103A3000041C01B11960043BF0E707FB01F31A19FC
:103A40001B5D0BB90131E1E71269551E08FB01222C
:103A500004EB82021832002DF4DB52F8040DFFF75C
:103A600005FF013D1060F6E7DC050020E4050020BD
:103A7000D8050020506D0120D08B012008000020C7
:103A8000506D0120A8050020787A0120C307F0B509
:103A900040D4214B1C68A0423CD3204B1D68A84257
:103AA00038D850F8043CABBB03680246C3F30F138D
:103AB000012673B9904242F8046C2BD0116851F87A
:103AC000043C51F82370176041F82320013B0A465B
:103AD000EFE752F82310CF0702EB830C18D48C4287
:103AE00016D88D4214D351F8047C8FB90F6807F0B3
:103AF0000F0EBEF1070F08D9CCF8007042F8043C55
:103B00000B680A60C3F30F13E1E741F8046CD0E7D8
:103B1000013BCEE7F0BD00BFDC050020D80500204A
:103B20000D4930B50D4C0B461A6853F8045CC2F3CE
:103B30000F12901C65B18B4214BF0A46002243F855
:103B4000042C01EB800103EB8003A342ECD330BDD6
:103B500012011A60F7E700BFE4050020506D012054
:103B6000144B2DE9F041144C1E464FF0000832680A
:103B7000C2F30F1712070FD07D1C9E424FEA850536
:103B800005D018462A46314606F049FA03465A1926
:103B900004352B44C2F80080023706EB8706A642A4
:103BA000E5D3E41AA410013C044A24011C6013600C
:103BB000BDE8F081E4050020506D0120D40500200F
:103BC0002DE9F0419AB0FFF7A1FB214D07460024F3
:103BD00055F824000134FFF759FF642CF8D11D4B30
:103BE0001868FFF753FF1C4B186808B1FFF74EFF2A
:103BF0001A4DDFF874800026D8F800309E4218DB9A
:103C0000FFF78EFFFFF7D0FEFFF7AAFFFFF77EFB5F
:103C1000134B14491B681B68C3F30F13C21B023BF1
:103C200001A806F06FFD01A801F063FF1AB0BDE81E
:103C3000F0812B7813B90136F035DDE72C69013CB2
:103C4000002CF8DB05EB84039869FFF71FFFF6E70C
:103C5000D08B012008000020506D0120787A0120CF
:103C6000D40500205CBB0000A80500202DE9F84326
:103C70001B4C23681B684D1CC3F30F139D42064663
:103C800088461746A1460CDBFFF79AFF23681B689E
:103C9000C3F30F139D4204DB0A20BDE8F843FDF790
:103CA00039BC08F10202D9F800009B1A1B0140F848
:103CB0002230002340F8043C06F00F06034646EA93
:103CC0000816940043F8046B0119083CC9F8001069
:103CD0001C44A34201D3BDE8F88343F8047BF8E712
:103CE000D4050020F8B510F0010704460E462CD18B
:103CF000174B1B68834228D8164B1B68834224D974
:103D0000154D28600068012200F00F00FFF7AEFF9C
:103D10002C682F600546C0B12146043051F8042BB1
:103D2000C2F30F12B242A8BF3246920006F06CF9FD
:103D3000FFF728FE44F8045CFFF736FE2268074BC5
:103D400044F8047C134023602C462046F8BD00BF95
:103D5000DC050020D8050020506D0120F0FF0F0089
:103D6000011D0022042091FBF0F1FFF77FBF38B561
:103D7000054608460C46FFF7F3FF50B1C21C2B4620
:103D8000591B8C4206DC002CACBF0419041C002318
:103D9000237138BD13F8011B02F8011FF0E7F0B5DD
:103DA00002289BB00C4604DC1C20FDF7B3FB1BB0C3
:103DB000F0BD0868C20706D4042804D9036803F0DC
:103DC0000F03042B01D00E20EFE74B6813F001071F
:103DD000F9D1042BF7D91B6803F00F03042BF2D1A0
:103DE0008B68DB0701D40D20DFE7FFF7A3FD064654
:103DF0006068FFF79FFDA5681AAC014604F8647D72
:103E00006D10304603F06DF829466423224603F016
:103E1000CAF8204606F0BCFC01462046FFF7A7FF83
:103E2000C5E7000010B50446ADF5806D10B9FFF789
:103E300097FF0BE002F07BFF0138062827D8DFE868
:103E400000F0080810172804230000200DF5806DED
:103E500010BD204602F0E5FF011B2046FFF787FF5B
:103E6000F4E7204602F091FF400040F00100EDE74A
:103E700069464FF48062204602F0A1FF684606F0D2
:103E800087FC01466846E9E704210348E6E700208D
:103E9000CDE70420DAE700BFE8BB0000022838B510
:103EA0000C4604DC1C20BDE83840FDF733BB086835
:103EB000C10706D4042804D9036803F00F03042BB8
:103EC00001D00E20EFE76368DA07FAD4042BF8D9A3
:103ED0001B6803F00F03042BF3D1A368DB0701D4A5
:103EE0000D20E0E7FFF726FD05466068FFF722FD9D
:103EF000A46801466410284602F0F3FF214603F04F
:103F00002FF8BDE83840FFF78DBF012838B50C46C3
:103F100004DC1C20BDE83840FDF7FCBA0868C10786
:103F200006D4042804D9036803F00F03042B01D03E
:103F30000E20EFE76368DA07FAD4042BF8D91B6880
:103F400003F00F03042BF3D1FFF7F4FC0546606880
:103F5000FFF7F0FC0146284602F0C3FF03F03FF8EC
:103F6000400040F0010038BD012870B505460C4600
:103F700004DC1C20BDE87040FDF7CCBA0868C1071E
:103F800006D4042804D9036803F00F03042B01D0DE
:103F90000E20EFE76368DA07FAD4042BF8D91B6820
:103FA00003F00F03042BF3D1FFF7C4FC064660684F
:103FB000FFF7C0FC022D014615D0A468E30712D517
:103FC0006410304602F08DFF054602F0B0FE012875
:103FD00012D1002C02DD0135012C07D12846BDE8A5
:103FE0007040FFF71FBF4FF0FF34EAE7284602F0AA
:103FF00027FF013C0546EFE70228EFD1002CEDDD5D
:104000000135012CEAD000221146284602F042FF79
:1040100002F016FF013C0546F3E70000086810B502
:1040200010F001041AD0441007EE904A9FED187A60
:10403000F8EEE77A67EE877A17EE900A05F046FC0D
:1040400004F06CF80022134B05F098FC04F01CF807
:1040500005F044FF400040F0010010BD042812D9D3
:10406000036803F00F03042B07D1FFF763FC0A2258
:10407000214606F051FC0446D6E7032B03D10A2261
:1040800021460430F5E70D20FDF744FACCE700BFE8
:10409000D30237390000D040086808B5C30706D4FA
:1040A000042804D9036803F00F03042B04D00E2066
:1040B000BDE80840FDF72EBAFFF73CFC0378232B40
:1040C00008BF01301022002106F026FC00F1005349
:1040D000B3F1804F01D31420EAE7400040F0010023
:1040E00008BD0000024A0348062101F0AFBA00BF34
:1040F000B8BB0000B3BB0000002070471E20FDF7D6
:1041000009BA1E20FDF706BA1E20FDF703BA1E20CD
:10411000FDF700BA1E20FDF7FDB91E20FDF7FAB924
:104120001E20FDF7F7B91E20FDF7F4B91E20FDF79C
:10413000F1B91E20FDF7EEB91E20FDF7EBB91E20E8
:10414000FDF7E8B91E20FDF7E5B91E20FDF7E2B93D
:104150001E20FDF7DFB91E20FDF7DCB9024A034837
:10416000112101F073BA00BF24BC0000ACBC0000F8
:10417000034B01221A60034B1868904010437047AC
:10418000706D0120546D01202DE9F041EFF3108294
:10419000012302F0010883F310881549154C0968C2
:1041A000154D164E01398B4003274FF00E0C4FF082
:1041B0000B0E002B18D02168296018420AD07246D5
:1041C00011000139FDDC2168316039000139FDDC65
:1041D0005B08EEE739000139FDDC21683160624699
:1041E00011000139FDDCF3E788F31088BDE8F081A8
:1041F00020000020646D0120080500500C050050CF
:1042000070B5084E084D002456F824000021FFF731
:1042100099F855F8240000210134FFF793F8052C94
:10422000F2D170BD98BD0000E4C0000008B5054B98
:1042300000221A60044B1B680BB102F017FD00202E
:1042400008BD00BF6C6D01205C78012010B5041E14
:104250000ADA0024074B53F8242001239340064A2E
:104260001360064A136010BDFFF76AF8A042F0DD44
:10427000F0E700BF44CB0000646D0120180500503A
:104280002DE9F843344B1B680C461BB94FF0FF3047
:10429000FFF7DCFF246814F0010525D0C4F3474381
:1042A000C4F34720C4F3470240F2596540435B43DF
:1042B00090FBF5F193FBF5F0000240EA0140134654
:1042C000534393FBF5F31843244B1B68202B01BF8A
:1042D000234BC4F3456453F8243043EA0020FFF72E
:1042E00053FF0020BDE8F883042CFAD9236803F0BB
:1042F0000F03092BF5D154F8046FDFF86080DFF865
:104300006090761040F25967B542EADA54F8042F0B
:10431000D3071FD5C2F34743C2F34720C2F3470177
:1043200040435B4390FBF7FC93FBF7F0000240EA4D
:104330000C400B464B4393FBF7F31843D8F800307F
:10434000202B02BFC2F3456259F8223043EA002015
:10435000FFF71AFF0135D7E7646D01202000002028
:1043600088BF000008B50B68DA074CBF5B104FF040
:10437000FF3301280DDD4A68042A14BF18222022C9
:10438000054918460A60FFF701F8FFF75FFF0020B4
:1043900008BD1822F4E700BF2000002010B510F07F
:1043A000010402D04410204610BD042812D902682E
:1043B00002F00F02042A07D1FFF7BCFA0A222146B5
:1043C000BDE8104006F0A8BA032A03D10A2221460C
:1043D0000430F5E70D20FDF79DF8E4E7086810F0DC
:1043E000010370B51CD0FFF7D9FF0346203B5E2BBD
:1043F00027D8154C03EB83030022012110462344E8
:10440000052A1AD09E5C052410252E4218BF40189C
:10441000013C4FEA41014FEA6505F6D10132EFE771
:104420000428E3D9026802F00F010429DED1C2F3A7
:104430000F13002BDAD00379D8E7400040F00100D9
:1044400070BD0120FCE700BFACBD000038B50868B6
:104450000D46FFF7A3FF04466868FFF79FFF621E43
:10446000042A014612D8431E042B0FD8084803EB38
:10447000830313440568012202FA03F32B4303600C
:10448000044B1B6813B1204602F0F1FB002038BD3D
:104490006C6D01205C78012038B508680D46FFF787
:1044A0007DFF04466868FFF779FF621E042A014613
:1044B00014D8431E042B11D8094803EB830313447B
:1044C000012202FA03F3026822EA0302054B0260AA
:1044D0001B681BB10022204602F0C9FB002038BD3A
:1044E0006C6D01205C7801202DE9F04F054685B008
:1044F00008680C46FFF752FF022D01903CDD606812
:10450000FFF74CFF0746A068FFF748FF0446231D4E
:10451000DFF8C8A00293661E4FF00108029B9E427E
:1045200006F1010935D006EB8602531E07F1050B93
:104530003D460393AB4522D0042E19D86A1E042AA7
:1045400016D8039B019ADAF800005919224B4FF054
:10455000010C18EA020E0CFA01F11B6811D001439C
:10456000CAF8001023B162464946284602F07FFB94
:104570004FEA48080135DDE701242746C7E74E46E4
:10458000CCE720EA0101CAF80010002BF0D07246F7
:10459000EAE73D1D042D1BD8012C19D1DFF83C8022
:1045A000DFF834900026D8F8003004FA05F223EA48
:1045B0000203C8F80030D9F80030013623B10022D8
:1045C0003146781D02F053FB052E05F10505EAD1B1
:1045D000002005B0BDE8F08F5C7801206C6D0120F3
:1045E000086808B5C30703D5FFF7D8FE054B186068
:1045F000054B1B681BB1034B186802F039FB002008
:1046000008BD00BF6C6D01205C7801202DE9F341ED
:104610003F4D4FF441732C68ADF804300A238DF8F8
:1046200006305CBBFFF7ECFDDFF8F480264658F857
:10463000267001213846FEF785FE013600213846F6
:1046400003F048FC052EF2D100260DF1040816F8FF
:10465000087001213846FEF775FE01360121384603
:1046600003F038FC032EF2D1FEF750FE294B186000
:1046700001232B60204602B0BDE8F081012C1CD143
:10468000244C2668FEF742FE864298BF801BC7284E
:1046900001D80024EEE700210420FEF753FE00219C
:1046A0000320FEF74FFE00210A20FEF74BFEFEF727
:1046B0002DFE022320602B60EBE7022C21D1154B4D
:1046C0001C68FEF723FE844298BF001BB0F57A6F8A
:1046D000DFD3042003F0DEFA0446032003F0DAFA05
:1046E00006460A2003F0D6FA34442044C0F53F6061
:1046F00003230D3090FBF3F0074B1860012003F00B
:10470000C9FA064A00232B6013600124B2E700BFF8
:10471000606D0120686D0120546D0120706D0120D5
:10472000E4C000002DE9F843434E326852B9434BD0
:104730001B683BB9424B1B68002B74D0BDE8F843A3
:10474000FFF764BF3F4D2C6884BB3D4B1B68002BBB
:1047500065D13A4A336810681146002865D13A4F4E
:104760003A4EDFF8F4800B60002157F82400FEF782
:10477000E9FD56F8249001214846FEF7E3FDB9F122
:10478000220F10D858F82920314B1F2AD8BF4FF0DC
:10479000A04302F01F0203EB8203D3F8002742F488
:1047A0004072C3F800270134052CDDD12B68264E5A
:1047B000DFF88890254F002BCCBF03F1FF33042393
:1047C000002156F82300FEF7BDFD2A68214B53F85F
:1047D0002280002404EB840101EB0803D9F80010C7
:1047E00057F82400194101F00101013403F072FB74
:1047F000052CEFD12B68012156F82300FEF7A2FD0E
:104800002B68002156F8230003F064FB2B6801336A
:1048100093FBF4F404EB84041C1B2C6003E0FFF70F
:10482000F5FE002895D1BDE8F883002B97D11360E1
:10483000BDE8F843FFF7E4BC6C6D01205C6D01201E
:10484000706D0120586D012098BD0000E4C000008B
:104850000003005088C0000044CB00004FF0FF3040
:10486000FFF7F4BC024A0348092100F0EFBE00BF85
:104870009CC00000F8C000004FF0805310B51A69CA
:10488000094B0224C3F8044522F00302884203D3F3
:104890000022C3F8042510BDD3F80044002CFBD03F
:1048A000C3F808051044F1E700E00140002815BFF7
:1048B0004FF4D2214FF4B4214FF4B4204FF496209A
:1048C000FFF7DABF00280CBF4FF496234FF4B42350
:1048D0001868030E532B0CBF20F07F400020704758
:1048E000064B0122C3F80425D3F80024002AFBD08C
:1048F00000220160C3F80425704700BF00E00140BA
:10490000002821F07F4141F0A6410CBF4FF49620D2
:104910004FF4B420FFF7E4BF0A4B30B50124C3F8CD
:104920000445002903DC0022C3F8042530BD52F8F9
:10493000044BD3F80054002DFBD040F8044B013950
:10494000EFE700BF00E0014038B54C68023405468F
:104950000A462146FFF7E0FF05EB840038BD000062
:10496000124B1B68002B0BBF4FF4B4224FF4D22222
:104970004FF496234FF4B42328B91A1DDB79522B38
:1049800008BF1046704782420DD9C378522B0AD116
:104990004368023300EB8300824204D9C378522B70
:1049A00018BF002070470020704700BF746E0120C0
:1049B0002DE9F0410020B4B0FFF7D2FF0024DFF86A
:1049C000A4800546274626464DBB224D2868FFF7A2
:1049D00079FF3B463246CDE900401F4902A805F069
:1049E00091FE02A801F085F81C4B1A682B68002B79
:1049F0000CBF4FF496234FF4B423D21A4FF47041F6
:104A000064235343009193FBF1F302A8144905F08A
:104A100079FE02A801F06DF834B0BDE8F081696854
:104A20002A6801918B1C1F44D1B2C2F307239C4218
:104A3000C2F30742009102A84146B8BF1C4605F0E8
:104A400061FE02A801F055F82846FFF789FF0136FC
:104A50000546B9E7746E012002C20000786E01209D
:104A6000ACC10000EEC1000070B50020FFF72AFFC6
:104A700005460120FFF726FF0C4B1E68B6FA86F4A8
:104A800085424FEA5414B8BF054620461C60FFF724
:104A90000DFF074A074B002E18BF1346064A691C34
:104AA0002046BDE870401360FFF72ABF746E0120F6
:104AB00004B0040004A00500786E012070B5002049
:104AC000FFF700FF02460120FFF7FCFE1F4E204CBF
:104AD000054672B968B94FF4D2214FF49620FFF71A
:104AE000CBFE01212846FFF70BFF1A4B35602360F0
:104AF00029E0AA4208DD00233360164B23604FF4FF
:104B0000B4212368002017E001233360124B236097
:104B10004FF4D221F5E7120E522A08D000B12360DB
:104B20000E4800F0E6FFBDE87040FFF79DBF5A68F1
:104B3000023203EB820301208B4205D21A68551C16
:104B4000E9D10028D3D170BD2160FCE7746E01204B
:104B5000786E012004B0040004A00500C7C1000065
:104B600010B50020FFF7FCFE014608B9084610BD4D
:104B70008478FFF7F5FEDA2C08BF0146F5E7000060
:104B80002DE9F04F4FF480729FB05F4C5F480021D9
:104B900005F05EFA4FF4807200215D4805F058FA86
:104BA000D4F80090B9FA89F84FEA58184046FFF750
:104BB0007DFEA246574B584C0020B9F1000F08BFAC
:104BC0001C46FFF7CDFF064638BB4846FFF77AFE86
:104BD000524D411C4046FFF793FECAF800802C60FE
:104BE000FEF736FEDAF800302A68002B0CBF4FF4CF
:104BF00096234FF4B423D21A4FF4704164235343E5
:104C0000009193FBF1F305A8454905F07BFD05A84C
:104C100000F06FFF1FB0BDE8F08F3568C5F30743A4
:104C2000A3F10A02092AC5F3072546D8374B595D77
:104C300091BB10223B48DFF8ECB005F009FA37468B
:104C40003A68C2F307218D4209D1C2F307410B290B
:104C500026D013292BD00A2901D1CBF80070384671
:104C6000FFF77EFE07460028EAD12E4F396881B152
:104C70002046FFF769FE0123044657F8231029B1A7
:104C800020460393FFF760FE039B04460133042B89
:104C9000F3D11E4A012353553046FFF761FE92E7D8
:104CA000D2B2022ADBDC0BEB82025760D7E710227C
:104CB0000021584605F0CCF9D1E7A3F11502082AE6
:104CC000EAD8134A525D002AE6D1152B0CBF3146B3
:104CD000002130460368C3F30742152A0ED01D2A6F
:104CE00008BF0021FFF73CFE0028F3D119B1204690
:104CF000FFF72AFE04460123054ACCE7C3F3072346
:104D00009D4208BF0146EDE7746E0120746D0120DD
:104D10007C6E012004A0050004B00400786E012020
:104D200091C10000608D0120FFF72ABF2DE9F84FE7
:104D3000DFF8A8B0274F03339246042293FBF2F624
:104D4000DBF80030B41C002B3B684FEA84040CBF36
:104D50004FF4B4224FF4D22223449A4281460D46A6
:104D6000B84614D2FFF70CFFDBF80030002B3B688D
:104D70000CBF4FF4B4224FF4D22223449A4206D2FD
:104D8000154800F0B6FE00273846BDE8F88F2D0222
:104D90005FFA8AF141F0A441ADB2D8F800700D433A
:104DA0004FEA094101F47F0129433846FFF798FD96
:104DB00007F108053146381DC8F80050FFF790FD8F
:104DC0001EB10A9A2846FFF7A7FD083C2544C8F8FB
:104DD0000050D9E7786E01206BC10000746E01208D
:104DE00030B59BB0FFF76AFE00214FF4FF621D480B
:104DF00005F02EF9FFF7B4FE1A490024A0B9194BAB
:104E0000024653F8301001B101320130FF28F8D1C9
:104E1000154901A805F076FC01A800F06AFE1348C8
:104E200000F067FE1BB030BD0368C3F307420A2AD7
:104E30000BD1C3F30722FF2A04D001EBC20541F8CE
:104E400032002B71FFF78CFDD8E7132AFAD1C3F398
:104E50000723FF2B1EBF01EBC30241F8334014713F
:104E6000F0E700BFD883012037C200004BC200002A
:104E70000A4B0022C3F8002101225A60D3F8002116
:104E8000002AFBD00022C3F80C2101229A60044BB7
:104E90000222C3F880211A60704700BF0010004052
:104EA00000E100E0074B0222C3F88020064B0022FD
:104EB000C3F8102101221A61D3F81021002AFBD077
:104EC000704700BF00E100E00010004008B5044951
:104ED0000A780AB1FFF7E6FF0020087008BD00BF9E
:104EE0007D6F01204FF08053586E400040F001006C
:104EF00070470000024B1868400040F00100704706
:104F000000700120024B1868400040F0010070471B
:104F100024000020024B1868400040F00100704758
:104F20000470012070B504460D461646FEF7F6F9EA
:104F30004FF0805301225B6E6270E270020A23F030
:104F40000043A271020CE2711A0A002160716372BF
:104F5000000EA2721A0C1B0E2670A1702571207211
:104F6000E272237370BD000010B5054C204605F0B9
:104F70000FFC01462046BDE81040FEF7F8BE00BF1A
:104F800009700120104B1B685A1C10B514D0CBB10E
:104F9000012B13D0022B13D0042B13D00B4C0C4A33
:104FA000052B08BF1446204605F0F2FB01462046BB
:104FB000BDE81040FEF7DBBE064CF4E7044CF2E718
:104FC000054CF0E7054CEEE728000020E1C20000A8
:104FD000E7C20000DCC200009BBA000094BA0000E7
:104FE00010B521480278002A3DD14FF08043C3F824
:104FF000002101221A60D3F80021002AFBD01B4BAC
:105000001B4C00220721C3F80C25C3F808151949C9
:10501000C3F81025C3F81C15C3F824250121C3F8D3
:105020002C250822C3F83015C3F81425C3F81845F9
:105030000224C3F834454FF6FF74C3F83C450E4CC8
:10504000C3F838451824C3F85445C3F80423D3F8EB
:10505000002242F01002C3F80022084AC3F80425D7
:10506000FFF706FF017010BD7D6F012000100040AA
:105070002000040274696275211001007E6F012016
:10508000F8B5104B1B7804460BB9FFF7A9FF0E4E7D
:105090003378ABB10D4A1278D21A02F003010C4AF0
:1050A00002EB411202F1200710685168254603C542
:1050B0000832BA422C46F7D1013B33700120F8BDCB
:1050C0001846FCE77D6F0120087001207C6F0120ED
:1050D0007E6F012030B5002889B02ADD0D6815F0FB
:1050E000010426D1042D26D92B6803F00F03092BC8
:1050F00021D16B683F2B1EDD6846FFF7C1FFB0B1C1
:105100009DF800200435A242A8BF1DF8043004F128
:105110000104A6BF5B0043F001030123202C45F8E6
:10512000043FF0D1054BDDF809201A60042009B0D6
:1051300030BD0020FBE72046F9E700BF04700120E6
:1051400030B5384B1B788BB00BB9FFF749FF02A87D
:10515000FFF796FF10B900200BB030BD9DF8083066
:105160000B2BF8D99DF80930012BF4D19DF80B30A9
:10517000012BF0D12C4D2D4C2D4ADDF811100023C0
:105180002B6023709DF80C3013602A4A116023B9FC
:10519000DDF815302B6000230FE0012B11D1DDF875
:1051A00015309DF819202B600DF11A010E23934242
:1051B000A8BF134600229A4230D10022E2540420B4
:1051C000CAE7022B05D19DF8152012230DF1160117
:1051D000EDE7042B0DD10AAA6B4652F8130D516866
:1051E00003C3DDE9000102F0C1FE04F077FE286090
:1051F000D1E7052BCFD10AAA6B4652F8130D51689F
:1052000003C3DDE9000102F0B1FE04F067FE9DF882
:105210001D2028600A230DF11E01C8E7885CA054F8
:105220000132C8E77D6F0120007001200970012064
:10523000280000200470012010B5154B1B7804468F
:105240000BB9FFF7CDFEFFF72DFE124B0022C3F87E
:105250000445C3F8002101221A60D3F80021002A76
:10526000FBD00022C3F80C2101229A60094AD2F82F
:105270000C31002BFBD0084B1978084B03EB411382
:10528000C2F80435FFF70EFEBDE81040FFF7F0BD91
:105290007D6F0120001000407C6F01207E6F012097
:1052A00000B5002889B01DDD0B6813F0010219D18B
:1052B000042B17D9196801F00F01092912D1596877
:1052C0003F290FDD043353F8040F10F0010118BF1C
:1052D000C0F347010DF802100132202AF3D16846CD
:1052E000FFF7AAFF002009B05DF804FB002810B505
:1052F00011DD0C68E3070ED56410532C0BD8074B57
:105300001B780BB9FFF76CFEFFF7CCFD044BC3F81D
:105310000845FFF7ADFD002010BD00BF7D6F0120E7
:1053200000100040002810B50DDD0C68E3070AD519
:105330006410FF2C07D8054B1B780BB9FFF750FE04
:10534000034BC3F82445002010BD00BF7D6F012032
:1053500000100040002813B515DD0C68E10712D5D8
:1053600064100A4A0A4B072CCDE900230BD8094BDD
:105370001B780BB9FFF734FE02AB1C44064B14F943
:10538000082CC3F80C25002002B010BDE2ECF0F4AC
:10539000F8FC00047D6F01200010004070B500286B
:1053A00088B020DD086810F001041CD104281AD947
:1053B000036803F00F03042B15D1FEF7BBFA064672
:1053C00005F0E6F9122828BF1220054600F10D026B
:1053D00002216846FFF7A6FD8DF80D50A54205DCB9
:1053E0006846FFF729FF002008B070BD0DEB0403ED
:1053F000325D9A730134F1E72DE9F041012888B05C
:105400000D4630DD086810F001042CD104282AD99B
:10541000036803F00F03042B25D14B68DB0722D56B
:10542000FEF788FA804605F0B3F96D680E2828BFAC
:105430000E206E10074600F1110201216846FFF7A9
:1054400071FD6B128DF80D606D14360E8DF80E30F7
:105450008DF80F508DF810608DF81170A74206DCA2
:105460006846FFF7E9FE002008B0BDE8F0810DEBCB
:10547000040318F804209A740134EFE730B50028CB
:1054800089B016DD0C68E30713D565106846102255
:105490000021FFF747FD63128DF80D5064142D0EA7
:1054A00068468DF80E308DF80F408DF81050FFF7DC
:1054B000C3FE002009B030BD174BD3F8002122B144
:1054C0000022C3F8002101229A60D3F80C2102B314
:1054D0000021C3F80C11D3F80024012A0F4A19D176
:1054E000D3F848355B4213600D4A1378032B9CBFF9
:1054F000013313700B4A1378013303F00303137065
:10550000094A02EB4313044AC2F80435024B012254
:105510009A6070471160F9E70010004024000020F5
:10552000087001207C6F01207E6F0120024A034831
:10553000102100F08BB800BF5CC2000053C2000015
:10554000044A05491368C8540133C3F309031360BF
:10555000704700BF387401203870012070B51149C0
:10556000114A0B68834202DC00230B6017E0855C64
:10557000A5F1FA06012E00F1010405D89C420FDACC
:10558000A55C013D1F2D01D92046EBE70446151A05
:10559000165D2E550134A342FADC181A086070BD5E
:1055A0001570FAE7447801204474012008B5FDF72E
:1055B000ADFE074B1A68824284BF00221A601B6846
:1055C000C01A44F62063984294BF0020012008BD11
:1055D0003470012070B5094C094D0A4E23682A68C1
:1055E000934200D170BDF05CFEF72CF90028F9D091
:1055F00023680133C3F309032360EFE73C74012000
:10560000387401203870012070B5074E074D0446EC
:1056100033682A689B1ADB43C3F30903A34200DB08
:1056200070BDFFF7D7FFF3E7387401203C74012009
:1056300010B5FFF795FA044608B9204610BD8378E7
:105640001D2B08BF0446FFF78BF9F5E7F0B5074DB2
:105650002B680B2B08DC064F0C245C433E19C6E973
:105660000112013338512B60F0BD00BF407401209E
:10567000708D012008B5FBF78FFDFFF7F3F8FBF7FE
:10568000AFFDFEF759F8FEF72DFDFEF767FDFFF7BA
:105690004DFF01F0C9F801F0EDFABDE8084001F056
:1056A00023BD000008B54FF416620021034804F042
:1056B000CFFC034B00221A6008BD00BF787A01209E
:1056C000A8050020174B53F83000836803F07F03D0
:1056D0001C2B70B50D46144601D0002070BDC36868
:1056E00003F07F02042AF8D1026902F07F02192A2E
:1056F000F3D11B0A00EB83001030FEF71BF903788F
:10570000064633B105F044F8A042E6D10023A34297
:1057100001DB0120E2E7F15CEA5C9142DDD101337B
:10572000F5E700BFD8830120064B074A1B681268C3
:105730009B1ADB43C3F309038342D4BF002001203B
:10574000704700BF387401203C740120F8B507464B
:105750000E4614461D4673B90320FFF7E5FF10B34C
:10576000FA20FFF7EDFEF8B2FFF7EAFEF0B2BDE86F
:10577000F840FFF7E5BE501DFFF7D6FF98B1FB20BC
:10578000FFF7DEFEF8B2FFF7DBFEF0B2FFF7D8FE60
:10579000E0B2FFF7D5FEC4F30720FFF7D1FE2E4697
:1057A000731B9C4200DCF8BD16F8010BFFF7C8FE26
:1057B000F6E70000F8B50C4E0C4D0024F0273368D6
:1057C000A34203DCBDE8F840FFF76CBF07FB04F31E
:1057D00059195B5D2BB100231A4649781120FFF758
:1057E000B5FF0134EBE700BFA8050020787A01205F
:1057F000F8B50E4C0E4E07460025BC4205F10105DA
:1058000011D0237853B100231A4661781120FFF795
:105810009DFFF0220021204604F01AFC0A2D04F11D
:10582000F004EAD1F8BD3560F8E700BF787A0120CE
:10583000A80500202DE9F04F12F00106ADF54F7DCF
:1058400082468B4617D001238DF8143042FA03F3B9
:1058500054128DF8153052141B0E8DF817208DF848
:1058600018308DF8164005AB0522FFF76FFF0DF5D8
:105870004F7DBDE8F08F042A2CD9116801F00F0389
:10588000042B38D105AD022310462B70FEF752F8D9
:10589000044604F07DFFB0F5487F034604F1FF3174
:1058A000A8BF4FF448739E4206F101020DD1B0F536
:1058B000487F06D96D4B19889B78ADF832138DF867
:1058C00034332B4659465046CFE7164611F8012F80
:1058D000AA55E8E740F0C680A2F1040CDCF1000212
:1058E0004FF0030342EB0C028DF814308DF81520B5
:1058F00005AB0222E6E7092B40F091801546042310
:105900008DF8143055F8043F4FEA6308B8F1200FC2
:105910008DF815804FEA6323A8BF4FF020088DF85B
:1059200016308DF8178006AC03220521B04502DC45
:1059300005ABE21AC6E755F8040F10F0010706D1CF
:10594000042847D9036803F00F03022B0DD14FF051
:10595000010323704310637047121B0E4014A7709D
:10596000E070237105340136E0E7042B30D1234683
:105970004FF0020C03F802CBCDE901210093039311
:10598000FDF7D8FF814604F003FF0C28DDE9012173
:105990000AD8009B6070874201D1DC19E3E719F84F
:1059A0000740DC550137F6E723460C2003F8010FCA
:1059B00009F1FF3009F1080910F8017F03F8017FB0
:1059C0004845F9D12E23E372237363730E34CAE77B
:1059D000012B08D12346071F03F8022B7842784198
:1059E00060701C46BFE7092B09D10423237043686C
:1059F000581060705B12A370E7700434B3E7032B98
:105A00000AD121700368C3F30F10C3F34173C3EBD2
:105A1000800363701B12EEE727700134A3E7032BAA
:105A20007FF425AF05238DF81430C1F30F13C1F3B4
:105A30004171C1EB830164294FEA21238DF81510D0
:105A4000A8BF64218DF816308DF8171003328E42EE
:105A500005AB01DB0A1D35E7334412F8010F18715D
:105A60000136F4E7002A7FF402AF35E710B70000F3
:105A70000F4970B5F022002402FB04135D788542C3
:105A800003D001340A2CF7D170BDF0221846002152
:105A900004F0DEFA074A1368013BA34200D1146008
:105AA000002329461A461120BDE87040FFF74EBE7C
:105AB000787A0120A805002030B5B3B032AC0223BB
:105AC000054604F8C83D04F063FEC72828BFC72078
:105AD000691E0023984207DC421C2346FE21142045
:105AE000FFF734FE33B030BD013311F8012FE2541B
:105AF000F0E770B5B2B032AC0223054604F8C83DF9
:105B000004F046FEC72828BFC72006460023681EAB
:105B10009E420BDC06F13200FFF776FD2346721C35
:105B2000FF211420FFF712FE32B070BD013310F8D0
:105B3000012FE254ECE700002DE9F04F0128B9B045
:105B40008146884603DC1B20FBF7E4FC58E008682C
:105B5000C2072BD4042829D9036803F00F03042BB0
:105B600024D1FDF7E7FE0546D8F80400C3071FD48B
:105B700004281DD9036803F00F03042B18D1FDF787
:105B8000D9FE0646214BDFF890A01B68039300273F
:105B9000039BBB420EDC00962B461D4AC82106A87B
:105BA00004F07CFD06A8FFF7A4FFCCE7194DDBE766
:105BB000184EE7E70C2303FB07F202EB0A03294622
:105BC00052F80A00049304F0D9FD049B044618B966
:105BD000D3E9013B9C4201DB0137D9E70BEBC4025F
:105BE00031465BF834000593049204F0C7FDDDE90B
:105BF000042340B9536808F10801A9F1020098474D
:105C000039B0BDE8F08F0134E4E700BF40740120F3
:105C1000B8C30000B2BB0000708D01202DE9F04137
:105C20001F4F204AD7F8008005460023F0209845F2
:105C30000EDC0024F02000FB04F15318565C8EB1FA
:105C400001340A2CF7D11848BDE8F041FFF751BFE5
:105C500000FB03F154186478AC4201D1515CE9B9FE
:105C60000133E4E7F0223146184604F0F1F90F4918
:105C7000457051F8351085700222A0450270C0E9C8
:105C80000212C0E9046601DC01343C6000232946AD
:105C90001A461020BDE8F041FFF758BDBDE8F0817D
:105CA000A8050020787A012001C80000D8830120CF
:105CB00070B5FFF77FFD094EFF246FF0070505FB68
:105CC000046393F8FC37043B012B03D8E043C0B2D4
:105CD000FFF7A4FF013CF2D170BD00BFD8830120C3
:105CE0002DE9F041DFF8348006460F46002408EB2A
:105CF000C4031B79062B01D0032B09D1E5B23A4628
:105D000031462846FFF7DEFC10B12846FFF786FF34
:105D10000134FF2CEBD1BDE8F08100BFD883012016
:105D2000F8B5094F0546FF246FF0070606FB04731C
:105D300093F8FC37AB4203D1E043C0B2FFF76EFFEC
:105D4000013CF3D1F8BD00BFD88301202DE9F84F05
:105D5000FDF7DCFA584B1A68824284BF00221A60B1
:105D60001A6842F20F71821A8A420BD9534918609D
:105D700000235A181279073A022A0FD90833B3F5CB
:105D8000FF6FF6D1BDE8F88F0720FFF7C9FF8AF84B
:105D900000802EE00820FFF7C3FF3FE0FDF7BEFACA
:105DA000002814BF044601240020FDF7A3FB814610
:105DB0000020FDF7B3FB424D424E0746B9F1000FFC
:105DC00017D02B68002B70D133682C60002B6FD05C
:105DD000DFF8F8B0DFF8F0A09BF800304FF00108D2
:105DE000002BD1D10920FFF79BFF8AF800808BF8A8
:105DF0000080AFB133689BB92B6834601BB3DFF808
:105E0000C8B0DFF8C8A09BF800304FF00108002BA5
:105E1000C0D10920FFF784FF8BF800808AF800804A
:105E20002B6883B1284A1178904661B99C4238BFEB
:105E30002C602B68E31A312B05D90720FFF770FF80
:105E4000012388F80030326882B1204B19789846D7
:105E500061B9A24288BF34603368E41A312C05D995
:105E60000820FFF75DFF012388F800302B685BB145
:105E7000B9F1000F08D1144C227812B90720FFF7AE
:105E80004FFF00232B6023703368002B3FF47AAF61
:105E9000002F7FF477AF0D4C227812B90820FFF75E
:105EA0003FFF0023336023706CE7002FA2D1B9E7D6
:105EB000002FA1D1B4E700BF30700120D8830120AA
:105EC0002070012028700120247001202C700120F6
:105ED00037B50546FFF76EFC02A8002440F8044DD4
:105EE000FDF7F0FA21462046FEF7A0F9FEF71AFC6E
:105EF000FDF728FBFDF7FCFBFDF716FCFEF7AEFCFB
:105F0000FDF72EFA25B1FDF7C5FC0248FFF7F1FDBC
:105F100003B030BDF2C70000002301461A4611202D
:105F2000FFF714BC07B513128DF801208DF802306D
:105F30001314120E8DF800108DF803308DF8042024
:105F400001466B4605221320FFF700FC03B05DF805
:105F500004FB0A4601461220FFF76CBC70B50546EB
:105F60000C46FDF7E7F958B104F13200FFF74CFB9E
:105F70002B46224600211B20BDE87040FFF7E6BB00
:105F800070BD10B4144603460A46142021465DF83D
:105F9000044BFFF7DBBB000030B5084C01444FF069
:105FA000FF33884201D3D84330BD10F8015BDAB229
:105FB0006A4054F8222082EA1323F2E7D4C3000097
:105FC000FE2837B5044614D80B4B53F8300080B187
:105FD000416808308900FFF7DFFF02AD45F8040D86
:105FE0000920FFF711FB2B46042221461720FFF75B
:105FF000ADFB03B030BD00BFD8830120F8B5074624
:10600000FFF716FB4FF0FF3504460CB92846F8BDE4
:106010002668C6F30743152B0CD104F10801384656
:1060200004F0ACFB08B9C6F307252046FEF798FC40
:106030000446EAE71D2B08BF4FF0FF35F5E70000E7
:106040002DE9F047BF4CC04D9CB0FFF7C3FA206864
:10605000C0F580612844FDF7DDFB23680344064654
:1060600023607BB1B94F002E0FDC2B78FA2B40F068
:1060700030812368022B16DCFFF798FA10B101205B
:10608000FFF76CFA1CB0BDE8F0872068C0F58061AE
:106090002844FDF7BFFB2368034406462360FDF751
:1060A00035F93860DFE76878AC78831E182B00F28A
:1060B0000681DFE813F019002D00310035003800AB
:1060C000410004014B0080008A008E00A400E00023
:1060D000F1000401040104010401040104010401AC
:1060E000040104010401FF00FF2C0FD02046FFF73C
:1060F000BFFC974A002342F8343002EBC402214629
:106100001371132000931A46FEF710FE0320B7E721
:106110002046FFF783FDF9E72046FFF7A9FCF5E7E6
:10612000FFF7C6FDF2E7FFF745FB0020FFF7D0FEC3
:106130008848FFF7DEFCE9E7632CE7D8864B214669
:1061400053F824201520FFF775FBDFE7FFF770FAFF
:106150006FF007080446002CD8D02768C7F3074320
:10616000152B04D02046FEF7FBFB0446F3E704F1B1
:106170000806304604F00CFB05460530FFF744FAEC
:10618000FB20FFF7DDF91D20FFF7DAF9C7F3072041
:10619000FFF7D6F9E8B2FFF7D3F9C5F30720FFF709
:1061A000CFF9A8EB0407F3199D42DBDD16F8010BCC
:1061B000FFF7C6F9F7E7002300931A4619461D209A
:1061C000FEF7B4FDFDF766FBA0E72046FFF7F8FEFB
:1061D0009CE7FDF7B1F8614A00906421604B03A889
:1061E00004F05CFA022303A88DF80C3004F0D0FA16
:1061F00003AB024600211620FFF7A8FA86E7544FAA
:10620000002557F8354007EBC5035CB3D4F804808C
:1062100093F804A04FEA8806B01DFFF7F5F9FB20BC
:10622000FFF78EF9012006F10109FFF789F9E8B2BD
:10623000FFF786F95FFA89F0FFF782F9C9F30720C3
:10624000FFF77EF95046FFF77BF9083404EB0609A7
:10625000A1450BD8FFF7BEF906EB080001F068FC7A
:10626000FFF7B8F90135FF2DCBD14FE714F8010B3B
:10627000FFF766F9ECE70024FFF79CFA2246214677
:1062800000942346DA20FEF751FD4FF4FF622146C9
:106290002F4803F0DDFE95E7012C02D1FEF788FBC5
:1062A00034E7022C02D1FEF73FFD2FE70120FFF774
:1062B0000FFE2BE700231A4621461A209CE7A0F187
:1062C000C803052B3FF622AF00221146FAF792FFD2
:1062D0001CE7FB2B7FF4D3AE2268042A7FF7CCAEF9
:1062E000B5F8037040F2F6339F423FF7C8AE3B1D4E
:1062F0009A427FF7C1AEEB5CFE2B7FF4C0AE6878AC
:10630000AC781B2807F1FF367AD02DD807285ED04D
:10631000082837D001282CD1FF2C11D02046FFF7B8
:10632000A7FB6D790F4B00932146BB1E2A460A201E
:10633000FEF7FCFC064B43F8340003EBC404257164
:10634000781D9DE6447801204474012034700120BA
:10635000D8830120D4C70000D08B0120EBC70000F8
:10636000E6C700004A7401201D285BD04DD31E28CB
:1063700070D0A0F1C803052BE2D83F4A3146FAF7A6
:1063800039FFDDE7632CDBD86B79022B0CD0032BB4
:1063900014D0012BD4D1D5F80630384A5B0043F035
:1063A000010342F82430CBE7002EC9DDB91E344882
:1063B000FDF7DDFC314B43F82400C1E7AB79002B3E
:1063C0002E4B0CBF0022042243F82420B8E7632E92
:1063D000B6DC3246284903A803F016FE1CAB1E4467
:1063E00003A8002306F8643CFFF708FE0028A7DB9B
:1063F000224B214653F820201520FFF71BFA9FE778
:1064000031461D48FFF76CFC9AE7FF2C98D06A795B
:10641000022A95D81A4B00932146BB1E0B20FEF78B
:1064200085FC8DE7632EA8BF6326002303A9B34232
:106430000BDB1CAA26EAE6731344002203F8642C43
:1064400015200091731C2146E9E7EA185279CA54D5
:106450000133ECE7012C7FF473AF002E7FF770AFB0
:106460006B791BB1322BA8BF32231C4664235C43DB
:10647000044B1C6064E700BF49740120D08B0120ED
:106480004A74012004000020084B01221A60084AC7
:106490001368002BFCD0074B1868042390FBF3F023
:1064A0000638400040F00100704700BF00C00040C7
:1064B00000C1004008C500400120704710B5064CDF
:1064C000204600F009FF0549204600F06BFF044B11
:1064D00001221A6010BD00BF80780120801A0600DA
:1064E0004878012010B5064C204600F0F5FE05491D
:1064F000204600F057FF044B01221A6010BD00BF78
:106500003C790120801A06004C7801201FB500213B
:106510000E20FCF717FF01210F20FCF713FF0121CC
:106520000D20FCF70FFF1B4B1B491B681B4A8B42BE
:1065300012780FD84FF000730193002303938DF866
:10654000082004AB13E90E00154805B05DF804EB14
:1065500000F030BE13498B4202D84FF08063EBE766
:1065600011498B4202D84FF00063E5E70F498B4297
:1065700002D84FF08053DFE70D498B4202D84FF02D
:106580000053D9E70B498B4294BF4FF080434FF043
:106590000043D1E73000002048E801002C00002033
:1065A0006078012090D0030020A1070040420F0036
:1065B00080841E0000093D00002814DD0B68DA0706
:1065C00011D50D4A5B10012813600C4A09D04B68A5
:1065D000D90706D55B10022B09D0032B09D0012B5C
:1065E00003D002231360002070470023FAE703233F
:1065F000F8E70123F6E700BF300000202C00002060
:106600002DE9F8430C68E30704D40D20BDE8F843F6
:10661000FAF780BF64102FD4FCF792FEA0422BDB68
:1066200000212046FCF78EFE4FF4FA62012120463D
:1066300001F0B6FA00B3DFF86C8000254FF00109D5
:10664000002707264FF47A720121204601F0A8FAAC
:1066500090B12828C4BF09FA06F31F4316F1FF368C
:10666000F0D205F808700135052DE9D10122062187
:106670000920FDF7FBFA08B900200FE003460B22C2
:1066800043F8042F064900F1180411F8012F5200B5
:1066900042F0010243F8042F9C42F6D1BDE8F88392
:1066A0004F78012050780120F0B5002885B00C46C5
:1066B0002DDD0B6813F0010529D1042B27D91B68A8
:1066C00003F00F03032B22D14FF0007301930395C6
:1066D0008DF8085004AB13E90E000E480D4F00F082
:1066E00069FD266856F8033BC3F30F14C3F34173E7
:1066F000C3EB8404AC4207DD16F8011F384600F0F6
:1067000066FD01353070F5E7024800F05FFD0020BE
:1067100005B0F0BD6078012010B50468E30704D42B
:106720000D20BDE81040FAF7F5BE6410FF2C01D92A
:106730001720F6E7FFF7EAFEE1B2044800F047FD54
:10674000024800F043FD002010BD00BF607801202A
:1067500038B5074DFFF7DAFE0021284600F037FD77
:106760000446284600F032FD600040F0010038BDCC
:1067700060780120274A82B001210023ADF806305D
:10678000C2F8F015C2F8001519461A0102F180424C
:1067900002F5E0420133082BC2F81415C2F81015B7
:1067A000F3D11C4B4FF4E062C3F818250422C3F860
:1067B0001425C3F810250DF10602C3F82C2601227A
:1067C000C3F830261A60D3F80021002AFBD000223B
:1067D000C3F8002101225A600E4B1A46D3F8041167
:1067E0000029FBD00021C3F8041101219960D2F8DF
:1067F0001431002BFBD00020C2F81401C2F80005B0
:10680000BDF806301BB28342C8BFA3F50B70400031
:1068100002B070470070004008B5FFF7ABFF4000C2
:1068200040F0010008BD0000024A03480D21FEF7B8
:106830000DBF00BF18C8000080C8000070B5066812
:10684000F10705D54568EA0702D58468E30704D453
:106850000D20BDE87040FAF75DBE7610802E01D99C
:106860001520F6E76D10FF2D01D91620F1E7641011
:10687000FF2C01D91720ECE70A4B1B680BB9FFF777
:106880001DFEF1B2084800F00BFEE9B2064800F028
:10689000EBFCE1B2044800F0E7FC034800F06BFEBB
:1068A000002070BD48780120807801200C4B1B68C7
:1068B00070B506460D4614460BB9FFF713FEF1B24C
:1068C000084800F0EDFDE9B2064800F0CDFCE1B269
:1068D000044800F0C9FC0348BDE8704000F04BBE1E
:1068E0004C7801203C790120002808B507DD0B68B1
:1068F000DB0704D5302223211920FFF7D7FF002022
:1069000008BD00000128F8B536DD0D68EA0733D56B
:106910001A4B4C681B686D100BB9FFF7CFFDE9B23D
:10692000174800F0BDFD14F001050DD0C4F3470178
:10693000134800F099FC124800F01DFE18B1232006
:10694000FAF7E8FD0020F8BD042CF4D9236803F021
:106950000F03092BEFD154F8046F094F7610AE42A4
:10696000E9DD54F8041FCB0704D5C1F347013846CD
:1069700000F07AFC0135F2E70120E4E748780120D5
:106980008078012038B50468E20702D54568EB0736
:1069900004D40D20BDE83840FAF7BCBD6410802C4B
:1069A00001D91520F6E76D10FF2D01D91620F1E76A
:1069B000124B1B680BB9FFF781FDE4B2214610486A
:1069C00000F06EFDE9B20E4800F04EFC00210C48CC
:1069D00000F070FD20B14042400040F0010038BDA1
:1069E00001222146064800F058FD054800F033FC1E
:1069F0000028F1D0024800F031FCEDE74878012092
:106A00008078012038B5124B1B6804460D460BB93F
:106A1000FFF768FDE4B221460E4800F041FDE9B2FF
:106A20000C4800F021FC0B4800F0A5FD08B14042E5
:106A300038BD01222146074800F02FFD054800F02F
:106A40000AFC0028F4D00348BDE8384000F006BC3A
:106A50004C7801203C790120F8B5354E354D37682A
:106A600004466FB90D211D20FFF7CCFF5A2816D11F
:106A700001222A702A211D20FFF718FF012333600D
:106A800095F90030022B29D0032B44D0012B45D19E
:106A900021461D20FFF7B6FF4FF0FF3424E00F2101
:106AA0001920FFF7AFFF332805D102232B708F2267
:106AB00020211920E0E70D211E20FFF7A3FFC728A2
:106AC0000AD103233A462A211E202B70FFF7EEFE3F
:106AD0001B222A211E20CFE72F70CFE7012C13D1D4
:106AE00029211920FFF78EFF7F28C8BFA0F58070ED
:106AF0006FF07E039842B8BF1846C82358437F23DF
:106B000090FBF3F06043F8BD032C0BD12B2119202F
:106B1000C0E72D21FBE721461E20BBE74FF0FF34E5
:106B20000020EAE7052CF4D04FF0FF340020DFE727
:106B3000587801203400002008B50120FFF78CFFB1
:106B4000400040F0010008BD08B50320FFF784FFB6
:106B5000400040F0010008BD08B50520FFF77CFFAC
:106B6000400040F0010008BD38B5104B1B6813B958
:106B70000120FFF771FF0120FFF76EFF044603209D
:106B8000FFF76AFF05460520FFF766FF6D4304FB2C
:106B9000045400FB004002F087FE01F003FB03F009
:106BA0009DF9400040F0010038BD00BF5878012039
:106BB0000128F8B535DD0F68FB0732D54D6815F0B3
:106BC00001062ED1042D2CD92B6803F00F03092BBD
:106BD00027D16C68144B64101B68202CA8BF20249C
:106BE0000BB9FFF76BFCC7F3470122460F480F4F65
:106BF00000F053FC0435A64211DA0C4800F02BFBE0
:106C000018B9700040F00100F8BD384600F026FBCE
:106C1000400040F0010045F8040F0136EBE760004A
:106C2000F0E70120F0E700BF4878012080780120DC
:106C300000207047012070470020704700207047F7
:106C400000207047012070470020704700207047E7
:106C500000207047002070470020704700207047D8
:106C60000020704700207047002070477047704731
:106C700070470000024A03480F21FEF7E7BC00BF3F
:106C80000CC9000084C90000024610460132037896
:106C9000013B1F2BF9D9704708B5FFF7F5FF0378C3
:106CA000002B39D0222B00F1010011D1037823B140
:106CB000222B00F1010204D11046BDE80840FFF785
:106CC000E3BF5C2B02D1437803B1821C1046EDE791
:106CD0003A2BF2D02C2BF0D07B2B0BD1FFF7D4FF2B
:106CE0000378002BE9D07D2B01D10130E5E7FFF7D8
:106CF000D3FFF5E75B2B10D00246104612F8013B9C
:106D0000002BDAD0202BD8DD2C2B05D003F0DF01AF
:106D10005D2901D0222BF0D108BDFFF7B5FF037824
:106D2000002BCAD05D2BE0D0FFF7B6FFF7E708B520
:106D3000F0B1FFF7A9FF0378222B1AD07B2B1AD0D2
:106D40005B2B1AD0A3F13002092A05D92D2B05D1CE
:106D50004278303A092A07D8032009E0742B0ED074
:106D6000662B0ED06E2B0ED0181C18BF012040428F
:106D700008BD0420FCE70220FAE70120F8E705201F
:106D8000F6E70620F4E70720F2E738B5FFF77CFFC7
:106D900003782D2B11D101304FF0FF34431E002119
:106DA0000A2501E005FB012113F8012F303AD0B28A
:106DB0000928F7D904FB01F038BD0124EEE710B52E
:106DC0001446FFF761FF0378222B02D000230B70DB
:106DD00010BD621E01300378222BF7D0002BF5D0B6
:106DE0005C2B07D0441C002AF0DD01F8013B013A7E
:106DF0002046F0E74378622B00F1020409D0662BAD
:106E000009D06E2B09D0722B09D0742B08BF09232F
:106E1000E9E70823E7E70C23E5E70A23E3E70D2387
:106E2000E1E710B50446FFF737FF0346A3421846D3
:106E300005D90278013A1F2A03F1FF33F6D910BDB4
:106E400008B590B1037883B1FFF71EFF037803F014
:106E5000DF035D2B09D0FFF71FFF03782C2B08BF42
:106E60000130BDE80840FFF70FBF002008BD38B56E
:106E70000D1E0DDD03785B2B0AD10130FFF704FFF7
:106E80000124A54205D0FFF7DBFF10B10134F8E77C
:106E9000002038BD38B5154609B100230B70F8B194
:106EA0000378E3B1FFF7F0FE03782C2B044603D1FF
:106EB0000130FFF7E9FE044623787D2B0FD019B18E
:106EC0002A462046FFF77BFF2046FFF7E5FE0378C2
:106ED0003A2B05D10130BDE83840FFF7D5BE002080
:106EE00038BD2DE9F0410D469AB004462F789FB386
:106EF0002E21284603F035FC804690B1461B303FDA
:106F0000092F13D82846FFF740FF01462046FFF718
:106F1000AEFF044604B3B8F1000F1DD0013635446E
:106F2000E4E7284603F034FC0646E8E723787B2BA9
:106F300011D1601C642201A9FFF7ACFF044658B1CF
:106F40003246294601A803F02BFC0028E2D0204657
:106F5000FFF7A2FEEEE7002420461AB0BDE8F0815C
:106F600038B50D1E04461CDDFFF7E1FE012807D1F0
:106F7000601C012D00D138BDFFF762FF013DF8E72D
:106F800002280ED100221146601CFFF783FF012D5D
:106F9000F1D0FFF755FF00221146FFF77BFF013DBF
:106FA000F5E70020E7E7F8B50C1E074615461E4634
:106FB00013DDFFF7BCFE02280FD132462946781CAC
:106FC000FFF768FF012C00D1F8BDFFF739FF32460B
:106FD0002946FFF75FFF013CF4E70020F4E710B516
:106FE0000446C8B1FFF750FE03787B2B0AD101306D
:106FF000002400221146FFF74DFF68B1FFF74CFE59
:107000000134F6E75B2B06D101300024FFF718FFAF
:1070100010B10134FAE70024204610BD002870B5F5
:1070200014DD0D68EB0711D56D10013DFDF798FDDE
:1070300000264FF0FF3460B916B3304603F0A8FBCA
:1070400001463046BDE87040FCF791BE4FF0FF3579
:10705000ECE70368C3F30742152A0BD1C3F30723F8
:107060009C42B8BF1C469D4201D100F10806FDF7C5
:1070700077FCE0E71D2A04BF00264FF0FF34F6E757
:10708000601C400040F0010070BD000010B50868B1
:107090000C46FCF74FFCFEF7B1FF0028A2BF034BE4
:1070A000626843F82020002010BD00BFD08B012073
:1070B00008B50868FCF73EFCFEF7A0FF0028AABF51
:1070C000024B012053F8200008BD00BFD08B0120E7
:1070D00008B50868FCF72EFCFEF790FF0028ACBF4F
:1070E0000420002008BD0000024A03480421FEF7E6
:1070F000ADBA00BF20CA00001ACA000008B5FCF7EC
:1071000025FBFCF7EBFBFEF7B5FA0448FEF7F1FCB4
:10711000FDF766FEBDE80840FEF7CABD6FCA000075
:10712000FBF77CBF38B50025057329B90B4B0C4A1A
:107130000C48252102F0FAFE01600B4951F822208B
:10714000027151F8233083719DF8103051F82330CB
:1071500043710223C371856038BD00BF87CA000038
:10716000E6CA000095CA000044CB000084B00DF1CF
:10717000100C0CE90E009DF808100268002301298C
:10718000C2F80035039B12D00BD303290CD0C2F8F0
:107190005435019BC2F824350123C2F8003504B0F0
:1071A000704743F00203F2E743F00403EFE743F0D4
:1071B0000603ECE710B485B001AC84E80E0094E857
:1071C0000E0005B05DF8044BFFF7D0BF70470368B1
:1071D000C3F81C15D3F80821002AFBD0D3F81805F2
:1071E0000022C3F80821C0B27047000007B5094B60
:1071F00009490A484FF080421A6000229A60022230
:107200001A710F2300930E220D23FFF78BFF03B09B
:107210005DF804FB747801200030024060780120A2
:107220002DE9F84380460D46174601EB02090C464E
:107230004C45A4EB05060BD0D8F8003014F8011B20
:107240001B68404698470028F2D13046BDE8F883D5
:107250003E46FAE77047203000F03CBA203000F09C
:107260002BBA203000F03CBA38B5437F0D460BB93D
:10727000002038BD00F16804204600F039FA0028EB
:10728000F6D12046294600F008FA0120F1E7000077
:107290002DE9F0411E4600254FF47A73C0E90153F1
:1072A0000C4B044640F8203B8846174600F0ECF9AA
:1072B00004F1680000F0E8F99DF8183063769DF855
:1072C0001C302676C4E90487A37665772046BDE89E
:1072D000F08100BF2CCB0000F0B5837E2E4C2F4DEB
:1072E0000121C17654F82320437E54F8233012F054
:1072F000200F14BF2F464FF0A04702F01F0213F0DB
:10730000200F03F01F0308BF4FF0A04502F5E07205
:1073100003F5E07340F20C6647F8226045F82360FD
:1073200003694FF0CC72C3F8242503690622C3F821
:107330000025827E036954F82220C3F80825427E86
:10734000036954F82220C3F80C2590F91830144A28
:107350005C0903F01F03994004F1600342F8231015
:1073600090F91830002BBDBF03F00F0302F6FC327A
:10737000D2189B18B5BF40234022137683F8002310
:1073800090F918300122590903F01F0302FA03F3A0
:10739000034A42F82130F0BD44CB00000003005006
:1073A00000E100E0C37EA3B103690022C3F8002519
:1073B0000A4B99420ED90A4B994294BF4FF0806113
:1073C0004FF0C8610369C3F8241503690622C3F8A6
:1073D000002570474FF0CC71F4E700BFA086010094
:1073E00090D003002DE9F041044688461F4615461B
:1073F000002A50D000F12006304600F059F92369E8
:10740000C3F88885236901221A622369C3F83465A9
:107410002369C3F8385523691A602269D2F84C31C0
:107420001BB9D2F82431002BF8D00023C2F84C311C
:107430002269D2F85C311BB9D2F82431002BF8D084
:107440000023C2F85C3122696FB9D2F8243153B9F4
:107450000123D3612369D3F84821002AFBD00022FD
:10746000C3F8482109E0012353612369D3F80421BB
:10747000002AFBD00022C3F804212369D3F8242179
:1074800012B10022C3F824212369D3F83C052066F9
:10749000C0B2BDE8F0811046FBE70123FFF7A2BFB1
:1074A00010B5044680F8B010683000F001F90123EF
:1074B000637710BDF8B500234377036990F8B020D7
:1074C000C3F88825036901261E62036900F1680577
:1074D0000446C3F8445528460F4600F0FBF82369DC
:1074E000C3F8480523699E602369D3F850211AB96F
:1074F000D3F82421002AF8D00022C3F850212846CE
:1075000000F0E8F8236930B1D3F860211AB9D3F854
:107510002421002AF8D00022C3F8602123696FB922
:10752000D3F8242152B90122DA612369D3F8482122
:10753000002AFBD00022C3F8482109E001225A6149
:107540002369D3F80421002AFBD00022C3F80421C8
:107550002369D3F8240168B10022C3F824212369E8
:10756000D3F8C404C3F8C404022803D004280CBF11
:1075700003200420F8BD0121FFF79CBF70B54369CB
:10758000D3F86421044692B10022012500F12006BF
:10759000C3F864210577304600F08AF86369C3F8C0
:1075A000346563694022C3F8382563691D636369E4
:1075B000D3F86821DAB10025C3F8685104F16806F0
:1075C000012363772577304600F072F8D4F8B430A1
:1075D00003B19847636965773046C3F8446500F0A6
:1075E00079F86369C3F84805636901225A636369DE
:1075F000D3F8042162B10022C3F80421237F3BB1F8
:107600006369D3F83C05D4F8B830206603B19847D5
:107610006369D3F8242152B10022C3F8242163699D
:10762000D3F8D024C3F8D024636901225A6170BD15
:107630000148FFF7A3BF00BF807801200148FFF792
:107640009DBF00BF3C79012007B514231322CDE96B
:1076500000324FF04022114604230848FFF718FE7D
:10766000074A08481E231F21CDE900310323114694
:10767000FFF70EFE03B05DF804FB00BF8078012029
:10768000003000403C79012008B54022002102F082
:10769000DFFC0022C0E9102208BD026C10B5531CAB
:1076A000446C03F03F039C421CBF8154036410BD33
:1076B0000023C0E910337047D0E9102393421FBF65
:1076C000C25C013303F03F03436414BF10464FF024
:1076D000FF307047D0E91030181A48BF403070476B
:1076E000D0E91023934214BFC05C4FF0FF307047C5
:1076F000036C406C013303F03F031B1A584258419E
:10770000704700000649074A074B9B1A03DD043BFC
:10771000C858D050FBDC00F013F8F8F791FD0000DA
:10772000E8CF00000000002040020020FEE7FEE756
:10773000FEE7FEE7FEE7FEE7FEE7FEE7FEE7FEE721
:10774000394B1A680D2A08D14FF080420021C2F847
:107750000C11C2F81011C2F838151B680D2B46D158
:107760004FF08052314BD2F80414C3F82015D2F8F0
:107770000814C3F82415D2F80C14C3F82815D2F84D
:107780001014C3F82C15D2F81414C3F83015D2F81D
:107790001814C3F83415D2F81C14C3F84015D2F8E5
:1077A0002014C3F84415D2F82414C3F84815D2F8AD
:1077B0002814C3F84C15D2F82C14C3F85015D2F87D
:1077C0003014C3F85415D2F83414C3F86015D2F845
:1077D0003814C3F86415D2F83C14C3F86815D2F80D
:1077E0004014C3F86C15D2F84424C3F870250E4B2E
:1077F0001B680D2B09D14FF08043D3F80024D2072A
:1078000044BF6FF00102C3F80024094AD2F888305F
:1078100043F47003C2F88830BFF34F8FBFF36F8F0C
:10782000044B054A1A6070473001001000C0004048
:1078300000ED00E0380000200090D00301207047E8
:1078400003681322DB69184770470369C3F81C15E6
:107850000369D3F81C21002AFBD00022C3F81C21A5
:107860000120704710B490F95C30144C5909012282
:10787000203103F01F0302FA03F344F821300369B7
:107880005DF8044B0421C3F8081303695A600369C7
:10789000DA6003690022C3F8002502694FF0FF3364
:1078A000C2F80C350269C2F814350269C2F808350D
:1078B00002691430C2F81035FFF7FABE00E100E0AB
:1078C0001430FFF707BF1430FFF70ABF1430FFF77B
:1078D000F3BE0000036990F85E2010B5C3F80C25D4
:1078E000036990F85D20C3F8142590F861200369BE
:1078F000012A01BF90F85F40C3F81045036990F872
:10790000604006BFC3F8084503690022B1F5966FD1
:10791000C3F86C2569D9B1F5166F69D9B1F5965FD1
:1079200069D9B1F5165F68D9B1F5615F67D9B1F56D
:10793000964F66D9B1F5E14F65D9B1F5164F64D9C7
:10794000B1F5614F64D9B1F5963F64D9B1F5E13F26
:1079500063D9B1F5613F63D9364B994263D9B1F52B
:10796000E12F63D9B1F5612F94BF4FF070634FF0F1
:1079700080530269C2F8243503690422C3F8002544
:1079800001690023C1F808310169C1F81C3101699E
:1079900001230B6001698B600169C1F8042390F930
:1079A0005C20510902F01F0293406031224A42F8E4
:1079B000213090F95C30002BBDBF03F00F0302F6BD
:1079C000FC32D2189B18B5BF60236022137683F86F
:1079D000002390F95C300122590903F01F0302FAD9
:1079E00003F3154A42F8213010BD4FF49E23C0E73F
:1079F0004FF41D23BDE7114BBBE7114BB9E7114B0A
:107A0000B7E7114BB5E7114BB3E74FF41D03B0E7F0
:107A10004FF46B03ADE70E4BABE74FF0EB73A8E70A
:107A20004FF06C73A5E74FF08063A2E74FF0E86377
:107A30009FE700BF90D0030000E100E000B013001A
:107A40000050270000F03A0000A04E0000C0750072
:107A500000903A012DE9F0411E4600254FF47A735B
:107A6000C0E901530D4B044640F8143B17468846C5
:107A7000FFF70AFE0A4AC4F8108084F85C7052F8D6
:107A8000263084F85D309DF8183052F8233084F8A1
:107A90005E3084F861502046BDE8F081D8CB00000C
:107AA00044CB000010B50369D3F8082104464AB15D
:107AB000D3F818151430C9B2FFF7EFFD236900227F
:107AC000C3F8082110BD00000148FFF7EBBF00BF5D
:107AD000F879012007B522230093022221230349CC
:107AE0000348FFF7B7FF03B05DF804FB0020004038
:107AF000F879012008B102F079BD70470A4B196886
:107B00000A4B30B5D3F804050C060D0A44EA00020E
:107B10004FF47A712B46A2FB014501FB0355E00BA4
:107B200040EA454030BD00BF5C7A012000100140B2
:107B300038B5044648B1FFF7E1FF054600F01AF8F2
:107B4000FFF7DCFF401BA042F8D338BD074B0022F3
:107B5000C3F8042182B0D3F80431054A0193019B94
:107B600013680133DBB2136002B0704700100140AC
:107B70005C7A01207047704708B500F067F8FFF79E
:107B8000FAFF0120FFF7D4FFFFF7B8FA034CFFF725
:107B9000C7FA002CFBD0AFF30080F8E7000000002C
:107BA00038B5174B174D53F82030174813F0200FF6
:107BB0004FF0010403F01F0304FA03F408BF4FF071
:107BC000A04000292B681149B3FBF1F300F5A26036
:107BD00002FB03F321464FF00A02B3FBF2F314BF9A
:107BE0002246002200F014F842F2107358434FF47A
:107BF0007A722B68B3FBF2F3B0FBF3F038BD00BF31
:107C000044CB0000380000200003005040420F0029
:107C100030B504680C40944206D1013B002BF8D1EA
:107C200012E0013B002B0FD004680C409442F8D1C5
:107C3000002405680D40954204D101349C42F8D1DE
:107C4000002002E0201C00E0181C30BD0D4BE0229B
:107C500083F811234FF40032C3F880211A604FF0EB
:107C600080430122C3F818259A6003F58833002168
:107C7000C3F808150221C3F80413C3F844131A60AB
:107C8000704700BF00E100E0014B1860704700BF83
:107C900054000020222837B50CD84B4B53F8203025
:107CA000052B00F0828007D8032B12D07BD8022B43
:107CB00000F08180002074E01D2B78D003D81C2BAD
:107CC000F8D1052206E01E2B73D01F2BF2D108221B
:107CD00000E002223D4B196808296EDD0A296FDD9C
:107CE0000D29B5BF0C240E24022303233848C0F805
:107CF000F0350123C0F8003500200546030103F1EB
:107D0000804303F5E04301300828C3F81455C3F855
:107D10001055F3D12F4B18682F4B1B6800021B0323
:107D200003F4805300F4E0601843294BC3F81805AE
:107D3000C3F81425C3F810250DF10602C3F82C264C
:107D40000122C3F830261A60D3F80021002AFBD0A4
:107D50000022C3F8002101225A601D4B1A46D3F8B5
:107D600004010028FBD00020C3F804010120986022
:107D7000D2F81431002BFBD00023C2F81431BDF926
:107D800006209A42124AB8BFADF80630A142C2F8A6
:107D90000035BDF9060004D035BF611A091BC84083
:107DA000884003B030BD032294E7042292E7062204
:107DB00090E707228EE701228CE70824002395E74D
:107DC0000A24012392E700BF44CB00004C000020AE
:107DD0000070004050000020687A0120222830B551
:107DE0003CD8224B53F82000214B00221D4653F86B
:107DF0002240B4F1FF3F32D11E4C45F822006FEA19
:107E000041411D4D1D4B246853F822306FEA51410A
:107E100025F81210012101FA04F4C3F86005013CB1
:107E2000C3F8640505EB4202C3F86805C3F86C05A6
:107E30000020C3F80015C3F80C05C3F80405C3F807
:107E40000845C3F81405C3F81005C3F82025C3F886
:107E50002415C3F82815C3F82C05996030BD844259
:107E6000CAD00132042AC2D1F8E700BF44CB0000D7
:107E70003C00002054000020607A012000CC00006B
:107E8000222815D8114B124A53F8203013F0200F36
:107E900008BF4FF0A04203F01F03032908D8DFE812
:107EA00001F00210080C03F5E073002142F82310E2
:107EB000704703F5E0730C21F8E703F5E073042144
:107EC000F4E703F5E0730321F0E700BF44CB0000C3
:107ED00000030050222813D80A4B53F820000A4B05
:107EE00010F0200F4FF0010200F01F0008BF4FF00C
:107EF000A043824011B9C3F80C257047C3F8082588
:107F0000704700BF44CB000000030050222810D867
:107F1000094B0A4A53F8203013F0200F08BF4FF0E6
:107F2000A04203F01F03D2F81005D84000F0010072
:107F300070470020704700BF44CB00000003005092
:107F40002DE9F04106460D4601EB02080C4644457A
:107F5000A4EB050707D0336814F8011B1B683046F3
:107F600098470028F3D13846BDE8F0812DE9F0416B
:107F7000C1F30A57A7F2FF35132D82B002460B4614
:107F80000C464FEAD178064633DC002D4EDB3C49E7
:107F9000294103EA0100104326D049080B4052EA68
:107FA00003060CD04FF48023132D24EA010143FA79
:107FB00005F444EA01040CBF4FF0004600263149A5
:107FC00001EBC8082346D8E9004532462046294639
:107FD00001F01EFBCDE9000122462B46DDE9000140
:107FE00001F014FB02460B461046194602B0BDE8EC
:107FF000F081332D07DDB5F5806FF5D101F008FB79
:1080000002460B46F0E7A7F213474FF0FF31F94065
:108010000842E9D049080842D1D04FF0804320EA15
:10802000010143FA07F741EA0706C8E721F00041DA
:108030000143D9D0C3F3130101434E420E43114D06
:108040005C0C360B640406F4002305EBC80243EA1B
:108050000401D2E900450B4602462946204601F0BC
:10806000D7FACDE9000122462B46DDE9000101F0F7
:10807000CDFA21F00041024641EAC873B4E700BFDF
:10808000FFFF0F0010CC0000F8B5C1F30A57A7F2AC
:10809000FF35132D02460B460C4610DC002D29DB64
:1080A0008C461D4929410B422AD04FF400242C4113
:1080B000644424EA0104002621463046F8BD332DED
:1080C00005DDB5F5806F1ED010461946F8BDA7F244
:1080D00013474FF0FF3121FA07F73842F4D001235C
:1080E000C5F1330503FA05F5461928BFE41826EA59
:1080F0000706E1E7013501F0004407D00026DBE781
:108100000028D2D1E0E701F083FAF8BD44F07F54B3
:1081100044F440140026CFE7FFFF0F0030B51F4A9C
:1081200021F00043934287B01CDD1D4A934205DDD8
:1081300002460B4601F06AFA07B030BD02AA00F011
:108140008FF800F003000128DDE9042312D0022893
:108150001CD0A0B1DDE9020100F066FB01F1004195
:1081600007B030BD002300930022002301F084F803
:1081700007B030BDDDE9020100F056FBDCE7012469
:10818000DDE90201009401F077F8D5E70124DDE98B
:108190000201009401F070F8E0E700BFFB21E93F25
:1081A000FFFFEF7F2DE9F04F8BB004460D4600F046
:1081B00079FA294B93F900A0BAF1FF3F06460F4622
:1081C00012D022462B462046294601F071FE8346F6
:1081D00050B94FF000084FF00009204629464246AA
:1081E0004B4601F03DFE20B9304639460BB0BDE8A4
:1081F000F08F0122194BCDF820B00092CDE9044553
:10820000CDE902450193BAF1000F17D042464B4623
:108210004046494601F0DCFCBAF1020FCDE9060107
:108220000ED101F0A1FE21230360089B73B9DDE9A3
:108230000667304639460BB0BDE8F08FCDE90689B8
:10824000684601F055F90028EFD1EAE701F08CFE0D
:10825000089B0360EBE700BF5800002020CC000023
:108260002DE9F047CA4B21F000479F4290B080466D
:10827000894640F38F80C74B9F420C46924626DCCE
:108280000029B9A3D3E9002340F38F8001F0BEF9A0
:10829000C14B9F4204460D4600F04781B4A3D3E989
:1082A000002301F0B3F902460B46CAE90023204639
:1082B000294601F0ABF9AEA3D3E9002301F0A6F9FA
:1082C0000125CAE90201284610B0BDE8F087B34B8A
:1082D0009F4240F38980B24B9F4200F31C813D15C1
:1082E000A5F21645A7EB055319461F46064601F0B1
:1082F000F5FD01F0D9FA8046894642464B463046A4
:108300003946CDE90A8901F081F90022A54B01F037
:1083100035FB8946804601F0E1FD01F0C5FA0646CD
:108320000F4632463B4640464946CDE90C6701F0D0
:108330006DF900229B4B01F021FB00220023CDE9C7
:108340000E0101F083FD002800F06081002330461B
:108350003946002201F07AFD002814BF01230223D0
:10836000914A019202212A4600910AA8514600F042
:1083700083FB002C054614DADAF80420DAF80C3016
:1083800002F1004203F100434542CAF80420CAF852
:108390000C3006E000200021C2E90089C2E9020198
:1083A0000025284610B0BDE8F08701F031F97A4B7E
:1083B0009F4204460D4600F00B816DA3D3E90023D4
:1083C00001F026F902460B46CAE900232946204659
:1083D00001F01CF966A3D3E9002301F019F94FF06D
:1083E000FF35CAE90201DCE700F0FCFF62A3D3E934
:1083F00000238046894601F0C1FA00226B4B01F050
:1084000007F901F06BFD054601F04EFA56A3D3E9DA
:108410000023CDE9060101F0B1FA02460B464046C1
:10842000494601F0F3F852A3D3E900238046894678
:10843000DDE90601CDE9028901F0A0FA1F2D02460F
:108440000B46CDE9042340F3B380DDE90423DDE9E5
:10845000020101F0DBF8804689463F15C9F30A5353
:10846000FB1A102B40F3B18045A3D3E90023DDE9CB
:10847000060101F083FA8046894602460B46DDE993
:10848000020101F0C3F802460B46DDE90201CDE925
:10849000082301F0BBF842464B4601F0B7F83AA377
:1084A000D3E9002380468946DDE9060101F066FA3A
:1084B00042464B4601F0AAF80B46CDE904010246BC
:1084C000DDE9080101F0A2F8C1F30A53FF1A312FC8
:1084D0008046894600F39C809DED087BCAE90089AF
:1084E0008DED027B42464B46DDE9020101F08EF83C
:1084F000DDE9042301F08AF8002CCAE90201BFF685
:1085000050AF09F1004401F100436D42CAE9008413
:10851000CAE9020345E702460B4601F077F8002559
:10852000CAE90201CAE900013BE715A3D3E9002328
:1085300001F06CF814A3D3E900230D46044601F0C2
:1085400065F802460B46CAE900232946204601F099
:108550005DF80DA3D3E9002301F058F80125CAE91D
:1085600002011EE7AFF3008000004054FB21F93FF9
:108570003163621A61B4D03D83C8C96D305FE43F96
:108580000000601A61B4D03D7370032E8A19A33BBA
:10859000FB21E93F7BD90240FB21F93FFB21394117
:1085A000FFFFEF7F00007041A8CC00000000E03F1B
:1085B0004046494601F02AF8394B6A1E804653F876
:1085C0002230BB4289463FF448AFCAE9008989E7B7
:1085D0002BA3D3E9002301F01BF82BA3D3E900233D
:1085E0000D46044601F014F802460B46CAE9002382
:1085F0002946204601F00AF823A3D3E9002301F01D
:1086000007F84FF0FF35CAE90201CAE60323A7E6DF
:108610001FA3D3E90023DDE9060101F0AFF9064607
:108620000F4602460B46DDE9080100F0EFFF8046E9
:10863000894602460B46DDE90801CDE9028900F0D2
:10864000E5FF32463B4600F0E1FF13A3D3E90023E8
:1086500006460F46DDE9060101F090F932463B4639
:1086600000F0D4FF02460B4640464946CDE90423BC
:1086700000F0CCFF80468946A7E700BFAFF300803B
:108680000000601A61B4D03D7370032E8A19A33BB9
:108690000000002E8A19A33BC14920259A837B390B
:1086A00028CC00005E4A8A432DE9F04104460D467D
:1086B00000F0958000290B460646844656DD0F15CE
:1086C00000F0A580C3F31303A7F2FF3743F4801330
:1086D0004FEADC72F80702EB43034FEA4C0504D57E
:1086E000ED0F05EB43034FEA8C0500267F10B446DF
:1086F00016224FF400110CEB010098424FEAD5749A
:108700004FEA450503DC1B1A00EB010C0E44013A4D
:1087100004EB43034FEA5101EDD110469646202465
:108720004FF0004209E051D05B00013C03EBD573F0
:108730004FEA52024FEA450537D0634502EB0E017E
:10874000F1DD002901EB020E0ADBE046A3EB0C038E
:10875000A94288BF03F1FF336D1A1044C446E3E712
:10876000BEF1000FF1DB0CF10108EFE721F0004250
:10877000024329D0002942D10146CA0A153B4905C6
:10878000002AFAD012F4801001D044E06046520072
:10879000D40200F1010CF9D5CCF1200401FA0CFC53
:1087A000E1401F1A41EA02038CE72B4321D1440820
:1087B000731003F17F53F20703F5001348BF44F031
:1087C000004403EB07512046BDE8F081A942ABD835
:1087D000002901EB020EC3DB98460023BCE70246EA
:1087E0000B4601F0CBF822462B4600F011FFBDE806
:1087F000F081411C16BF421C01365408D8E70246DE
:1088000000F004FF02460B4601F0E2F9DCE71A46ED
:1088100031463B46B6E78C4620244FF0FF30BFE799
:108820000000F07F000000002DE9F04F21F000482B
:10883000B8F1795F85B006460F4692469B466BDAE3
:1088400001F04CFB002800F0E18032463B46304608
:10885000394601F093F874A3D3E9002304460D468A
:1088600001F08CF872A3D3E9002300F0D1FE224678
:108870002B4601F083F870A3D3E9002300F0C6FE75
:1088800022462B4601F07AF86DA3D3E9002300F0CD
:10889000BFFE22462B4601F071F86BA3D3E90023FB
:1088A00000F0B4FE22462B4601F068F868A3D3E935
:1088B000002300F0ADFE22462B4601F05FF8CDE923
:1088C00000010022664B2046294601F057F8DDE9F9
:1088D0000023804689462046294601F04FF852463B
:1088E00004460D465B463046394601F047F80246DD
:1088F0000B462046294600F089FE02460B464046BC
:10890000494600F083FE02460B460020554900F020
:108910007DFE05B0BDE8F08F02460B4601F02EF853
:1089200041A3D3E9002304460D4601F027F840A3F4
:10893000D3E9002300F06CFE22462B4601F01EF81E
:108940003DA3D3E9002300F061FE22462B4601F04F
:1089500015F83BA3D3E9002300F05AFE22462B462C
:1089600001F00CF838A3D3E9002300F04FFE2246B3
:108970002B4601F003F836A3D3E9002300F048FEAC
:108980002B46224600F0FAFF374B9845CDE900010F
:1089900097DD364B98453EDCA8F5001300220020F9
:1089A00030499046994600F031FECDE9020100229F
:1089B0002B4B2046294600F0E1FF42464B4600F093
:1089C00025FEDDE90023804689462046294600F041
:1089D000D5FF524604460D465B463046394600F008
:1089E000CDFF02460B462046294600F00FFE024608
:1089F0000B464046494600F009FE02460B46DDE9BB
:108A0000020100F003FE05B0BDE8F08F154900201B
:108A100005B0BDE8F08F9FED107B4FF000088DEDA5
:108A2000027BDFF84C90C2E7D43888BEE9FAA8BDD3
:108A3000C4B1B4BD9EEE213EAD529C804F7E923EAD
:108A40009015CB19A001FA3E7751C1166CC1563F63
:108A50004C5555555555A53F000000000000E73F17
:108A60000000E03F0000F03F3233D33F0000E93F19
:108A70000000D23F000000002DE9F04FADF5197D58
:108A8000BE4CA29EBE4D54F826600793D41E85FBB3
:108A90000475E417C4EBA50424EAE4741D46631CC2
:108AA000A3EB8303013D02EBC30305937319049603
:108AB0000994019503900B91A4EB05071AD43B444C
:108AC000002400255E1C0DF18008DDF88C9208E082
:108AD00059F8270000F0E8FE0137B742E8E8020144
:108AE00008D0002FF4DA013720462946B742E8E8DB
:108AF0000201F6D1049B002B079B4FEAC3030293AC
:108B00002ADB039A20A902EB030801EB0309049B6B
:108B100072AA02EBC30B0DF5E07A019B002B4FF01C
:108B200000064FF0000711DB039C4D4675E9022358
:108B3000F4E8020100F022FF02460B4630463946B7
:108B400000F066FD444506460F46EFD1EAE80267AD
:108B5000DA4509F10809E0D1DDE90204049920446D
:108B60008B0082460BA8A3F10802C31808930CAB34
:108B700013440A938B4698AB03EBCB03BBF1000F76
:108B800053E9284529DD70AB03EBCB080DF1300923
:108B900000227C4B2046294600F0F0FE01F09EF9B1
:108BA00000F082FE0022784B06460F4600F0E6FEFB
:108BB00002460B462046294600F028FD01F08EF9BA
:108BC00078E9022349F8040B3946304600F020FDCD
:108BD00070AB984504460D46DAD1DDF81490204676
:108BE00029464A4600F088FC00224FF07F53044695
:108BF0000D4600F0C3FE00F0FBFB0022634B00F0CB
:108C0000BDFE02460B462046294600F0FFFC0D46FD
:108C1000044601F063F9804600F046FE0B4602462A
:108C20002946204600F0F2FC4B46002B06460F4634
:108C300040F3E1800BF1FF320CA9C9F1180351F8A0
:108C4000225045FA03F101FA03F30CA8EB1A40F89D
:108C50002230C9F11705884443FA05F5002D2CDDB3
:108C6000BBF1000F08F1010840F381820C9C002C3D
:108C700040F0A780BBF1010F0AD00CA9012251F8E6
:108C8000044F531C002C40F09E809B451A46F6D1A1
:108C9000059B002B0EDD012B00F0D980022B09D1A2
:108CA0000BF1FF320CAB0CA953F82230C3F31503C0
:108CB00041F82230022D00F0AF8000220023304620
:108CC000394601F0C3F8002800F05382049B0BF1F1
:108CD000FF394B4510DC0BF180430CAA013B08988F
:108CE00002EB8303002253F80419834242EA010293
:108CF000F9D1002A40F0B680049B0CAA013B52F83F
:108D00002330002B40F0A1800A9A012352F8041965
:108D100001330029FAD05B440BF101099945069310
:108D20004CDC099A079909EB020801EB0B0508F1E5
:108D3000804802EB030BA39B08F1FF3803EB880884
:108D400070AB03EBC909A39B20A903EB8B0301EBD9
:108D5000C505029358F8040F00F0A6FD0B460199D3
:108D60000246002905F1080BC5E900234FF0000673
:108D70004FF000071CDB039C0CE000BFF0CD0000AF
:108D8000ABAAAA2A0000703E0000704100002040FB
:108D900075E90223F4E8020100F0F0FD02460B46FB
:108DA0003046394600F034FC544506460F46EFD1B4
:108DB000029B9845E9E802675D46CBD1DDF818B023
:108DC000D9E6012300220CA9C4F180749B4541F827
:108DD00022400EDD51F8232001EB8B0001EB8303D1
:108DE0006FF07F4100E01A688A1A43F8042B83422F
:108DF000F9D101244CE706D10BF1FF330CAA52F84C
:108E00002350ED152AE700227B4B01F03DF80028A6
:108E100040F0A381054650E732463B4600207749A3
:108E200000F0F4FB06460F46002C3FF446AF059ACF
:108E30007249002000F060FB02460B46304639467E
:108E400000F0E4FB06460F4637E7012363E70BF12A
:108E5000FF320CAB0CA953F82230C3F3160341F8D0
:108E6000223027E70CAB059A53F82930183ACDE9A0
:108E7000068505926BB909F18043013B0CA901EB12
:108E8000830353F8041909F1FF39183A0029F8D07F
:108E90000592059A5949002000F02EFBB9F1000F08
:108EA00004460D46C0F2C0814FEAC90370AA02EB26
:108EB000030808930CAB03EB8906DFF844B14FF0CD
:108EC000000A08F10807043656F8040D00F0ECFC1F
:108ED00022462B4600F052FD5B4667E902015246EE
:108EE0002046294600F04AFD0CAB9E4204460D4642
:108EF000EAD148AB03930193CDF8149009F1010333
:108F0000DDF810900293C3464FF0000AB9F1000F4C
:108F1000C0F22A81DFF8EC805D4635A3D3E9002357
:108F200000260027002403E0544510DCF8E8022363
:108F3000F5E8020100F022FD02460B4630463946B4
:108F400000F066FB0134A14506460F46ECDA019BB2
:108F5000E3E802670193029B0AF1010A9A45ABF12B
:108F6000080BD3D1A29BDDF81490032B39D8DFE88E
:108F700013F0D900060006004D0048AB0393B9F189
:108F8000000F4FF000004FF0000109DB039D05EBDF
:108F9000C904083474E9022300F03AFBA542F9D170
:108FA000079B002B40F01E810B9BC3E900010B4681
:108FB00003990246D1E9000100F028FBB9F1000F46
:108FC0000CDD4AAD01240134F5E8022300F020FB5A
:108FD000A145F8DA079B002B40F014810B9BC3E9F5
:108FE0000201069B03F007000DF5197DBDE8F08F27
:108FF00000000040FB21F93F0000E03F0000F03F8F
:109000000000703EB8CD000048AB0393B9F1000FEB
:1090100040F32781039ACDF810904FEAC9030193DA
:10902000D318D3E900AB09F10053013B02EBC908A7
:109030000293914678E9026752465B4630463946CC
:1090400000F0E6FA04460D4602460B463046394625
:1090500000F0DCFA52465B4600F0DAFAC145A2465F
:10906000AB46C8E90201C8E90045E3D1DDF810903C
:10907000B9F1010F40F3F580019B039A0299134463
:10908000C900D3E9006701F1080A019192440DF586
:10909000947B7AE9028932463B464046494600F0D5
:1090A000B7FA04460D4602460B464046494600F0D4
:1090B000ADFA32463B4600F0ABFAD34526462F4682
:1090C000CAE90201CAE90045E3D1019C039B1034BF
:1090D000002000211C4403F1100574E9022300F074
:1090E00097FAA542F9D1039C079ED4E90023D4E95D
:1090F0000245002E00F08A8003F1004701F1004391
:109100000B99C1E90403069B2646944605F10044E9
:1091100003F00700C1E900C7C1E902640DF5197D3C
:10912000BDE8F08F089C039D0834002000212C44EA
:1091300074E9022300F06CFAA542F9D1079B13B140
:1091400001F1004319460B9BC3E90001069B03F0A4
:1091500007000DF5197DBDE8F08FBBF1000F08F198
:10916000010874DD022581E500260027EFE60024D2
:109170008EE5CDE90685059D304639466A4200F008
:10918000BBF90022384B06460F4600F07DFE00B3C7
:109190000022364B3046394600F0F0FB00F09EFED0
:1091A000044600F081FB00222F4B00F0E7FB0B464A
:1091B00002463946304600F029FA00F08FFE0BF1E6
:1091C00001090CAB183543F82B00059543F82940ED
:1091D0005FE63046394600F081FE0CABD94643F8D5
:1091E0002B0056E60B9C01F10043C4E900030B463B
:1091F00003990246D1E9000100F008FAB9F1000F25
:109200003FF7DFAE01F100431946E7E60B9EC6E9E2
:109210000023069BC6E9040103F00700C6E90245E6
:109220000DF5197DBDE8F08FA29B032B3FF6D9AE5B
:1092300001A252F823F000BF499200007B8F00008A
:109240007B8F0000099000000020002176E7324665
:109250003B460020064900F0D9F9022506460F4694
:109260002BE5002000213EE7000070410000703E29
:109270000000F03F000000002DE9F04F21F0004613
:10928000B6F1795F85B004460D469046994604DAFA
:1092900000F024FE002800F0858022462B46204660
:1092A000294600F06BFB06460F4602460B46204659
:1092B000294600F063FB41A3D3E9002382468B4695
:1092C0003046394600F05AFB3EA3D3E9002300F0B4
:1092D0009DF932463B4600F051FB3CA3D3E9002305
:1092E00000F096F932463B4600F048FB39A3D3E93B
:1092F000002300F08BF932463B4600F03FFB37A3DA
:10930000D3E9002300F084F90E9BCDE900019BB363
:109310000022294B4046494600F030FBDDE900239E
:10932000CDE902015046594600F028FB02460B46A3
:10933000DDE9020100F06AF932463B4600F01EFB0F
:1093400042464B4600F062F919A3D3E900230646D2
:109350000F465046594600F011FB02460B46304678
:10936000394600F055F902460B462046294600F0E2
:109370004DF905B0BDE8F08F02460B463046394640
:1093800000F0FCFA0AA3D3E9002300F03FF95246AB
:109390005B4600F0F3FA22462B4600F039F905B09F
:1093A000BDE8F08F2046294605B0BDE8F08F00BF2C
:1093B000495555555555C53F0000E03F7CD5CF5A1E
:1093C0003AD9E53DEB9C2B8AE6E55A3E7DFEB15746
:1093D000E31DC73ED561C119A0012A3FA6F81011AF
:1093E0001111813F21F00043194670470000000031
:1093F0002DE9F041C1F30A57A7F2FF35132D0246BC
:109400000B460C46884606461DDC002D3CDB364FDD
:109410002F4101EA070C5CEA000C19D030A3D3E914
:10942000002300F0F5F80022002300F037FDC8B358
:10943000002C04DA4FF4801343FA05F5A84428EA17
:10944000070400262EE0332D06DDB5F5806F2DD004
:1094500010461946BDE8F081A7F213474FF0FF3CD4
:109460002CFA07F70742F3D01DA3D3E9002300F03D
:10947000CFF80022002300F011FD98B1002C21DB71
:1094800026EA070644460DE015A3D3E9002300F0C1
:10949000BFF80022002300F001FD18B1002C08DB0A
:1094A0000026344621463046BDE8F08100F0B0F891
:1094B000D0E724F000430D4A1E43002E18BF144687
:1094C0000026EFE7142D08D00123C5F1340503FA77
:1094D00005F5AE1928BF9844D2E704F10108CFE79B
:1094E0009C7500883CE4377EFFFF0F000000F0BF52
:1094F0000020704700000000F8B5C1F30A5304468D
:109500000D460E4617460BBB21F00046034633437B
:109510001BD0354B002200F031FA344B9F420446F9
:109520000D4635DBC1F30A530E46363B3B4440F251
:10953000FE72934232DC002B11DD26F0FF4626F44A
:10954000E00646EA035520462946F8BD40F2FF7280
:109550009342EBD102460B4600F05AF8F8BD13F1E6
:10956000350F28DA4CF250339F4222462B460ADD53
:1095700019A1D1E9000100F03DF817A3D3E90023B8
:1095800000F0FCF9F8BD16A1D1E9000100F032F8B5
:1095900013A3D3E9002300F0F1F9F8BD22462B46CE
:1095A0000DA1D1E9000100F025F80BA3D3E90023B8
:1095B00000F0E4F9F8BD26F0FF4626F4E006363365
:1095C00046EA0355204629460022094B00F0D6F909
:1095D000F8BD00BFAFF300809C7500883CE4377E87
:1095E00059F3F8C21F6EA50100005043B03CFFFFC5
:1095F0000000903C03F0004321F0004242EA0301E6
:10960000704700BF81F0004102E000BF83F00043DB
:1096100030B54FEA41044FEA430594EA050F08BF0D
:1096200090EA020F1FBF54EA000C55EA020C7FEAD1
:10963000645C7FEA655C00F0E2804FEA5454D4EB4E
:109640005555B8BF6D420CDD2C4480EA020281EA18
:10965000030382EA000083EA010180EA020281EA50
:109660000303362D88BF30BD11F0004F4FEA0131A2
:109670004FF4801C4CEA113102D0404261EB4101B1
:1096800013F0004F4FEA03334CEA133302D0524237
:1096900063EB430394EA050F00F0A780A4F10104F3
:1096A000D5F1200E0DDB02FA0EFC22FA05F280182D
:1096B00041F1000103FA0EF2801843FA05F3594113
:1096C0000EE0A5F120050EF1200E012A03FA0EFC92
:1096D00028BF4CF0020C43FA05F3C01851EBE371BC
:1096E00001F0004507D54FF0000EDCF1000C7EEBD9
:1096F00000006EEB0101B1F5801F1BD3B1F5001F17
:109700000CD349085FEA30004FEA3C0C04F1010435
:109710004FEA445212F5800F80F09A80BCF1004F5E
:1097200008BF5FEA500C50F1000041EB045141EAE0
:10973000050130BD5FEA4C0C404141EB010111F4E1
:10974000801FA4F10104E9D191F0000F04BF01468C
:109750000020B1FA81F308BF2033A3F10B03B3F16A
:1097600020020CDA0C3208DD02F1140CC2F10C02FA
:1097700001FA0CF021FA02F10CE002F11402D8BF58
:10978000C2F1200C01FA02F120FA0CFCDCBF41EA24
:109790000C019040E41AA2BF01EB0451294330BDF3
:1097A0006FEA04041F3C1CDA0C340EDC04F11404D0
:1097B000C4F1200220FA04F001FA02F340EA0300A7
:1097C00021FA04F345EA030130BDC4F10C04C4F1ED
:1097D000200220FA02F001FA04F340EA03002946CD
:1097E00030BD21FA04F0294630BD94F0000F83F417
:1097F000801306BF81F480110134013D4EE77FEAFA
:10980000645C18BF7FEA655C29D094EA050F08BF45
:1098100090EA020F05D054EA000C04BF1946104626
:1098200030BD91EA030F1EBF0021002030BD5FEA6A
:10983000545C05D14000494128BF41F0004130BD92
:1098400014F580043CBF01F5801130BD01F00045E6
:1098500045F0FE4141F470014FF0000030BD7FEA59
:10986000645C1ABF194610467FEA655C1CBF0B4654
:10987000024650EA013406BF52EA033591EA030F6B
:1098800041F4002130BD00BF90F0000F04BF002163
:10989000704730B54FF4806404F132044FF0000596
:1098A0004FF0000150E700BF90F0000F04BF00210F
:1098B000704730B54FF4806404F1320410F0004575
:1098C00048BF40424FF000013EE700BF42004FEA70
:1098D000E2014FEA31014FEA02701FBF12F07F43ED
:1098E00093F07F4F81F06051704732F07F4208BFA4
:1098F000704793F07F4F04BF41F40021704730B5AB
:109900004FF4607401F0004521F000411CE700BFF6
:1099100050EA010208BF704730B54FF000050AE079
:1099200050EA010208BF704730B511F0004502D57A
:10993000404261EB41014FF4806404F132045FEA7C
:10994000915C3FF4D8AE4FF003025FEADC0C18BF25
:1099500003325FEADC0C18BF033202EBDC02C2F117
:10996000200300FA03FC20FA02F001FA03FE40EAA9
:109970000E0021FA02F11444BDE600BF70B54FF0AD
:10998000FF0C4CF4E06C1CEA11541DBF1CEA13558B
:1099900094EA0C0F95EA0C0F00F0DEF82C4481EAF3
:1099A000030621EA4C5123EA4C5350EA013518BF13
:1099B00052EA033541F4801143F4801338D0A0FB00
:1099C00002CE4FF00005E1FB02E506F00042E0FBAD
:1099D00003E54FF00006E1FB03569CF0000F18BFB3
:1099E0004EF0010EA4F1FF04B6F5007F64F540745B
:1099F00004D25FEA4E0E6D4146EB060642EAC621EE
:109A000041EA55514FEAC52040EA5E504FEACE2E5A
:109A1000B4F1FD0C88BFBCF5E06F1ED8BEF1004F5D
:109A200008BF5FEA500E50F1000041EB045170BDD9
:109A300006F0004646EA010140EA020081EA03011D
:109A4000B4EB5C04C2BFD4EB0C0541EA045170BD19
:109A500041F480114FF0000E013C00F3AB8014F193
:109A6000360FDEBF002001F0004170BDC4F10004DC
:109A7000203C35DA0C341BDC04F11404C4F120055D
:109A800000FA05F320FA04F001FA05F240EA0200B8
:109A900001F0004221F0004110EBD37021FA04F6EE
:109AA00042EB06015EEA430E08BF20EAD37070BDA8
:109AB000C4F10C04C4F1200500FA04F320FA05F007
:109AC00001FA04F240EA020001F0004110EBD37009
:109AD00041F100015EEA430E08BF20EAD37070BD79
:109AE000C4F1200500FA05F24EEA020E20FA04F352
:109AF00001FA05F243EA020321FA04F001F0004101
:109B000021FA04F220EA020000EBD3705EEA430E71
:109B100008BF20EAD37070BD94F0000F0FD101F0A0
:109B20000046400041EB010111F4801F08BF013CD9
:109B3000F7D041EA060195F0000F18BF704703F017
:109B40000046520043EB030313F4801F08BF013D9E
:109B5000F7D043EA0603704794EA0C0F0CEA13555A
:109B600018BF95EA0C0F0CD050EA410618BF52EA14
:109B70004306D1D181EA030101F000414FF000001A
:109B800070BD50EA410606BF1046194652EA430628
:109B900019D094EA0C0F02D150EA013613D195EA9C
:109BA0000C0F05D152EA03361CBF104619460AD1E4
:109BB00081EA030101F0004141F0FE4141F47001EE
:109BC0004FF0000070BD41F0FE4141F4780170BDDE
:109BD00070B54FF0FF0C4CF4E06C1CEA11541DBF43
:109BE0001CEA135594EA0C0F95EA0C0F00F0A7F845
:109BF000A4EB050481EA030E52EA03354FEA013172
:109C000000F088804FEA03334FF0805545EA131384
:109C100043EA12634FEA022245EA111545EA10654C
:109C20004FEA00260EF000419D4208BF964244F1E3
:109C3000FD0404F5407402D25B084FEA3202B61A02
:109C400065EB03055B084FEA32024FF480104FF4D6
:109C5000002CB6EB020E75EB030E22BFB61A75464A
:109C600040EA0C005B084FEA3202B6EB020E75EBDD
:109C7000030E22BFB61A754640EA5C005B084FEA45
:109C80003202B6EB020E75EB030E22BFB61A754612
:109C900040EA9C005B084FEA3202B6EB020E75EB1D
:109CA000030E22BFB61A754640EADC0055EA060EDE
:109CB00018D04FEA051545EA16754FEA06164FEA21
:109CC000C30343EA52734FEAC2025FEA1C1CC0D1CD
:109CD00011F4801F0BD141EA00014FF000004FF05A
:109CE000004CB6E711F4801F04BF01430020B4F11B
:109CF000FD0C88BFBCF5E06F3FF6AFAEB5EB030CD3
:109D000004BFB6EB020C5FEA500C50F1000041EBCF
:109D1000045170BD0EF0004E4EEA113114EB5C049C
:109D2000C2BFD4EB0C0541EA045170BD41F480116F
:109D30004FF0000E013C90E645EA060E8DE60CEA77
:109D4000135594EA0C0F08BF95EA0C0F3FF43BAF94
:109D500094EA0C0F0AD150EA01347FF434AF95EA4B
:109D60000C0F7FF425AF104619462CE795EA0C0F2F
:109D700006D152EA03353FF4FDAE1046194622E7FC
:109D800050EA410618BF52EA43067FF4C5AE50EAD6
:109D900041047FF40DAF52EA43057FF4EBAE12E7C6
:109DA0004FF0FF3C06E000BF4FF0010C02E000BFA7
:109DB0004FF0010C4DF804CD4FEA410C7FEA6C5C8A
:109DC0004FEA430C18BF7FEA6C5C1BD001B050EA2D
:109DD000410C0CBF52EA430C91EA030F02BF90EA18
:109DE000020F0020704710F1000F91EA030F58BFD7
:109DF000994208BF90422CBFD8176FEAE37040F039
:109E0000010070474FEA410C7FEA6C5C02D150EAD6
:109E1000013C07D14FEA430C7FEA6C5CD6D152EA91
:109E2000033CD3D05DF8040B704700BF8446104656
:109E300062468C461946634600E000BF01B5FFF755
:109E4000B7FF002848BF10F1000F01BD4DF808ED25
:109E5000FFF7F4FF0CBF012000205DF808FB00BFF6
:109E60004DF808EDFFF7EAFF34BF012000205DF850
:109E700008FB00BF4DF808EDFFF7E0FF94BF01209D
:109E800000205DF808FB00BF4DF808EDFFF7CEFF9E
:109E900094BF012000205DF808FB00BF4DF808EDDD
:109EA000FFF7C4FF34BF012000205DF808FB00BFAE
:109EB0004FEA410C7FEA6C5C02D150EA013C0AD1C6
:109EC0004FEA430C7FEA6C5C02D152EA033C02D1B8
:109ED0004FF0000070474FF0010070474FEA410219
:109EE00012F5001215D211D56FF47873B3EB6252EC
:109EF00012D94FEAC12343F0004343EA505311F013
:109F0000004F23FA02F018BF404270474FF00000A4
:109F1000704750EA013005D111F0004008BF6FF0E2
:109F2000004070474FF00000704700BF1FB51C464F
:109F3000094B1B680546D86852B1084B0091CDE922
:109F4000013207492B46224600F028F800F0BAFDFE
:109F5000044B1A46F2E700BF5C00002000CE000070
:109F60000DCE0000B2BB0000014B1868704700BF67
:109F70005C00002008B5074B044613B10021AFF385
:109F80000080054B1868836A03B19847204601F0AA
:109F900071FB00BF000000003CCE00000EB403B512
:109FA000014603AB054853F8042B0068019300F009
:109FB00081F802B05DF804EB03B070475C0000204C
:109FC00070B50D4E0D4CA41BA4100025A54209D15F
:109FD0000B4E0C4C01F050FBA41BA4100025A54215
:109FE00005D170BD56F8253098470135EEE756F893
:109FF000253098470135F2E72C0200202C02002082
:10A000002C0200203C02002010B5431E0A4491425D
:10A0100000D110BD11F8014B03F8014FF7E788425A
:10A0200010B501EB020307D8421E99420AD011F87D
:10A03000014B02F8014FF8E78342F5D98118D21A93
:10A04000D34200D110BD13F8014D01F8014DF7E7DF
:10A0500002440346934200D1704703F8011BF9E71D
:10A060009368013B002B10B4936008DA9469A34213
:10A0700001DB0A2903D15DF8044B00F063BC1368CF
:10A08000581C1060197008465DF8044B7047F8B50D
:10A0900006460F461446D518AC4201D1002007E011
:10A0A0003A4614F8011B3046FFF7DAFF431CF3D1A0
:10A0B000F8BD00002DE9F04F9DB00C461746039304
:10A0C000064618B183690BB900F0F4FD7B4B9C4246
:10A0D00057D17468A38918075DD52369002B5AD01E
:10A0E0000023099320238DF8293030238DF82A305E
:10A0F0004FF0010BB846454615F8013B0BB1252B37
:10A1000054D1B8EB070A0BD053463A4621463046A5
:10A11000FFF7BDFF013000F0C280099B5344099353
:10A1200098F80030002B00F0BA8000234FF0FF3287
:10A13000CDE90523049307938DF853301A93A8466D
:10A14000052218F8011B5E4800F0C2FE049B78BB94
:10A15000D90644BF20228DF853201A0744BF2B2272
:10A160008DF853202A782A2A2AD0079AA846002058
:10A170000A25414611F8013B303B092B69D960B3F0
:10A1800024E0504B9C4201D1B468A3E74E4B9C4263
:10A1900008BFF4689EE72146304600F025FC002801
:10A1A0009ED04FF0FF301DB0BDE8F08FA846A2E76B
:10A1B000434A801A0BFA00F0184304904546BEE764
:10A1C000039A111D12680391002A01DB079204E033
:10A1D000524243F002030792049398F800302E2B6A
:10A1E0000ED198F801302A2B38D1039B1A1D1B6819
:10A1F0000392002BB8BF4FF0FF3308F1020805931C
:10A20000324D98F800100322284600F061FE40B15C
:10A210004023401B03FA00F0049B034308F10108AC
:10A22000049398F800102A488DF82810062208F1A7
:10A23000010700F04DFE002837D0264B1BBB039BC7
:10A24000073323F0070308330393099B4B44099317
:10A2500050E705FB0232012088468AE7002308F117
:10A260000108059319460A25404610F8012B303A9B
:10A27000092A03D9002BC3D00591C1E705FB0121B1
:10A2800001238046F0E703AB00932246124B04A95A
:10A290003046AFF30080B0F1FF3F8146D5D1A389AE
:10A2A0005B063FF57EAF09987DE703AB009322463E
:10A2B000094B04A9304600F087F8ECE794CE000083
:10A2C00040CE0000B4CE000074CE000046CE0000A8
:10A2D0004ACE0000000000008FA000002DE9F047EA
:10A2E00091461F468A680B69DDF820809342B8BF0B
:10A2F0001346C9F8003091F8432006460C4612B1C7
:10A300000133C9F800302368990642BFD9F80030FC
:10A310000233C9F80030256815F0060507D104F1AD
:10A32000190AE368D9F800209B1AAB4228DC94F89C
:10A3300043302268003318BF012392062DD404F164
:10A34000430239463046C047013020D02368E568D3
:10A35000D9F8002003F00603042B08BFAD1AA36848
:10A3600022690CBF25EAE57500259342C4BF9B1AFC
:10A37000ED184FF000091A344D451AD1002008E0BD
:10A380000123524639463046C047013003D14FF0D1
:10A39000FF30BDE8F0870135C3E7E1185A1C3020D3
:10A3A00081F84300224494F8451082F843100233A8
:10A3B000C5E70123224639463046C0470130E6D082
:10A3C00009F10109D8E700002DE9F04301F1430C40
:10A3D0000C46097E85B06E291746064698460C9AAB
:10A3E00000F0B38022D8632936D00AD8002900F0C3
:10A3F000B980582900F0838004F1420584F84210A6
:10A4000032E0642901D06929F6D120681368050675
:10A4100003F104012AD51B681160002B03DA2D22F9
:10A420005B4284F843206F480A2239E0732900F028
:10A430009D8008D86F2920D07029DDD1236843F092
:10A440002003236003E0752917D07829D4D178231D
:10A4500084F84530644855E01368191D1B68116085
:10A4600004F1420584F8423001238CE01B6811603E
:10A4700010F0400F18BF1BB2CFE713682568181DF6
:10A480001060280601D51B6802E06806FBD51B8812
:10A4900054486F2914BF0A220822002184F843106F
:10A4A0006568A560002DC0F29580216821F0040147
:10A4B0002160002B3DD1002D40F08E806546082A9A
:10A4C0000BD12368DB0708D5236962689A42DEBF97
:10A4D000302305F8013C05F1FF35ACEB05032361A2
:10A4E000CDF800803B4603AA21463046FFF7F6FE32
:10A4F00001304DD14FF0FF3005B0BDE8F083394851
:10A5000084F84510136821681D1D1B6815600A0634
:10A510000BD5CA0744BF41F0200121601BB9226856
:10A5200022F0200222601022B7E74D0648BF9BB2FE
:10A53000EFE76546B3FBF2F102FB1133C35C05F8AC
:10A54000013D0B460029F5D1B9E71368256861691B
:10A55000181D106028061B6801D5196002E06A0604
:10A56000FBD51980002323616546B9E71368191DDF
:10A5700011601D6862680021284600F0A9FC08B13E
:10A58000401B606063682361002384F84330A7E7C1
:10A5900023692A4639463046C0470130AAD023688D
:10A5A0009B0713D4E068039B9842B8BF1846A3E703
:10A5B00001234A4639463046C04701309AD001351A
:10A5C000E368039A9B1AAB42F2DCEBE7002504F147
:10A5D0001909F5E7002BACD1037884F8423004F177
:10A5E00042056CE751CE000062CE000038B50D4B3D
:10A5F0001C68A36B05467BB9182000F04DFC0A4A85
:10A600000A4BA063C0E90023094B83600B238381BD
:10A6100001220023C0E90423A36B00221D615A61BB
:10A6200038BD00BF5C0000200E33CDAB34126DE6A8
:10A63000ECDE050038B5134B1C68A36B7BB9182002
:10A6400000F02AFC104A114BA063C0E90023104B14
:10A6500083600B23838101220023C0E90423A16BC3
:10A660000C480A694B690C4C504304FB0300A2FBE5
:10A6700004230344541C43F10005C1E9044525F0BB
:10A68000004038BD5C0000200E33CDAB34126DE6C7
:10A69000ECDE05002DF451582D7F954C0CB430B5EF
:10A6A000174B0C1E9DB01D6808DA8B232B604FF0F2
:10A6B000FF301DB0BDE8304002B070474FF4027368
:10A6C000ADF8143014BF04F1FF332346049307930D
:10A6D0004FF6FF7302900690ADF81630209A21AB2A
:10A6E00002A92846019300F06BFD431CBCBF8B23DD
:10A6F0002B60002CDDD0029B00221A70D9E700BF2E
:10A700005C0000200EB400B59CB01DAB029006901A
:10A710006FF00041094807910491094953F8042B4F
:10A7200005910068019302A900F04AFD029B0022F6
:10A730001A701CB05DF804EB03B070475C00002099
:10A740000802FFFF10B503461A785C1C3AB9013BBA
:10A7500011F8012B03F8012F002AF9D110BD23466F
:10A76000F2E7C9B2034610F8012B1AB18A42F9D1B7
:10A7700018467047002918BF0023F9E710F8012B8D
:10A7800011F8013B012A28BF9A42F7D0D01A70472E
:10A79000034613F8012B002AFBD1181A0138704721
:10A7A00010B56AB10139841810F8013B11F8012F76
:10A7B000934203D1A04201D0002BF5D1981A10BDCD
:10A7C0001046FCE770B50139044602B970BD234656
:10A7D00011F8015F03F8015B561E2DB91444A34222
:10A7E000F4D003F8015BFAE71C463246EDE7F0B51A
:10A7F00003787BB1044623782046661C7BB14A1E51
:10A80000631E12F8015F4DB113F8017FAF42344669
:10A81000F7D0F0E70B78002B18BF0020F0BD1846EA
:10A82000FCE72DE9F0478046894692461E460F46D2
:10A830003D46089815F8014B00F0C6FA20444378CD
:10A8400013F0080332D12D2C32D17C78BD1C0122AB
:10A85000002E5DD0102E09D1302C07D12B7803F0BB
:10A86000DF03582B4FD16C7810260235002A14BF15
:10A870004FF000416FF000410027B1FBF6FC384675
:10A8800006FB1C1EA4F13003092B17D81C46A64258
:10A8900023DD7B1C07D084451CD301D1A64519DBE1
:10A8A00000FB0640012715F8014BEBE72F46BFE7F9
:10A8B0002B2C04BFBD1C7C781A46C9E7A4F14103C8
:10A8C000192B01D8373CE2E7A4F16103192B04D816
:10A8D000573CDCE74FF0FF37E5E77B1C08D122232C
:10A8E000C8F800300846BAF1000F07D1BDE8F0877C
:10A8F00002B14042BAF1000FF8D00FB105F1FF39B3
:10A90000CAF80090F2E73024002EAFD10826ADE758
:10A91000302CA3D00A26A9E7084B37B51C68084D90
:10A92000236A002B08BF2B46009313460A460146B4
:10A930002046FFF776FF03B030BD00BF5C0000206B
:10A94000C0000020F8B50E461446054618B18369CC
:10A950000BB900F0AFF9214B9C422AD16C68A36976
:10A96000A360A3891A072ED5236963B323692068DE
:10A97000C01A6369F6B28342374604DC2146284692
:10A9800000F02EF928BBA368013BA36023685A1C82
:10A9900022601E7063690130834204D0A389DB0703
:10A9A00019D50A2E17D12146284600F019F990B181
:10A9B0000FE00B4B9C4201D1AC68D0E7094B9C42A5
:10A9C00008BFEC68CBE72146284600F00DF80028C8
:10A9D000CCD04FF0FF373846F8BD00BF94CE000012
:10A9E000B4CE000074CE0000324B70B51D68064630
:10A9F0000C4625B1AB6913B9284600F05BF92E4B24
:10AA00009C420FD16C68B4F90C309AB215072CD463
:10AA1000D00611D40922326043F04003A3814FF0E5
:10AA2000FF303EE0254B9C4201D1AC68EBE7244B64
:10AA30009C4208BFEC68E6E7510712D5616B41B153
:10AA400004F14403994202D0304600F091FA002309
:10AA50006363A38923F02403A38100236360236934
:10AA60002360A38943F00803A38123694BB9A38919
:10AA700003F42073B3F5007F03D02146304600F085
:10AA8000CBF9A28912F001030CD00023A360636903
:10AA90005B42A361236953B9B4F90C3013F0800011
:10AAA000BAD170BD920758BF6369A360F2E7002076
:10AAB000F7E700BF5C00002094CE0000B4CE000099
:10AAC00074CE000008B5062000F0A8FC012000F0BC
:10AAD000D1FD00008A892DE9F041054610070C469A
:10AAE00058D44B68002B05DC0B6C002B02DC0020DB
:10AAF000BDE8F081E66A002EF9D0002312F48052FE
:10AB00002F68216A2B6032D0606DA3895A0705D562
:10AB10006368C01A636B0BB1236CC01A0023024632
:10AB2000E66A216A2846B047431CA38906D12968F2
:10AB30001D2948D8294ACA40D60744D50022626058
:10AB4000D9042269226004D5421C01D12B6803B9C3
:10AB50006065616B2F600029C9D004F144039942FC
:10AB600002D0284600F004FA00206063C0E7012309
:10AB70002846B047411CC8D12B68002BC5D01D2BDF
:10AB800001D0162B01D12F60B1E7A38943F0400318
:10AB9000A381ADE70F69002FA9D093070E6808BF06
:10ABA0004B690F6018BF0023A6EB07088B60B8F154
:10ABB000000F9CDD43463A46216AA66A2846B04704
:10ABC000002806DCA38943F04003A3814FF0FF3047
:10ABD0008EE70744A8EB0008E9E700BF010040202A
:10ABE00038B50B6905460C46DBB118B183690BB962
:10ABF00000F060F80C4B9C4209D16C68B4F90C3041
:10AC00007BB121462846BDE83840FFF763BF074BBC
:10AC10009C4201D1AC68F1E7054B9C4208BFEC684F
:10AC2000ECE7002038BD00BF94CE0000B4CE000099
:10AC300074CE0000002310B50446C0E900338360E1
:10AC400081814366C281C0E90433836119460822C9
:10AC50005C30FFF7FDF9054B6362054BA362054BC2
:10AC6000E362054B2462236310BD00BF55B40000AE
:10AC700077B40000AFB40000D3B40000014900F085
:10AC800085B800BFE1AB000070B54A1E682555438A
:10AC90000E4605F1740100F0B9F9044640B10021F7
:10ACA000C0E900160C30A06005F16802FFF7D0F98A
:10ACB000204670BD836910B5044633BBC0E912332A
:10ACC0000365124B124A1B688262984204BF01233B
:10ACD000836100F01FF86060204600F01BF8A06060
:10ACE000204600F017F80022E06004216068FFF7BA
:10ACF000A1FF01220921A068FFF79CFF0222122177
:10AD0000E068FFF797FF0123A36110BD3CCE000070
:10AD10007DAC0000F8B51B4B1E68B369074613B93C
:10AD20003046FFF7C7FF4836D6E90134013B03D56B
:10AD3000336833B13668F7E7B4F90C506DB1683455
:10AD4000F4E704213846FFF79FFF30600028F1D177
:10AD50000C233B6004462046F8BD0B4B6566C4E9F6
:10AD60000055A560C4E90335C4E905550822294604
:10AD700004F15C00FFF76CF9C4E90D55C4E9125504
:10AD8000E9E700BF3CCE00000100FFFF2DE9F843DA
:10AD90008046894600F14804002614B93046BDE8D3
:10ADA000F883D4E90175013F01D52468F5E7AB8943
:10ADB000012B07D9B5F90E30013303D0294640469F
:10ADC000C84706436835EEE7D0F8EC00704770B529
:10ADD0000E46B1F90E10002996B014461D4607DA4A
:10ADE00000232B60B3891A0610D44FF480630EE061
:10ADF0006A4600F0A1FB0028F2DB019A02F47042DF
:10AE0000A2F500535A425A412A60EEE7402300203F
:10AE1000236016B070BD00008B8973B59D07064690
:10AE20000C4607D504F147032360236101236361C6
:10AE300002B070BD01AB6A46FFF7C9FF0099054635
:10AE4000304600F0E3F848B9B4F90C309A05EFD475
:10AE500023F0030343F00203A381E3E70D4BB36246
:10AE6000A389206043F08003A381009B6361019B61
:10AE700020615BB1B4F90E10304600F06FFB28B1D1
:10AE8000A38923F0030343F00103A381A3891D4396
:10AE9000A581CDE77DAC0000024B0146186800F0AB
:10AEA000B5B800BF5C00002082B001B901A942B171
:10AEB0004BB113780B601278101C18BF012002B040
:10AEC00070471046FBE76FF00100F8E70000000054
:10AED00001F0FF01102A2BDB10F0070F08D010F84B
:10AEE000013B013A8B422DD010F0070F42B3F6D14F
:10AEF000F0B441EA012141EA014122F007047FF068
:10AF000000070023F0E80256083C85EA010586EABE
:10AF1000010685FA47F5A3FA87F586FA47F6A5FAFA
:10AF200087F68EB9EED1F0BC01F0FF0102F0070206
:10AF300032B110F8013B013A83EA010313B1F8D1B1
:10AF40000020704701387047002D06BF3546033892
:10AF5000073815F0010F07D1013015F4807F02BFCB
:10AF6000013015F4C03F0130F0BC0138704700BF1C
:10AF700038B50546002945D051F8043C0C1F002B7C
:10AF8000B8BFE41800F00CFB1F4A1368104633B931
:10AF9000636014602846BDE8384000F002BBA3425D
:10AFA0000CD921686218934204BF1A685B68636019
:10AFB00004BF521822600460ECE713465A680AB1D5
:10AFC000A242FAD919685818A0420BD1206801444E
:10AFD000581882421960DDD1106852685A600144E5
:10AFE0001960D7E702D90C232B60D3E7206821181A
:10AFF0008A4204BF11685268626004BF0918216068
:10B000005C60C7E738BD00BF6C7A012070B5CD1C0D
:10B0100025F0030508350C2D38BF0C25002D0646FC
:10B0200001DBA94203D90C233360002070BD00F07E
:10B03000B7FA214A1468214691B9204C23681BB9FC
:10B04000304600F0B3F920602946304600F0AEF9F2
:10B05000431C24D10C233360304600F0A2FAE4E70D
:10B060000B685B1B18D40B2B0FD90B60CD50CC1881
:10B07000304600F096FA04F10B00231D20F0070083
:10B08000C31AD3D05A42E250D0E78C424B6816BF65
:10B09000636013600C46EBE70C464968CCE7C41CC0
:10B0A00024F00304A04205D0211A304600F07EF9B6
:10B0B0000130CFD02560DBE76C7A0120707A012067
:10B0C000F8B5074614460E4621B91146BDE8F840CA
:10B0D000FFF79CBF22B9FFF74BFF25462846F8BD76
:10B0E00000F060FAA0420FD221463846FFF78EFFEB
:10B0F00005460028F2D031462246FEF785FF31464C
:10B100003846FFF735FFE9E73546E7E72DE9F04731
:10B110008E689E4282460C469046994637D88A8968
:10B1200012F4906F31D0256809696F1A656902239E
:10B1300005EB450595FBF3F509F101033B449D4201
:10B1400038BF1D46530530D52946FFF75FFF064639
:10B1500050B90C23CAF80030A38943F04003A381FF
:10B160004FF0FF30BDE8F0873A462169FEF74CFF0B
:10B17000A38923F4906343F08003A3812661656172
:10B180003E44ED1B2660A5604E464E4500D94E4616
:10B19000324641462068FEF742FFA3689B1BA3602E
:10B1A00023681E4426600020DCE72A46FFF788FF5C
:10B1B00006460028E2D121695046FFF7D9FEC8E7CC
:10B1C0002DE9F04F9DB0804603938B891D060C46F8
:10B1D00016460FD50B696BB94021FFF717FF2060AA
:10B1E000206128B90C23C8F800304FF0FF30C7E0C9
:10B1F000402363610023099320238DF829303023F5
:10B200008DF82A304FF0010B37463D4615F8013BCB
:10B210000BB1252B3ED1B7EB060A0BD05346324675
:10B2200021464046FFF772FF013000F0A480099BE1
:10B23000534409933B78002B00F09D8000234FF08E
:10B24000FF32CDE90523049307938DF853301A9309
:10B250002F46052217F8011B4F48FFF739FE049BC4
:10B26000D0B9D90644BF20228DF853201A0744BF15
:10B270002B228DF853202A782A2A15D0079A2F4698
:10B2800000200A25394611F8013B303B092B4DD9E6
:10B29000B8B10FE02F46B8E73F4A801A0BFA00F02A
:10B2A000184304903D46D3E7039A111D1268039199
:10B2B000002A01DB079204E0524243F002030792A6
:10B2C00004933B782E2B0CD17B782A2B33D1039B14
:10B2D0001A1D1B680392002BB8BF4FF0FF330237D3
:10B2E00005932E4D397803222846FFF7F1FD38B13A
:10B2F0004023401B03FA00F0049B034301370493EF
:10B30000397827488DF8281006227E1CFFF7E0FDCB
:10B31000002838D0234B13BB039B073323F00703CC
:10B3200008330393099B4B4409936DE705FB0232F5
:10B3300001200F46A6E700230137059319460A2589
:10B34000384610F8012B303A092A03D9002BC8D00F
:10B350000591C6E705FB012101230746F0E703AB92
:10B3600000932246104B04A94046AFF30080B0F191
:10B37000FF3F8146D6D1A3895B063FF536AF0998DA
:10B380001DB0BDE8F08F03AB00932246064B04A925
:10B390004046FFF719F8EAE740CE000046CE00002D
:10B3A0004ACE0000000000000DB1000038B5064C88
:10B3B000002305460846236000F046F9431C02D1ED
:10B3C000236803B12B6038BD008E01201F2938B5DA
:10B3D00004460D4604D9162303604FF0FF3038BDF4
:10B3E000426C12B152F821304BB9204600F030F8CF
:10B3F0002A4601462046BDE8384000F017B8012B28
:10B400000AD0591C03D1162303600120E7E700246A
:10B4100042F82540284698470020E0E7024B0146C5
:10B420001868FFF7D3BF00BF5C00002038B5074C99
:10B430000023054608461146236000F0EDF8431C42
:10B4400002D1236803B12B6038BD00BF008E0120FC
:10B4500000F0D2B810B50C46B1F90E1000F0AAF801
:10B460000028ABBF636DA3891B1823F48053ACBFC6
:10B470006365A38110BD2DE9F0411F468B89DB0573
:10B4800005460C46164605D502230022B1F90E10DA
:10B4900000F074F8A389B4F90E1023F48053A3814B
:10B4A00032463B462846BDE8F04100F023B810B5CF
:10B4B0000C46B1F90E1000F061F8431CA38915BFCA
:10B4C000606523F4805343F48053A38118BFA381A4
:10B4D00010BDB1F90E1000F01FB849B1FF2A85BFA9
:10B4E0008A2303600A704FF0FF3098BF0120704735
:10B4F0000846704738B5074C0546084611460022F5
:10B5000022601A4600F0AEF8431C02D1236803B152
:10B510002B6038BD008E012038B5064C002305464F
:10B520000846236000F058F8431C02D1236803B199
:10B530002B6038BD008E012038B5074C002305462E
:10B5400008461146236000F04FF8431C02D12368DF
:10B5500003B12B6038BD00BF008E012038B5064C0A
:10B56000002305460846236000F04EF8431C02D134
:10B57000236803B12B6038BD008E012038B5074C1D
:10B58000054608461146002222601A4600F04CF893
:10B59000431C02D1236803B12B6038BD008E01200B
:10B5A0007047704751F8043C181F002BBCBF0B5864
:10B5B000C018704738B5074C0546084611460022AA
:10B5C00022601A4600F038F8431C02D1236803B108
:10B5D0002B6038BD008E0120024B58221A604FF0BC
:10B5E000FF307047008E0120024B58221A604FF046
:10B5F000FF307047008E0120024B58221A604FF036
:10B60000FF307047008E0120024B58221A60002044
:10B61000704700BF008E0120024B58221A604FF085
:10B62000FF307047008E0120024B58221A604FF005
:10B63000FF307047008E0120024B58221A604FF0F5
:10B64000FF307047008E0120044A05491368002B23
:10B6500008BF0B461844106018467047747A0120E2
:10B66000088E0120024B58221A604FF0FF307047BD
:10B67000008E0120FEE700BFF8B500BFF8BC08BC93
:10B680009E467047F8B500BFF8BC08BC9E467047A0
:10B69000646174610000000014B700001D03000025
:10B6A0001DB700000D04000025B70000E9090000E7
:10B6B0002CB70000F90A000031B700004306000073
:10B6C0003CB700007704000041B70000350D0000D2
:10B6D0004DB700004F03000057B7000001090000FC
:10B6E00065B70000CF07000072B700000B0600002E
:10B6F00072616E646F6D00616C6C006C61737400DC
:10B7000066616C7365007472756500252E31357342
:10B710002E2E2E006D616B654C697374006164643C
:10B720004C6173740064656C657465006A6F696E62
:10B7300000636F707946726F6D546F0066696E6456
:10B74000006A6F696E537472696E677300756E6913
:10B75000636F6465417400756E69636F64655374EB
:10B7600072696E67006E65774279746541727261C5
:10B770007900667265654D656D6F72790000000035
:10B78000E5B70000AD110000EAB70000C7110000E6
:10B7900025B70000CB110000F0B70000B111000088
:10B7A000FAB70000CF11000003B80000D311000069
:10B7B0000DB80000D711000018B80000DB11000020
:10B7C00024B80000B51100002DB80000BF11000022
:10B7D00037B80000B911000042B80000C3110000E2
:10B7E00066696C65006F70656E00636C6F736500F1
:10B7F000656E644F6646696C6500726561644C698C
:10B800006E65007265616442797465730061707081
:10B81000656E644C696E6500617070656E64427936
:10B820007465730066696C6553697A650073746149
:10B8300072744C697374006E657874496E4C6973E8
:10B84000740073797374656D496E666F0000000053
:10B8500090150000A0150000B41500002816000087
:10B860005A1600008A160000BC160000DE16000002
:10B870001A17000054170000A4170000E217000078
:10B880004218000080180000A0180000D418000022
:10B890001419000036190000601900008A19000010
:10B8A000382F0000361A0000FE1A0000701B00003E
:10B8B000BA1B00001C1C0000381C0000561C0000B5
:10B8C000941D0000D41D0000461E0000741E0000E0
:10B8D000A41E0000D21E0000361F00009A1F0000A8
:10B8E000FE1F000062200000D62000005021000052
:10B8F000B2210000142200004A2200008E22000023
:10B90000D42200001A2300006C230000C223000090
:10B910000024000074240000A8240000EE2400008D
:10B92000342500007A250000B4250000FA25000027
:10B93000402600009C27000060190000D418000079
:10B94000B426000090150000E82600000E27000035
:10B9500042270000682700009015000090150000A5
:10B960009015000090150000122800004E280000DD
:10B970008E280000DE280000042900007229000043
:10B98000BC290000EC290000901500009015000073
:10B990000A2A00003C2A00006E2A0000A22A0000A9
:10B9A000C62A0000242B0000482B00006A2B000050
:10B9B0008C2B0000BE2B0000F02B0000142C00008C
:10B9C000382C00006A2C00008E2C0000901500001E
:10B9D00090150000901500009015000090150000D3
:10B9E000C02C0000E62C00000C2D0000322D0000C1
:10B9F000582D00008C2D0000C02D0000F42D0000FB
:10BA0000282E00004E2E0000742E0000A82E0000EC
:10BA10009015000090150000901500009015000092
:10BA20009015000090150000901500009015000082
:10BA30009015000090150000901500009015000072
:10BA4000CE2E0000CE2E0000AC2F0000DC2F000018
:10BA50005B2564206974656D206C6973745D0028D2
:10BA600025642062797465732900286F626A6563B2
:10BA70007420747970653A202564290053746163D9
:10BA80006B20756E646572666C6F7700626F6F6CA9
:10BA900065616E006E756D62657200737472696EB9
:10BAA00067006C69737400627974652061727261F9
:10BAB0007900000007000000030000001DBB00002B
:10BAC000F530000025BB0000A13100002EBB0000B6
:10BAD000EF32000037BB0000F930000040BB00002F
:10BAE000F332000048BB0000E132000051BB00000F
:10BAF0002D320000000000000100000002000000E4
:10BB000003000000040000000A0000001D00000007
:10BB10006D6963726F3A626974207632006861738E
:10BB2000546F6E6500706C6179546F6E650068616A
:10BB300073536572766F00736574536572766F0028
:10BB4000646163496E697400646163577269746506
:10BB500000737175617265576176650047432074A3
:10BB60006F6F6B2025642075736563733B2066726D
:10BB7000656520256420776F726473003C496E749C
:10BB8000656765723E003C4C6973743E003C4F62D1
:10BB90006A6563743E003C427974654172726179F2
:10BBA0003E000D0A564D2050616E69633A202573A0
:10BBB0000D0A006D69736300EDBB00009940000041
:10BBC000F6BB00001D400000FABB0000693F00000A
:10BBD00002BC00000B3F00000CBC00009D3E0000BA
:10BBE00018BC00009F3D00006E756C6C00686578A5
:10BBF000546F496E740073696E006A736F6E4765A7
:10BC000074006A736F6E436F756E74006A736F6E43
:10BC100056616C75654174006A736F6E4B6579414E
:10BC200074000000B0BC0000F9400000B8BC000087
:10BC3000FD400000C2BC00000F410000CBBC000072
:10BC400015410000D6BC00001B410000E2BC000012
:10BC500021410000F0BC000027410000F8BC0000BA
:10BC60002D410000FEBC00003341000013BD000068
:10BC70003941000028BD00003F41000034BD0000F4
:10BC80004541000044BD00004B41000050BD000094
:10BC9000514100005DBD0000574100006CBD000037
:10BCA000034100007FBD0000094100006E65740083
:10BCB00068617357694669007374617274576946A5
:10BCC000690073746F7057694669007769666953D4
:10BCD0007461747573006D79495041646472657361
:10BCE00073007374617274535349447363616E00DB
:10BCF00067657453534944006D794D41430068743E
:10BD000074705365727665724765745265717565B6
:10BD1000737400726573706F6E64546F48747470DE
:10BD2000526571756573740068747470436F6E6EDC
:10BD300065637400687474704973436F6E6E6563F5
:10BD4000746564006874747052657175657374000D
:10BD500068747470526573706F6E73650077656296
:10BD6000536F636B657453746172740077656253CB
:10BD70006F636B65744C6173744576656E740077A0
:10BD80006562536F636B657453656E64546F436C87
:10BD900069656E74000000000400000003000000EC
:10BDA0000A0000000700000006000000000000007C
:10BDB0000008080800080A4A4000000A5FEA5FEA33
:10BDC0000ED92ED36E19324489330C924C924D0801
:10BDD0000800000004880808040804848488000A15
:10BDE000448A4000048EC480000000048800000ED5
:10BDF000C000000000080001224488100C9252523A
:10BE00004C048C84848E1C824C901E1EC244924C26
:10BE100006CA525FE21FF01EC13E02448ED12E1FA1
:10BE2000E24488100ED12ED12E0ED12EC4880008E7
:10BE300000080000048004880244880482000EC0C8
:10BE40000EC008048244880ED126C0040ED135B33A
:10BE50006C0C925ED2521C925C925C0ED010100E52
:10BE60001C9252525C1ED01C901E1ED01C90100EB4
:10BE7000D013712E12525ED2521C8808081C1FE289
:10BE800042524C1254981492101010101E113B750F
:10BE9000B131113935B3710C9252524C1C925C90F5
:10BEA000100C92524C861C925C92510ED00C825C0B
:10BEB0001FE4848484125252524C1131312A4411AD
:10BEC0003135BB7112524C9252112A4484841EC4E3
:10BED00088101E0EC808080E10080482410EC242C7
:10BEE000424E048A400000000000001F0804800049
:10BEF00000000ED2524F10101C925C000ED0100E9B
:10BF000002424ED24E0C925C900E06C81C88080E5F
:10BF1000D24EC24C10101C92520800080808024071
:10BF200002424C10149814920808080806001B7569
:10BF3000B131001C925252000C92524C001C925C87
:10BF400090000ED24EC2000ED010100006C8049809
:10BF500008080EC807001252524F0011312A44003F
:10BF6000113135BB00124C8C9200112A4498001EEE
:10BF7000C4881E06C48C8486080808080818080CA3
:10BF8000881800000C836000000000000100000021
:10BF90000200000003000000040000000500000093
:10BFA0000600000007000000080000000900000073
:10BFB0000A0000000B0000000C0000000D00000053
:10BFC0000E0000000F000000100000001200000032
:10BFD0001400000016000000180000001A00000005
:10BFE0001C0000001E0000002000000023000000D4
:10BFF00026000000290000002C0000002F00000097
:10C0000032000000360000003A0000003E00000050
:10C0100042000000460000004B00000050000000FD
:10C02000550000005A000000610000006800000098
:10C030006F000000760000007D000000840000001A
:10C040008B0000009200000099000000A00000009A
:10C05000A7000000AE000000B5000000BC0000001A
:10C06000C3000000CA000000D1000000D80000009A
:10C07000DF000000E6000000ED000000F40000001A
:10C08000FB000000FF0000000000000002000000B4
:10C0900004000000010000000300000000C10000D7
:10C0A000714100000BC10000E145000015C1000016
:10C0B0002D42000022C100004D44000029C10000B3
:10C0C0009944000032C10000E94400003EC1000074
:10C0D000DD4300004FC10000814200005CC1000050
:10C0E0006543000015000000160000001700000066
:10C0F0001800000019000000646973706C61790019
:10C100006C696768744C6576656C006D6244697330
:10C11000706C6179006D62446973706C61794F660F
:10C1200066006D62506C6F74006D62556E706C6F5E
:10C1300074006D62447261775368617065006D626E
:10C140005368617065466F724C6574746572006EF9
:10C15000656F506978656C53656E64006E656F50ED
:10C160006978656C53657450696E004E6F74206514
:10C170006E6F75676820726F6F6D206576656E20D3
:10C18000616674657220636F6D70616374696F6E50
:10C1900000436F6D70616374656420466C61736801
:10C1A00020636F64652073746F72650A2564206272
:10C1B00079746573207573656420282564252529A5
:10C1C000206F6620256400426164207265636F728F
:10C1D0006420666F756E6420647572696E6720698D
:10C1E0006E697469616C697A6174696F6E00256447
:10C1F0002025642025642028256420776F726473CD
:10C2000029002564207265636F7264732C20256495
:10C2100020776F7264732C206D6178494420256407
:10C220002C20636F6D70616374696F6E2063796336
:10C230006C657320256400526573746F72656420A9
:10C24000256420736372697074730053746172742F
:10C25000656400726164696F00000000ECC2000058
:10C26000CD4E0000F9C200004151000009C300009A
:10C27000D550000017C30000A152000022C30000E7
:10C28000F54E000032C30000854F000046C3000099
:10C29000694F000055C300007D54000061C30000D9
:10C2A000F95300006AC300009D53000075C30000ED
:10C2B000ED52000080C300002553000089C3000038
:10C2C0005553000092C30000054F0000A1C30000B9
:10C2D000E54E0000AAC30000154F00006E6F6E65AA
:10C2E000006F7468657200706169720064697361DF
:10C2F000626C65526164696F006D65737361676537
:10C300005265636569766564007061636B6574523C
:10C31000656365697665007061636B657453656E0E
:10C3200064007265636569766564496E7465676506
:10C33000720072656365697665644D6573736167E4
:10C3400065547970650072656365697665645374D8
:10C3500072696E670073656E64496E7465676572B5
:10C360000073656E64506169720073656E64537426
:10C3700072696E67007365744368616E6E656C0008
:10C3800073657447726F757000736574506F77656D
:10C3900072007369676E616C537472656E6774685E
:10C3A000006465766963654944006C6173744D652A
:10C3B0007373616765494400556E6B6E6F776E20CD
:10C3C0007072696D6974697665205B25733A2573AF
:10C3D0005D00000000000000963007772C610EEE33
:10C3E000BA51099919C46D078FF46A7035A563E9CC
:10C3F000A395649E3288DB0EA4B8DC791EE9D5E0F3
:10C4000088D9D2972B4CB609BD7CB17E072DB8E7F1
:10C41000911DBF906410B71DF220B06A4871B9F346
:10C42000DE41BE847DD4DA1AEBE4DD6D51B5D4F47F
:10C43000C785D38356986C13C0A86B647AF962FDE4
:10C44000ECC9658A4F5C0114D96C0663633D0FFA31
:10C45000F50D088DC8206E3B5E10694CE44160D537
:10C46000727167A2D1E4033C47D4044BFD850DD221
:10C470006BB50AA5FAA8B5356C98B242D6C9BBDB34
:10C4800040F9BCACE36CD832755CDF45CF0DD6DC2F
:10C49000593DD1ABAC30D9263A00DE518051D7C8D6
:10C4A0001661D0BFB5F4B42123C4B3569995BACF61
:10C4B0000FA5BDB89EB802280888055FB2D90CC682
:10C4C00024E90BB1877C6F2F114C6858AB1D61C1FB
:10C4D0003D2D66B69041DC760671DB01BC20D2981A
:10C4E0002A10D5EF8985B1711FB5B606A5E4BF9FA7
:10C4F00033D4B8E8A2C9077834F9000F8EA809969A
:10C5000018980EE1BB0D6A7F2D3D6D08976C649104
:10C51000015C63E6F4516B6B62616C1CD83065851D
:10C520004E0062F2ED95066C7BA5011BC1F40882FA
:10C5300057C40FF5C6D9B06550E9B712EAB8BE8B3B
:10C540007C88B9FCDF1DDD62492DDA15F37CD38CC4
:10C55000654CD4FB5861B24DCE51B53A7400BCA3C2
:10C56000E230BBD441A5DF4AD795D83D6DC4D1A4F4
:10C57000FBF4D6D36AE96943FCD96E34468867ADCB
:10C58000D0B860DA732D0444E51D03335F4C0AAA6A
:10C59000C97C0DDD3C710550AA41022710100BBE6D
:10C5A00086200CC925B56857B3856F2009D466B9B4
:10C5B0009FE461CE0EF9DE5E98C9D9292298D0B0E9
:10C5C000B4A8D7C7173DB359810DB42E3B5CBDB796
:10C5D000AD6CBAC02083B8EDB6B3BF9A0CE2B60317
:10C5E0009AD2B1743947D5EAAF77D29D1526DB04CC
:10C5F0008316DC73120B63E3843B64943E6A6D0D17
:10C60000A85A6A7A0BCF0EE49DFF099327AE000A61
:10C61000B19E077D44930FF0D2A3088768F2011EF4
:10C62000FEC206695D5762F7CB67658071366C198B
:10C63000E7066B6E761BD4FEE02BD3895A7ADA10AC
:10C64000CC4ADD676FDFB9F9F9EFBE8E43BEB7178D
:10C65000D58EB060E8A3D6D67E93D1A1C4C2D83817
:10C6600052F2DF4FF167BBD16757BCA6DD06B53F7D
:10C670004B36B248DA2B0DD84C1B0AAFF64A0336BC
:10C68000607A0441C3EF60DF55DF67A8EF8E6E313B
:10C6900079BE69468CB361CB1A8366BCA0D26F2584
:10C6A00036E2685295770CCC03470BBBB9160222D1
:10C6B0002F260555BE3BBAC5280BBDB2925AB42BE6
:10C6C000046AB35CA7FFD7C231CFD0B58B9ED92CFB
:10C6D0001DAEDE5BB0C2649B26F263EC9CA36A7560
:10C6E0000A936D02A906099C3F360EEB8567077217
:10C6F00013570005824ABF95147AB8E2AE2BB17B7E
:10C70000381BB60C9B8ED2920DBED5E5B7EFDC7C04
:10C7100021DFDB0BD4D2D38642E2D4F1F8B3DD685B
:10C720006E83DA1FCD16BE815B26B9F6E177B06F56
:10C730007747B718E65A0888706A0FFFCA3B066643
:10C740005C0B0111FF9E658F69AE62F8D3FF6B61D0
:10C7500045CF6C1678E20AA0EED20DD75483044E72
:10C76000C2B30339612667A7F71660D04D47694900
:10C77000DB776E3E4A6AD1AEDC5AD6D9660BDF4013
:10C78000F03BD83753AEBCA9C59EBBDE7FCFB247C6
:10C79000E9FFB5301CF2BDBD8AC2BACA3093B353AB
:10C7A000A6A3B4240536D0BA9306D7CD2957DE54B4
:10C7B000BF67D9232E7A66B3B84A61C4021B685D8D
:10C7C000942B6F2A37BE0BB4A18E0CC31BDF055A06
:10C7D0008DEF022D416C6C207461736B7320737448
:10C7E0006F70706564007631313300202573202529
:10C7F00073004D656D6F727920636C65617265645D
:10C80000004E6F2066726565207461736B20656EE3
:10C81000747269657300000088C80000696B0000CD
:10C8200095C8000089640000A1C80000396B0000B1
:10C83000A7C80000496B0000ADC80000596B00009C
:10C84000B3C80000E9680000C9C80000B96400006E
:10C85000D3C80000B16B0000DBC800000569000010
:10C86000E4C80000A9660000F0C80000B965000037
:10C87000F9C800000166000001C900001968000045
:10C8800073656E736F727300616363656C6572616B
:10C8900074696F6E0074656D706572617475726530
:10C8A0000074696C74580074696C74590074696C14
:10C8B000745A00736574416363656C65726F6D656E
:10C8C00074657252616E676500746F756368526556
:10C8D0006164006932635265616400693263577252
:10C8E0006974650073706945786368616E67650097
:10C8F000737069536574757000726561644448545F
:10C90000006D6963726F70686F6E650088C90000A2
:10C91000316C000096C90000416C0000A3C9000002
:10C92000356C0000ACC90000456C0000B6C90000C1
:10C93000496C0000BFC900004D6C0000C4C9000074
:10C94000516C0000C9C90000556C0000D5C9000039
:10C95000596C0000DCC900005D6C0000E5C90000F6
:10C96000616C0000EAC90000656C0000F5C90000B8
:10C97000696C0000FFC90000396C000009CA0000A2
:10C980003D6C000074667400656E61626C6544699C
:10C9900073706C6179007365744261636B6C696775
:10C9A00068740067657457696474680067657448E3
:10C9B000656967687400736574506978656C006CAC
:10C9C000696E65007265637400726F756E6465648C
:10C9D0005265637400636972636C650074726961A7
:10C9E0006E676C65007465787400746674546F7556
:10C9F0006368656400746674546F75636858007486
:10CA00006674546F7563685900746674546F756307
:10CA10006850726573737572650076617273000099
:10CA200040CA0000D17000004ACA0000B170000086
:10CA300053CA00008D7000005FCA00001D70000026
:10CA4000766172457869737473007661724E616DB8
:10CA50006564007365745661724E616D656400763D
:10CA600061724E616D65466F72496E6465780057FC
:10CA7000656C636F6D6520746F204D6963726F42E2
:10CA80006C6F636B732100705F73706920213D20B0
:10CA90004E554C4C002F686F6D652F6769742F2EB3
:10CAA000706C6174666F726D696F2F7061636B611A
:10CAB0006765732F6672616D65776F726B2D61723A
:10CAC0006475696E6F6E6F726469636E7266352F1E
:10CAD0006C69627261726965732F5350492F5350AC
:10CAE000492E63707000535049436C6173733A3A36
:10CAF000535049436C617373284E52465F535049FB
:10CB00005F547970652A2C2075696E74385F742CB7
:10CB10002075696E74385F742C2075696E74385F87
:10CB2000742900000000000000000000697200008D
:10CB300021720000577200005D72000063720000F5
:10CB40005572000002000000030000000400000015
:10CB50001F0000001C0000000E0000002500000067
:10CB60000B0000000A000000090000001E00000089
:10CB7000170000000C000000110000000100000080
:10CB80000D00000022000000FFFFFFFFFFFFFFFF7E
:10CB90001A00000020000000150000001600000030
:10CBA0000F00000018000000130000002400000027
:10CBB000000000001400000005000000100000004C
:10CBC0000800000019000000280000000600000016
:10CBD00000000000000000004B780000417F0000D2
:10CBE000C1780000CD780000C778000049780000C7
:10CBF00041780000D5780000657800003D7800009D
:10CC000000C00140001002400020024000D002405D
:10CC1000000000000000304300000000000030C3AE
:10CC20007371727400000000FB21F93FFB21094081
:10CC30007CD91240FB2119407A6A1F407CD92240DE
:10CC4000BBFD2540FB2129403A462C407A6A2F4003
:10CC50005C4731407CD932409C6B3440BBFD354051
:10CC6000DB8F3740FB2139401BB43A403A463C4009
:10CC70005AD83D407A6A3F404C7E40405C47414034
:10CC80006C1042407CD942408CA243409C6B444093
:10CC9000AC344540BBFD4540CBC64640DB8F4740EA
:10CCA000EB584840FB21494083F9A200444E6E00F6
:10CCB000FC291500D1572700DD34F50062DBC000E8
:10CCC0003C999500419043006351FE00BBDEAB00F0
:10CCD000B761C5003A6E2400D24D42004906E0001B
:10CCE00009EA2E001C92D100EB1DFE0029B11C00A8
:10CCF000E83EA700F535820044BB2E009CE9840085
:10CD0000B4267000417E5F00D6913900538339000C
:10CD10009CF439008B5F840028F9BD00F81F3B00AC
:10CD2000DEFF97000F980500112FEF000A5A8B00C5
:10CD30006D1F6D00CF7E360009CB2700464FB70030
:10CD40009E663F002DEA5F00BA277500E5EBC7003D
:10CD50003D7BF100F739070092528A00FB6BEA0035
:10CD60001FB15F00085D8D00300356007BFC46005C
:10CD7000F0AB6B0020BCCF0036F49A00E3A91D0095
:10CD80005E619100081BE60085996500A0145F00B4
:10CD90008D40680080D8FF0027734D0006063100E3
:10CDA000CA561500C9A873007BE260006B8CC000F6
:10CDB00000000040FB21F93F000000002D44743EBC
:10CDC000000000809846F83C0000006051CC783BA1
:10CDD00000000080831BF0390000004020257A38D5
:10CDE000000000802282E336000000001DF3693558
:10CDF0000200000003000000040000000600000024
:10CE00002C2066756E6374696F6E3A2000617373CF
:10CE1000657274696F6E2022257322206661696CC9
:10CE200065643A2066696C6520222573222C206C8B
:10CE3000696E65202564257325730A006000002053
:10CE4000232D302B2000686C4C00656667454647F3
:10CE50000030313233343536373839414243444576
:10CE600046003031323334353637383961626364E5
:10CE700065660000000000000000000000000000E7
:10CE800000000000000000000000000000000000A2
:10CE90000000000000000000000000000000000092
:10CEA0000000000000000000000000000000000082
:10CEB0000000000000000000000000000000000072
:10CEC0000000000000000000000000000000000062
:10CED00000000000504F534958000020202020201F
:10CEE000202020202828282828202020202020201A
:10CEF000202020202020202020202088101010100A
:10CF0000101010101010101010101004040404045D
:10CF10000404040404101010101010104141414189
:10CF20004141010101010101010101010101010171
:10CF30000101010101011010101010104242424283
:10CF40004242020202020202020202020202020241
:10CF50000202020202021010101020000000000065
:10CF600000000000000000000000000000000000C1
:10CF700000000000000000000000000000000000B1
:10CF800000000000000000000000000000000000A1
:10CF90000000000000000000000000000000000091
:10CFA0000000000000000000000000000000000081
:10CFB0000000000000000000000000000000000071
:10CFC0000000000000000000000000000000000061
:10CFD0000000000000000000000000000000000051
:08CFE0006032FF7F0100000038
:10CFE800FFFFFFFFE803000001000000E803DC0585
:10CFF800DC05DC05DC050000FFFFFFFFFFFFFFFF8E
:10D008001800000019FCFFFFFFFFFFFF02000000EF
:10D0180040420F00FF0000000090D003FFFFFFFF19
:10D02800FFFFFFFFFFFFFFFFFFFFFFFF0A000000FA
:10D03800010000000800000001000000600000205E
:10D048000000000094CE0000B4CE000074CE0000B2
:10D0580000000000000000000000000000000000C8
:10D0680000000000000000000000000000000000B8
:10D0780000000000000000000000000000000000A8
:10D088000000000000000000000000000000000098
:10D098000000000000000000000000000000000088
:10D0A8004300000000000000000000000000000035
:10D0B8000000000000000000000000000000000068
:10D0C8004300000000000000000000000000000015
:10D0D8000000000000000000000000000000000048
:10D0E80043000000000000000000000000000000F5
:10D0F8000000000000000000000000000000000028
:10D1080043000000000000000000000000000000D4
:10D118000000000000000000000000000000000007
:10D1280043000000000000000000000000000000B4
:10D1380000000000000000000000000000000000E7
:10D148004300000000000000000000000000000094
:10D1580000000000000000000000000000000000C7
:10D168004300000000000000000000000000000074
:10D1780000000000000000000000000000000000A7
:10D18800DBB40000A9AE000000000000DACE000009
:10D1980012B70000B2BB0000B2BB0000B2BB000077
:10D1A800B2BB0000B2BB0000B2BB0000B2BB0000C3
:10D1B800B2BB0000B2BB0000FFFFFFFFFFFFFFFF95
:10D1C800FFFFFFFFFFFF00000100415343494900F3
:10D1D8000000000000000000000000000000000047
:10D1E80000000000000000000000415343494900CE
:10D1F8000000000000000000000000000000000027
:10D2080000000000000000000000000025020000EF
:10D21800ED71000049760000D57A00000102000097
:04000003000077057D
:00000001FF
